:100000000080001039010000314100003141000042
:10001000314100003141000031410000000000008A
:10002000000000000000000000000000314100005E
:10003000314100000000000031410000314100006A
:1000400031410000314100003141000031410000E8
:1000500031410000314100003141000031410000D8
:1000600031410000314100003141000031410000C8
:1000700031410000314100003141000031410000B8
:1000800031410000314100003141000031410000A8
:100090003141000031410000314100003141000098
:1000A0003141000031410000314100003141000088
:1000B0003141000031410000314100003141000078
:1000C00031410000000000000000000000000000BE
:1000D0000000000000000000000000000000000020
:1000E0000000000000000000000000000000000010
:1000F0000000000000000000000000000000000000
:10010000FFFFFFFFFFFFFFFF73643269656320316C
:100110002E302E30414C504841302D39382D47413A
:100120004138333935432D6C7063313736382D61A2
:10013000726D326965633100024803498860416825
:0C014000084700000040000000ED00E057
:104000000080001009410000314100002D0801002E
:1040100039080100450801005108010000000000B6
:10402000000000000000000000000000314100001E
:10403000314100000000000031410000CD1B0100B3
:1040400031410000D1070100B507010031410000F6
:10405000314100005D0801003141000031410000A4
:1040600031410000314100003141000009010100EF
:104070003141000031410000314100003141000078
:104080003141000031410000314100003141000068
:1040900031410000E90701003141000031410000D9
:1040A0003141000031410000314100003141000048
:1040B0003141000031410000314100003141000038
:1040C000314100000000000000000000000000007E
:1040D00000000000000000000000000000000000E0
:1040E00000000000000000000000000000000000D0
:1040F00000000000000000000000000000000000C0
:10410000FFFFFFFFFFFFFFFF0A480B490B4A50F874
:10411000043B42F8043B8842FFF4F9AF08480949E0
:10412000094A40F8042B8842FFF4FBAF0CF0B4BE00
:10413000FFF7FEBF5C2801007C2801000000001092
:1041400020000010981B0010000000004FF0080233
:104150004FEA01614FEA4000490001D380F080003E
:1041600010F0800F01D080F00900013A7FF4F2AF27
:10417000C0B270470FF2400C11F8013B83EA1023E4
:104180003CF8133083EA002080B2013A7FF4F4AFA8
:10419000704709A281EA102132F8113083EA002029
:1041A00080B270470FF2102281EA0001C9B232F8E2
:1041B000113083EA10207047000021104220633044
:1041C0008440A550C660E770088129914AA16BB16F
:1041D0008CC1ADD1CEE1EFF1311210027332522217
:1041E000B5529442F772D662399318837BB35AA3BF
:1041F000BDD39CC3FFF3DEE36224433420040114E7
:10420000E664C774A44485546AA54BB5288509950E
:10421000EEE5CFF5ACC58DD55336722611163006B6
:10422000D776F6669556B4465BB77AA7199738875E
:10423000DFF7FEE79DD7BCC7C448E5588668A77876
:104240004008611802282338CCC9EDD98EE9AFF9AE
:10425000488969990AA92BB9F55AD44AB77A966A56
:10426000711A500A333A122AFDDBDCCBBFFB9EEBFE
:10427000799B588B3BBB1AABA66C877CE44CC55C26
:10428000222C033C600C411CAEED8FFDECCDCDDD4E
:104290002AAD0BBD688D499D977EB66ED55EF44EF6
:1042A000133E322E511E700E9FFFBEEFDDDFFCCF9E
:1042B0001BBF3AAF599F788F8891A981CAB1EBA1F2
:1042C0000CD12DC14EF16FE18010A100C230E3206E
:1042D0000450254046706760B9839893FBA3DAB316
:1042E0003DC31CD37FE35EF3B1029012F322D232BE
:1042F0003542145277625672EAB5CBA5A8958985E6
:104300006EF54FE52CD50DC5E234C324A01481040D
:104310006674476424540544DBA7FAB79987B897B5
:104320005FE77EF71DC73CD7D326F2369106B0165D
:1043300057667676154634564CD96DC90EF92FE975
:10434000C899E9898AB9ABA94458654806782768AD
:10435000C018E1088238A3287DCB5CDB3FEB1EFB55
:10436000F98BD89BBBAB9ABB754A545A376A167AFD
:10437000F10AD01AB32A923A2EFD0FED6CDD4DCD25
:10438000AABD8BADE89DC98D267C076C645C454C4D
:10439000A23C832CE01CC10C1FEF3EFF5DCF7CDFF5
:1043A0009BAFBABFD98FF89F176E367E554E745E9D
:1043B000932EB23ED10EF01E0000C1C081C140015B
:1043C00001C3C003800241C201C6C006800741C7C5
:1043D0000005C1C581C4400401CCC00C800D41CD95
:1043E000000FC1CF81CE400E000AC1CA81CB400B65
:1043F00001C9C009800841C801D8C018801941D935
:10440000001BC1DB81DA401A001EC1DE81DF401FC4
:1044100001DDC01D801C41DC0014C1D481D54015D4
:1044200001D7C017801641D601D2C012801341D3E4
:104430000011C1D181D0401001F0C030803141F174
:104440000033C1F381F240320036C1F681F74037C4
:1044500001F5C035803441F4003CC1FC81FD403D94
:1044600001FFC03F803E41FE01FAC03A803B41FB64
:104470000039C1F981F840380028C1E881E94029B4
:1044800001EBC02B802A41EA01EEC02E802F41EFC4
:10449000002DC1ED81EC402C01E4C024802541E5D4
:1044A0000027C1E781E640260022C1E281E34023E4
:1044B00001E1C021802041E001A0C060806141A1F4
:1044C0000063C1A381A240620066C1A681A74067C4
:1044D00001A5C065806441A4006CC1AC81AD406D94
:1044E00001AFC06F806E41AE01AAC06A806B41AB64
:1044F0000069C1A981A840680078C1B881B9407934
:1045000001BBC07B807A41BA01BEC07E807F41BFC3
:10451000007DC1BD81BC407C01B4C074807541B5D3
:104520000077C1B781B640760072C1B281B34073E3
:1045300001B1C071807041B00050C1908191405173
:104540000193C053805241920196C05680574197C3
:104550000055C19581944054019CC05C805D419D93
:10456000005FC19F819E405E005AC19A819B405B63
:104570000199C059805841980188C04880494189B3
:10458000004BC18B818A404A004EC18E818F404FC3
:10459000018DC04D804C418C0044C18481854045D3
:1045A0000187C047804641860182C04280434183E3
:1045B0000041C18181804040032A70B414D940EA8F
:1045C00001039B0711D10C46034625681E6821464E
:1045D000AE42184604F1040403F1040304D1043A82
:1045E000032A18462146F0D8C2B105780C78A542B6
:1045F00004BF02F1FF32002306D00CE010F8015F87
:1046000011F8014FA54206D1934203F10103F5D100
:10461000002070BC7047281B70BC70471046F8E73C
:104620000F2AF0B443D940EA01039B0743D1A2F11A
:1046300010073F0900EB071610360C4603462568A5
:10464000103343F8105C6568103443F80C5C54F880
:10465000085C43F8085C54F8045C43F8045CB3421B
:10466000EDD17B1C02F00F0C1B01BCF1030F1944B0
:10467000034422D90E461D46644656F8047B043C8A
:10468000032C45F8047BF8D8ACF1040424F00304AF
:10469000043402F003022344214432B10A4411F8E5
:1046A000014B914203F8014BF9D1F0BC704703462E
:1046B000002AF3D1F9E70346F0E76246002AEDD17C
:1046C000F3E700BFF0B4840743D0541E002A3ED065
:1046D000CDB2034603E0621E002C38D0144603F826
:1046E000015B9A07F7D1032C2AD9CDB245EA0525FB
:1046F0000F2C45EA054515D9A4F110073F0903F130
:10470000100606EB07161A46156055609560D560D1
:104710001032B242F8D104F00F040137032C03EB3E
:1047200007130DD91E462246043A032A46F8045BB5
:10473000FAD8221F22F003020432134404F00304C7
:104740002CB1C9B21C4403F8011BA342FBD1F0BC3D
:10475000704714460346C6E7C9B2F0B4002947D0F3
:1047600085070FD00278002A3FD091423ED0431CEB
:1047700005E013F8012B002A37D0914236D09A0772
:104780001846F6D1036841EA012747EA074783EA5A
:104790000702A2F10135A3F1013425EA020224EA5D
:1047A0000303134313F0803F11D1021D104652F84A
:1047B000043B83EA0704A4F10136A3F1013526EA9C
:1047C000040425EA0303234313F0803FEED003786B
:1047D000002B39D0994209D0431C01E0914205D009
:1047E000184613F8012B002AF8D11046F0BC704788
:1047F00084070BD00378002BF8D0431C03E0027829
:104800000133002AF2D099071846F8D10368A3F1C2
:10481000013222EA030313F0803F0AD1031D184638
:1048200053F8042BA2F1013121EA020212F0803F79
:10483000F5D00378002BD9D0431C1A7818460133E1
:10484000002AFAD1F0BC70471846CFE780EA01028F
:10485000844612F0030F4FD111F0030F32D14DF8FF
:10486000044D11F0040F51F8043B0BD0A3F10132B9
:104870009A4312F0803F04BF4CF8043B51F8043BCC
:1048800016D100BF51F8044BA3F101329A4312F044
:10489000803FA4F101320BD14CF8043BA24312F04B
:1048A000803F04BF51F8043B4CF8044BEAD0234648
:1048B0000CF8013B13F0FF0F4FEA3323F8D15DF8FA
:1048C000044B704711F0010F06D011F8012B0CF8C2
:1048D000012B002A08BF704711F0020FBFD031F83A
:1048E000022B12F0FF0F16BF2CF8022B8CF80020C1
:1048F00012F47F4FB3D1704711F8012B0CF8012B44
:10490000002AF9D1704700BF20F0030110F0030026
:10491000C0F1000051F8043B00F1040C4FEACC0C4C
:104920006FF000021CBF22FA0CF213434FF0010C8F
:104930004CEA0C2C4CEA0C4CA3EB0C0222EA0302CE
:1049400012EACC1204BF51F8043B0430F4D013F047
:10495000FF0F1FBF013013F47F4F013013F47F0F9F
:1049600018BF0130704700BF40EA01039B0770B4D5
:104970002BD1032A84BF0C46034626D9214654F87E
:10498000045BA5F1013626EA050616F0803F05D145
:10499000043A032A43F8045B2146EFD89AB10C7815
:1049A000013A1C7001333CB16AB111F8014F013A70
:1049B00003F8014B002CF7D12AB11A44002103F867
:1049C000011B9342FBD170BC70470346E6E700BF72
:1049D00038B502460C46002511B909E0421C0546CF
:1049E00010462146FFF7B8FE0028F7D1284638BD0B
:1049F000BDE83840FFF7B0BE0020704738B50B4B1C
:104A0000482404FB0034217B41F3000161B9201DDF
:104A10004422FFF757FE237B43F0010323736423F3
:104A2000A371034B6361A36138BD00BF2413001061
:104A3000F949000070B500214FF490621048FFF76B
:104A400041FE104D0E490022482606FB02F005EB00
:104A5000022401320F2A0A4B4450F6D183F83E2437
:104A600093F84424084942F02D0283F84424074A6D
:104A7000C3F83814C3F84C24054AC3F8502470BD59
:104A800024130010200000100E1900102D920000B9
:104A9000F94900000A4A38B54821002301FB0324E4
:104AA000257BD8B2ED0703D4FFF7A8FF204638BD19
:104AB00001330F2BF2D1462004F0B4FB002038BDA7
:104AC0002413001008B5FFF7E5FF40B10023837100
:104AD000034B1A7801321A70024B01221A6008BD8A
:104AE000C5170010B40B38232DE9F74F00232C49CC
:104AF00007461C461A46482000FB0316367BDDB2EB
:104B000016F0010FDFF8988007D1002A08BF2C4665
:104B10000132D2B2BA4201D105E0002201330F2B9B
:104B2000EAD1BA420BD3482303FB048304EB070A00
:104B300003F106095FFA8AFB26461A4604E046207E
:104B400004F070FB002027E05E4509F1480517D00E
:104B500030460192FFF752FF124B01361978F6B238
:104B600001311970002305F8483C09F1420345F86A
:104B70002A3C019AA94645F82E2C05F8317CE3E73A
:104B8000094B012248200AF1FF3A1A6000FB0A8310
:104B900000FB048000225A6203B0BDE8F08F00BF22
:104BA00024130010C5170010B40B3823B0B182795C
:104BB0000F2A13D0037BD90710D56FF300030373BB
:104BC000DB0603D5064B197810391970632A03D810
:104BD000034B1A78013A1A700AF036BB704700BFCF
:104BE000C517001010B50446836998472046BDE8F4
:104BF0001040FFF7DBBF00002DE9F84F1A4D0024ED
:104C0000A5F10608074626464FF04809C24609FBAB
:104C100004831B7BD9071ED5BA0702D42B78632BDC
:104C200019D87B0704D409FB04A31B7B580612D4B4
:104C300017F0010FA5F1060B0AD03EB9D5F81230D6
:104C400058469847003018BF012000E00120C6B246
:104C50005846FFF7ABFF01340F2C05F14805D6D1BC
:104C60003046BDE8F88F00BF2A130010094930B55F
:104C70000023482404FB0312157BED0704D5957926
:104C8000854201D1104630BD0133102BF2D10020F6
:104C900030BD00BF24130010037BDA0609D443F0B3
:104CA00010030373034B1A7810321A70024B01225F
:104CB0001A607047C5170010EC033823037BD90630
:104CC0000CD5074A6FF3041303731378103BDBB260
:104CD00013701B0902D1034B01221A60704700BFF9
:104CE000C51700106C03382330B51E4C702505FB2A
:104CF000004090F860004B1E00F07F000128DBB2FE
:104D00002BD0042825D0222B83BFA1F12403DBB2B2
:104D100040F2AB200020102B02D80244152019E0ED
:104D2000172B05D802F265120244113B132006E04E
:104D30001D2B08D802F5F5720244183B122000FB27
:104D4000032080B230BD02F2562202441E3B1120E5
:104D5000F5E7282000FB032030BD02EB032398B2C7
:104D600030BD00BFC419001008B5FFF7BDFF000239
:104D700008BD0000064B1B681B689870C043D870C4
:104D80000A781A714A785A71C0229A71704700BF26
:104D9000280F001008B51F2004F044FA012008BDB8
:104DA0001F2004F03FBA2DE9F3414FF48076054609
:104DB000884617461846324600211C46FFF782FCFB
:104DC000FF23637041463A462846FFF7CDFF002394
:104DD0000146009328462246334607F02FF902B0D9
:104DE000BDE8F08173B50A780B460270097A044673
:104DF00001715A7A702642710020A0711D780D4B06
:104E000006FB053393F86060012E11D12846FFF7A9
:104E1000ABFF01AA01460223284607F0E7F808B1D4
:104E2000304605E09DF8043023719DF8053063712C
:104E300002B070BDC41900102DE9F0411E46104BA0
:104E4000702707FB0030071DFB780D460B44184602
:104E50009046A0211922FFF735FC0024034618F8DC
:104E6000041021B1102C02D019550134F7E73B7919
:104E70003168EA18E95033791371BDE8F08100BF59
:104E8000241A0010104B702202FB003090F86030A2
:104E900003F07F03012B14D0042B01D1282070478D
:104EA000232984BF2339C9B2112906D9182906D963
:104EB0001E298CBF11201220704715207047132027
:104EC00070474FF480707047C41900102DE9F04707
:104ED000044616469946BDF820809DF824A00D464C
:104EE00051B170274743404B3B449B788B4203D3DF
:104EF000FFF7C8FF864201D350465AE03B4B1F44A0
:104F000097F860A01AF0800F5ED0394F3B78A3422B
:104F100002D17B78AB4244D0012136482822FFF7EA
:104F2000D1FB0AF07F0103291BD004292AD00229D2
:104F300057D1294600222046FFF7D6FE2946824651
:104F40002046FFF79FFF0AF52A31034601F540711D
:104F50002046284A07F04AF8012842D83C707D7064
:104F60001FE0294600222046FFF7BEFE2946824662
:104F70002046FFF787FF0AF5AA21034601F5C06125
:104F80002046E6E7294600222046FFF7ADFE2946E7
:104F900082462046FFF776FF0AF548210346204661
:104FA000D7E73744B878831EDBB2092B06D8123016
:104FB000C0B22946324604F053F812E00F2803D15C
:104FC0004A2004F02FF90CE0294632462046FFF72C
:104FD000CBFE4A46014643462046BDE8F04707F06F
:104FE00005B80220BDE8F087281A0010C419001087
:104FF000C6170010C817001037B503684FF4807546
:105000001A784FF0430E80F820205A78044680F832
:1050100021201978C07F5A788DE82040FFF756FF8D
:1050200020B12046FFF7C2FD012011E002232168D4
:1050300063710A78237B32B9497843F020032171E8
:105040002373104604E0FF2260F34513227123739B
:1050500003B030BD13B54FF0420C04464FF48070DE
:105060008DE80110084611461A462368FFF72EFF07
:1050700002B010BD37B50446007B40F34000C0B11C
:105080000D4B257F1B78AB4212D9617FA27F28464A
:10509000FFF76AFE01230146009328464FF4807310
:1050A000226806F0CBFF237B6FF34103237300E0FC
:1050B000002003B030BD00BFC1190010F7B507468E
:1050C0000D461E46144662B1124B702202FB01339C
:1050D0009B78A34205D308462146FFF7D3FE8642BC
:1050E00007D342202146324603B0BDE8F04003F02A
:1050F000B7BF214632462846FFF736FE012300930C
:1051000001463A6828464FF4807306F097FF03B0D3
:10511000F0BD00BF281A001007B568460CF036FA3B
:105120009DF805106422B1FBF2F002FB1012094B4E
:105130005A769DF8042001329A769DF80320DA769B
:105140009DF802201A779DF801205A7703B05DF888
:1051500004FB00BFA417001070B50C4662780978F4
:105160000546FFF701FEA178044A00EB4111202318
:105170002846BDE8704006F039BF00BFA4170010F4
:1051800073B51D4A0678702505FB062292F860501B
:105190000446012D02D006F01DFF2AE0087810B960
:1051A0002572657225E00A8830465F2A16D1217A79
:1051B000627AFFF7D9FD01AA00F1220102233046ED
:1051C00006F014FFA0B99DF804301BB9207806F052
:1051D000DBFE0EE023729DF8053007E01C31FFF77F
:1051E000BBFF28B9054BDA7822721B79637200E0A5
:1051F000284602B070BD00BFC4190010A4170010EB
:10520000F7B583790446082B11D11C4D02234326A0
:10521000007821798DE8480062792B46FFF756FE29
:10522000D8B92B782BB323716B78A0716371257972
:1052300067796DB12678124B702202FB06339B789A
:10524000AB4205D330462946FFF71CFE874206D302
:10525000432029463A4603F003FF01200AE0304686
:10526000211DFFF779FF0028F7D1A3790133A3713E
:1052700000E0FF2040B203B0F0BD00BFA417001053
:10528000281A001038B51C31054600781446FFF77F
:1052900063FFA8B90B4B2268D978204611701B799F
:1052A000226853702B78084AE377237B6261074AB0
:1052B00043F0440322612373BDE83840FFF79CBEEE
:1052C00038BD00BFA4170010F94F0000954D000035
:1052D00073B50C461546097862780646FFF744FD1B
:1052E000A178009500EB4111034A3046202306F0D7
:1052F000A5FE02B070BD00BFA417001073B503680F
:1053000000221A700368027904465A70438C90F8A0
:105310002010013390F821204384A1B1C67F0125DC
:105320003046FFF721FD00950146226830464FF4D4
:10533000807306F083FE30B904F11C06E07F31462D
:10534000FFF70AFF08B1012018E00D4B9A7862F0D0
:105350007F029A70628C9A77120ADA77FFF7DCFE86
:105360002A46E07F3146FFF7B3FF05460028EAD121
:10537000044B2046A361FFF719FC284602B070BD1C
:10538000A4170010F9490000F8B501F11C04054606
:10539000214600781746FFF7DFFE0646A8B90B48FE
:1053A000A0211022FFF78EF9094833460133FA187D
:1053B00012F8011C11B11A181171F7E7287821466B
:1053C0000122BDE8F840FFF783BFF8BDA917001020
:1053D000A41700102DE9F0411F460478184B9046A1
:1053E000702202FB043393F860300646012B0CBF99
:1053F000427A00220D462046317AFFF7B5FC702331
:1054000003FB04880F4B08F1600818F803102A46C4
:1054100001443B46204606F0E9FD58B97B1EDBB24D
:105420002022E95CA02908BFEA54013BDBB2FF2B34
:10543000F7D102E00120BDE8F0810020BDE8F08155
:10544000C4190010C819001004220523FFF7C2BFB9
:1054500003221023FFF7BEBF174A30B50C46702158
:1054600001FB002292F8605085B0012D06D14FF467
:1054700082712246102306F0B9FD0BE0303204ABF6
:105480008DF8040092E8030003E9030001A8214617
:10549000FFF7DEFF08B101200CE00022227404F1C6
:1054A0000F03A34205D013F80119202901D15A7026
:1054B000F7E7002005B030BDC4190010F8B5364F2D
:1054C00006460C463046FFF79BFE0146002860D199
:1054D000BB78314D002BF5D030222046FFF7F2F893
:1054E0000423E376AB7883F0800303F00702072AF6
:1054F00008BF23F0070363747368A383C3F30743F0
:10550000013BA377EA7FAB7F03EB02236382FF2398
:105510002375224B224603F1100153F8040B8B42F2
:1055200042F8040BF9D10F230022E15CA02908BF47
:10553000E254013BDBB2FF2BF7D16A7F3C23B2FB85
:10554000F3F103FB112363762A7F1823B2FBF3F1F7
:1055500003FB11232376EA7E1F23013A92FBF3F12A
:1055600003FB11230133E375AA7E0C23013A92FB5E
:10557000F3F103FB11230133A3756B7E6422B3FBAC
:10558000F2F102FB1133DBB24F2B98BF643363752A
:10559000002040B2F8BD00BFA4170010A9170010EA
:1055A0002DE9F84F9A464D4B8046702000FB08339A
:1055B00093F8605005F07F05032D04D0042D16D01C
:1055C000012D0CD120E0232909D92AB924394D43D2
:1055D0001446EFB235251CE04739CFB204E08F0006
:1055E000002A08BF0137FFB20024122511E0282944
:1055F00036D801240627002A14BF0A220B2207FBF3
:1056000001212825CFB204E0CC0801F007010234C3
:105610004F01334B1A689946117F414505D1537F9D
:10562000AB4202D1937FA34211D0DFF8BCB0DBF8CC
:105630000030CBB1CBF800201A7FC9F800304245CA
:1056400029D15A7FAA4226D19B7FA34223D1D9F8E0
:105650000030002019680F44CAF80070BDE8F88FC8
:105660002839C9B20224C5E7FF2914D0FFF712FA7E
:10567000CBF8000060B365238371FF230377194BD8
:105680008361037B43F040030373D9F80030C9F80A
:105690000000CBF80030D9F80000114E836998471C
:1056A00098B9294622464046FFF75EFB336801461B
:1056B0001A6840464FF4807306F098FC58B9336876
:1056C00083F81C805D779C77C1E70120BDE8F88FE7
:1056D00003F0A8FDDFE7BDE8F88F00BFC419001094
:1056E000280F001075500000240F001037B5144625
:1056F00002AB002243F8042D0546FFF751FFD8B94D
:105700000F4B702202FB053595F86030019A012B92
:105710004FEAD40304F0070408D1802040FA04F4CF
:10572000D35C23420CBF0020012006E0D05C40FA8D
:1057300004F404F0010000E0FF2040B203B030BDEB
:10574000C4190010F7B504460D461646FFF7CEFF04
:1057500000283EDB3ED020462946002201ABFFF761
:105760001FFF002835D11C4F3B681A7B42F0020214
:105770001A731A4B702202FB043393F86030F2085C
:10578000012B06F00706019B08D1802141FA06F69D
:10579000D2B2995C21EA06069E541BE0D1B20122E6
:1057A00002FA06F6585C20EA06065E5420462946B0
:1057B00001ABFFF7F5FE60B9019A13783BB1013BED
:1057C00013703B681A7B42F002021A7302E018461B
:1057D00000E0012003B0F0BD280F0010C419001034
:1057E0002DE9F34705460C4692461F4600263246F1
:1057F000013628460121F6B2FFF7A4FF232EF6D189
:1058000048203946FFF7B6FA1F4A702101FB0522EE
:105810001E4B92781B6800211B6801261A72D4F86F
:1058200000804FF480724046FEF74CFF4FF0220993
:105830004823312288F8023088F8006088F8019007
:10584000FA703B712846216852463B46FFF7F4FA4E
:1058500023684FF4807183F820602368284683F81A
:1058600021600023009322680B4606F0E7FB40B955
:105870002368284631464A4602B0BDE8F047FFF7A4
:1058800092BA02B0BDE8F087281A0010280F001065
:105890002DE9F0470446194D89469246122100220F
:1058A0001E46FFF74FFF204612210122FFF74AFF55
:1058B0002B684FF012081B680127412183F80080F4
:1058C0005F7099703223F3702B683171204619682C
:1058D00052463346FFF7B0FA2A68A02311682046E3
:1058E00081F8A9301268414682F8AA30D9F8003010
:1058F0003A46BDE8F047FFF756BA00BF280F001040
:1059000038B50546FFF7C4FF074B80221B6800240B
:105910001B68DA702246013428463521E4B2FFF7CD
:1059200011FF132CF6D138BD280F001037B5002217
:10593000019209B9002038E0702404FB00F31C4CEC
:105940001C44A4788C42F5D31A4A134493F860207F
:1059500002F07F02012A1ED101ABFFF721FE0028D1
:10596000E8D1019D03462A5C0130510801F0550140
:1059700002F055021144C9B28A0801F0330402F062
:105980003302224402F00F0101EB121213442028CB
:105990009BB2E8D108E0012201ABFFF701FE00282D
:1059A000C8D1019B187800E0184603B030BD00BF95
:1059B000281A0010C41900102DE9F34704460F46B9
:1059C00091461D4600263246013620462821F6B271
:1059D000FFF7B8FE042EF6D1264E4FF028083368A4
:1059E00002221B68442083F80080336829461B6824
:1059F0004FF0000A5A70FFF7BDF929212046FFF742
:105A000095FF3368FF221B68442083F800A03368A9
:105A100029461B685A70FFF7ADF9336803261A7BD5
:105A2000204642F002021A733B6844229A7083F8BF
:105A300000805E703323EB702A7139684A462B462A
:105A4000FFF7FAF9CDF800A020464FF4C3213A68D9
:105A50004FF4807306F0F2FA40B93B6820464146A5
:105A6000324602B0BDE8F047FFF79DB902B0BDE88D
:105A7000F08700BF280F00102DE9F047154670226F
:105A800042435D4B0C46991891F860100746012976
:105A90009A4626782BD102F1600831463846FFF746
:105AA00045FF217870B9554B013643449B78F6B2D7
:105AB000B34203D0002E08BF012600E00126B14208
:105AC000EBD124E0B1420CBF95F800804FF0000804
:105AD000384631464246FFF709FE20B908F1010871
:105AE0005FFA88F8F4E7267085F8008080E060327D
:105AF0001344197903F10408B1420ED1FFF716FFE0
:105B000040B93F4B1B7813B9482003F08BFB0120B1
:105B1000BDE8F08798F8069001E098F805907023AA
:105B200003FB07AA0026022E2FD838462178FFF75C
:105B3000FDFE60BB237898F800209A4201D9013B12
:105B40000BE05A1CD2B222709AF8601001F07F016B
:105B5000032903D1352A01D102332370237833B9C5
:105B600098F80020013601322270F6B22B702278AC
:105B700098F802309A42D6D998F800300136013BA5
:105B8000237000232B70F6B2CDE7032EB9D02E7808
:105B900038464E44F6B22E702178FFF773F98642EC
:105BA00005D3361AF6B22E700EB1013E2E70632662
:105BB0004FF00009384621782A78FFF797FD002832
:105BC00014DC013EF6B2FF2E12D095F80080384664
:105BD00008F101085FFA88F885F800802178FFF75E
:105BE00051F9804528BF85F80090E3E7002E88D062
:105BF0000020BDE8F08700BFC4190010C8190010CC
:105C0000721900102DE9F74F06460C46084631463A
:105C1000FFF7E8F84B4D2046FFF7F2FA002828DCA2
:105C200006D1A8780028F6D1A379013BA37185E0BD
:105C300004F1040830784146621D94F804A094F8F9
:105C400005B0FFF719FF074698B93E4D2379514635
:105C50002B7063795A466B7096F800904846FFF7B0
:105C600083F8009701462A464846022306F0E6F9E3
:105C700008B1012062E0307821796279FFF762FD96
:105C80000028F6D13778304B702202FB073393F8A7
:105C90006090B9F1010F08D02A4800212022FEF7B8
:105CA00011FDFF236B70002737E0317A727A384696
:105CB000FFF75AF82A4600F124010323384606F07C
:105CC00095F90028D5D129780029E5D037786A7868
:105CD0003846FFF749F8A978EA1C1C310144022331
:105CE000384606F083F90028C3D1B5F80330297887
:105CF0000133A5F8033037786A783846FFF734F86F
:105D0000A978CDF800901C310144EA1C38460223E2
:105D100006F094F90028BFD0ABE7A7713078414670
:105D20000022FFF7D5FA0028A3D10137FFB2082FD0
:105D30006870F2D1034BFF225A70A07103B0BDE826
:105D4000F08F00BFA4170010C4190010F0B590F830
:105D5000203085B08DF80E3090F8213000258DF878
:105D60000F30438C04460133438403680DF10E0168
:105D70001D70027903685A70C07F0DF10F02FFF7A2
:105D80007BFE20B1224B8DF80E501D7813E0236866
:105D90009DF80E201A7023689DF80F209DF80E10B4
:105DA0005A70E07FFFF7CEFC20B12046FEF7FEFEE2
:105DB00001202AE00546E77F94F8201094F821207E
:105DC0003846FEF7D1FF0126014600963846226884
:105DD0004FF4807306F032F90028E6D19DF80E30BA
:105DE000267184F820309DF80F3084F8213002238A
:105DF0006371237B60F3410323732046FEF75EFF4C
:105E0000284615B103F00EFACFE705B0F0BD00BF8C
:105E1000721900102DE9F04170274743134B0646D5
:105E20000124002507EB030898F80230A34219D398
:105E30000F4B3B4493F8603003F07F03012B07D0F6
:105E4000042B01D1282C02E0122C07D0352C05D0D0
:105E500030462146FFF76AFD284485B2013414F02C
:105E6000FF04E1D12846BDE8F08100BF281A0010E8
:105E7000C41900102DE9F04F1C467F4E037892465E
:105E8000702202FB036393F83C3089B09B070746FE
:105E9000884601D41A2083E09DF8483083B1224619
:105EA000FFF7F0F9754D2B78002B40F0E180236867
:105EB0001B78002B00F08180636920469847F2E749
:105EC00002A9FFF79FFE0546002840F0D180294631
:105ED0001F226B48FEF7F6FB10226A48A021FEF74E
:105EE000F1FB694A2846013008EB000313F8013C36
:105EF000DFF8949113B111180B71F4E789F802A03F
:105F000097F80080702303FB08F3F21892F86020E2
:105F1000012A03D060330125334429E0022503F12F
:105F2000600640462946FFF701FD68BB574B013527
:105F300033449B78EDB2AB4203D015B1022DF0D1C2
:105F400096E00125EDE719795FFA85FACAEB0101C0
:105F50004046C9B20193FFF7E9FC019B70B9CAF151
:105F60000005EDB26AB2002AC4BFCAF10105EDB264
:105F70001E1DB2784FFA85FB9345E4DBB3789B4551
:105F800009D033785D1BEDB2002640462946FEF766
:105F900079FF864207D3394B1B78002B68D1482004
:105FA00003F040F964E0404629463246FFF79EFB85
:105FB000002831DC0136F6B2E7E7D8F81C20A283CE
:105FC000120CA277304A917FD27F013901EB022275
:105FD00021796284227B013163F38202C9B2227388
:105FE0006171D2B211B942F0020201E063F34102E1
:105FF000274B22736361274BA361274B2361237BCC
:1060000043F048032373FFF787F8E07F04F11C0196
:106010000122FFF75DF92BE089F8035089F804604D
:10602000387829463246FFF78DFB08BBFFF774F836
:10603000387803A90122FFF74BF9C8B9237B0D2259
:1060400043F048032373022363712371114BA3614F
:106050000F4B6361104B236123689A70039BA383EA
:106060001B0CA3773B7884F82050E37784F82160F9
:1060700009B0BDE8F08F00BFC419001072190010FC
:10608000A6170010A9170010A4170010C8190010B7
:106090004D5D0000FD520000954D00002DE9F743D5
:1060A000164604460D46FFF721FB021E42DB43D194
:1060B0002046294601ABFFF773FA00283AD1204F5A
:1060C0003B681A7B42F002021A731E4B702202FBDD
:1060D000043393F86030F208012B06F00706019BA9
:1060E00007D1802141FA06F6D2B2995C0E439E5444
:1060F00023E0D1B2012202FA06F6585C06435E5450
:106100002046294601ABFFF74BFA98B920462946AD
:10611000FEF7B8FEDDF8048098F8009081450BD2B8
:1061200009F1010988F800903B681A7B42F00202ED
:106130001A7301E0012000E0002003B0BDE8F08305
:10614000280F0010C41900102DE9FF4101F11C05B2
:10615000044629460078FEF7FFFF08B1FF202AE039
:10616000164B0227DA781E468DF80C201A794FF06C
:1061700043088DF80D209DF80C109DF80D20207817
:10618000FFF78CFF20789DF80C109DF80D208DE80E
:10619000800103ABFEF79AFE0028DFD19DF80C20AA
:1061A000002AE8D1B270207829460122FFF790F842
:1061B0000028D3D1012004B0BDE8F081A41700105D
:1061C0002DE9F041844A03780E46702101FB032338
:1061D00093F860308AB0012B044601D01F201AE0EA
:1061E000FEF770FC0546002800F0F280204604A966
:1061F000FFF708FD002840F0EB80237A20788DF827
:106200000C30637A03A90DF10D028DF80D30FFF704
:1062100033FC18B1482003F005F8D9E020789DF848
:106220000C109DF80D20FFF78DFA002840F0D0806B
:106230009DF80C3020788DF80E309DF80D300DF162
:106240000E010DF10F028DF80F30FFF715FC50B164
:10625000482002F0E7FF20789DF80C109DF80D20F3
:10626000FFF71CFFB4E020789DF80E109DF80F207A
:10627000FFF768FA0746002840F0AA8039464FF435
:1062800080722868FEF71EFA286819220430A021BF
:10629000FEF718FA2B689DF80E2038461A709DF804
:1062A0000F205A7048229A702B689DF80C2083F8B2
:1062B00020209DF80D2083F82120227A83F82220C7
:1062C000627A83F823209DF8142083F824209DF817
:1062D000152083F825209DF816205201023283F8FC
:1062E00026202A680130331813F8017C17B11318DF
:1062F000DF70F7E72B6832789DF80C109A7572788A
:10630000DA7531225A7648229A7694F800809DF800
:106310000D204046FEF728FD009701462A684046BA
:106320004FF4807305F08AFE0746002850D1286894
:1063300039464FF48072FEF7C5F92B68FF225A7078
:1063400094F800809DF80E109DF80F204046FEF74F
:106350000BFD009701462A6840464FF4807305F014
:106360006DFE0546A0BB29461F221C48FEF7AAF970
:1063700010221B48A021FEF7A5F91A4A2846013031
:10638000331813F8013C174D13B111180B71F6E7D0
:106390008623AB709DF80C30EB709DF80D302B719F
:1063A0000223AB77FEF7B8FE24789DF814109DF811
:1063B00015202046FEF7D8FC9DF81610012300EBAF
:1063C0004111009320460231AA1C1E2305F036FE1F
:1063D0000AB0BDE8F08100BFC4190010A617001074
:1063E000A9170010A417001008B5064B186808B1CB
:1063F00083699847044B186808B18369984700205F
:1064000008BD00BF280F0010240F00102DE9F04F29
:106410001646634A702303FB00238A4693F86010F4
:106420008BB001290446904609D193F834203033CB
:10643000012A40F0B1805B79012B40F0AD80FEF77E
:1064400041FB0546002800F0A780037B43F00803CA
:106450006FF386130373FEF71FFC4FF48072002165
:106460002868FEF72FF9FFF7BFFF4E4BFF221B688E
:106470001A774D4B1B6803B11A77002E33D04B4B64
:10648000702202FB043301270393039A9378BB42E3
:1064900022D34FF0000B5FFA87F920464946FEF7FA
:1064A000F1FC834515D249465FFA8BF22046FEF790
:1064B0005BFC0022009201462A6820464FF480735C
:1064C00005F0BCFD002867D10BF1010C1FFA8CFB15
:1064D000E3E70137BFB2D8E733788DF8143073782B
:1064E0008DF815302CE0702707FB048797F864308F
:1064F00007A88DF8243005A901238DF81C406037CA
:106500008DF82530FEF7A0FF002845D13F79B14630
:1065100020463946FEF7B6FC864211D23946F2B221
:106520002046FEF721FCCDF8009001462A6820465F
:106530004FF4807305F082FD70BB0136B6B2E7E719
:1065400070276743A0238DF81630184B0126FB18DF
:106550000393039A9378B34217D34FF0000B5FFA7B
:1065600086F920464946FEF78DFC83450AD25FFA3C
:106570008BF220464946FFF791FD0BF101031FFA0C
:1065800083FBEEE70136B6B2E3E74744FE6E2046F2
:106590002946524605ABB0470BB0BDE8F08F00BFAF
:1065A000C4190010280F0010240F0010281A001022
:1065B0002DE9F041494E0778702303FB0763484AF1
:1065C0009C6C0546944224D00CD8464A944219D07B
:1065D000454A944232D1454A643307CA822483E84B
:1065E00007004CE0B4F5482F1AD0414A94421ED01F
:1065F000404A944222D1404A643307CA832483E844
:1066000007003CE0394A643307CA022483E80700E4
:1066100035E0394A643307CA032483E807002EE0D3
:10662000364A643307CA042483E8070027E0334A64
:10663000643307CA842483E8070020E0A3B21BB1B7
:106640004F2002F0EFFD43E0B4F5403F09D108468A
:106650002E21FEF7BDF98378362B02D1C378342B77
:10666000EED04FF0700C0CFB076C254A240C0CF19B
:10667000640307CA83E807008CF866400124DFF84A
:106680009080D8F8003073B9FEF704FAC8F800001B
:10669000F0B165228271FF2202771A4A8261027B81
:1066A00042F04002027370235F43F319603783F8AE
:1066B00060403E4433792B7273796B72124B1A78B7
:1066C00001321A70220606D5104BFF221A7002E022
:1066D0000120BDE8F0810020BDE8F081C419001060
:1066E0000056050000AB0200ABAD0200981E010091
:1066F000808C0C00565B05008C1E0100A41E01005E
:10670000B01E010075500000200F0010C6170010C9
:10671000280F001010B50B68027A70241A700378E5
:106720000D4A04FB032393F86030012B08BF427A23
:106730000B6818BF00225A700378084ACB770B7B8E
:106740004A61074A43F044030A610B730846BDE8F7
:106750001040FEF751BC00BFC4190010F94F0000F3
:10676000954D000038B5074D00242868FEF71EFA45
:106770002C60054D2868FEF719FA044B2C601C703C
:1067800038BD00BF280F0010240F0010200F00108C
:1067900070B5134D0646286838B1826990472B685A
:1067A0001A7FB24204BFFF221A770E4C206838B11C
:1067B0008269904723681A7FB24204BFFF221A778A
:1067C000094A1378013BDBB2137043B12868FEF726
:1067D000EDF92068FEF7EAF900232B60236070BD15
:1067E000280F0010240F0010200F00101B4A012357
:1067F0001360C2F8C8371A4B19680A311A68521A5E
:10680000002AFBDB174901220A60C1F8C827144A95
:1068100011680A311A68521A002AFBDBC10705D435
:10682000820707D5104A0121116003E00B4A0121BC
:106830001160F5E719680A311A68521A002AFBDB61
:10684000084901220A60C1F8C827054A11680A31BF
:106850001A68521A002AFBDB704700BFEC0338238A
:10686000941B00106C033823B40B38232DE9F74F29
:10687000544F0025052097F800903D70FEF7BCF9B5
:10688000514B524F1A78AA4642F020021A702E46F7
:106890002C4698463B78A34255D34D48514606F0C6
:1068A0009DFD38B94A484B49F9220DF1060306F01F
:1068B00013FC18B1012104F091FB7CE0BDF8063017
:1068C000F82B02D9444B002513E042495854002BC1
:1068D000F8D13A789A46FF2A06BF04F1FF343C709B
:1068E0003B70FF242CE00A2B07D03A2B08BF012570
:1068F00033465E1C5B780D2BF5D1324601E00A2B46
:1069000006D1137893460D2B02F10102F7D1F8E777
:10691000BAF1000F0DD12F4830490822FDF74CFE87
:1069200038B998F80030013C23F0200388F8003093
:10693000E4B2284BC3EB0B0B0AEB0B0C1FFA8CFADF
:106940000134E4B2A6E7264A002333701078254BC1
:10695000702101FB00318C6B23491E468C4214468A
:1069600001D005F011FB2278204B1A70702303FB35
:1069700002631F4A303392E8030083E8030035B90D
:10698000154C63782F2B04D03A23237002E0114C6E
:1069900000E0013498F80030980602D520460BF04C
:1069A000D4F9204600F0BCFA064A13782BB1492BE3
:1069B00003D082F80090002000E0012003B0BDE881
:1069C000F08F00BF72190010F3170010380F00107D
:1069D0003C0F0010FB170010FA170010091F0100F0
:1069E0002C0F0010C419001074240100C0190010ED
:1069F000300F0010F8B51F4B16461A781E4D22F0C6
:106A000004021A706B6804460F463BB1284606F034
:106A1000DEFC284600212422FDF754FE3B783BB3E0
:106A2000164B2078702202FB00306168816120786B
:106A3000114902FB00303A46012306F07FFA20B1EB
:106A40000121BDE8F84004F0C9BA0D4B94E80700F5
:106A500083E807000B4B16B1FF221A7000E01E708E
:106A6000FFF704FF20B10320BDE8F840FFF7BEBEEA
:106A7000F8BD00BFF31700103C0F0010C419001040
:106A80002C0F0010380F00100022FFF7B3BF0000DA
:106A90002DE9F043714BA1B05A681F46704C002A93
:106AA00040F0A7806F497048FDF7D0FE6F4B702112
:106AB0001A786F4B03AD01FB0231303103C985E811
:106AC0000300217820AD05F8782D01F0020101F0D6
:106AD000FF02654E9846284611B13146012200E07A
:106AE0003146FFF787FF7B68002B79D123785A075F
:106AF00072D5604905A8FDF7A9FE9DF8080070272A
:106B000007FB0080039909AA06F0EEFC002863D178
:106B1000574B9DF8080017A907FB003005AA0A2368
:106B200006F00CFA002857D1534B01221A60074691
:106B300016960DF1480809A80EA906F0EFFC0028EA
:106B400039D19DF84830002B35D09DF84030DB0618
:106B5000F1D4404604F0DCFE02288146EBD1424BE2
:106B60003778002F0CBF47461F463846FDF7CCFE4E
:106B7000394682B20DF1060317A806F045FB08B1AD
:106B8000012718E0BDF80630002BF9D00D238DF851
:106B900048300A238DF8493017A812A94A460DF14A
:106BA000060306F031FB0028EAD1BDF80630002BC1
:106BB000E6D00127BFE717A806F009FC2F4B0122FA
:106BC0001A604FB10022284605A9FFF713FF2C4B8E
:106BD0001A7842F004021A70002002F023FB04E04D
:106BE000274B1A7842F004021A702378002323708E
:106BF00031E02378DE070CD5224B1A7801321A7067
:106C0000237803F0FE032370FFF730FE18B3022051
:106C10001FE0237803F0020303F0FF0263B1194B76
:106C20001A78013A1A70237803F0FD032370FFF7F6
:106C30001DFE80B101200CE023785D070BD5114BC0
:106C40001A70237803F0FB032370FFF70FFE10B1D7
:106C50000320FFF7CBFD21B0BDE8F0833C0F00100F
:106C60008C1B0010FC1E0100A4170010C01900109E
:106C7000C4190010111F0100B40B3823340B382342
:106C8000F3170010380F001008B524220448002123
:106C9000FDF718FD034B1A7822F004021A7008BDA4
:106CA0003C0F0010F3170010044B05481A78002120
:106CB0001044C2F1FC02FDF705BD00BFF117001042
:106CC000FA170010F7B5FFF7EFFF53482D21FDF736
:106CD00043FD514D0646002800F0988000232846C9
:106CE0003A210093FDF738FD019030B92846FDF7B1
:106CF0000BFE022823D9AB1C0193019B02AF013389
:106D000047F8043D0024019BE2B21B78ABB1042C90
:106D100012D001990B78202B02D101310191F8E7B3
:106D20001D2BFAD02C2BF8D03BB138460AF076FB5D
:106D30000DF804000134E6E72246D3B200E0FF2359
:106D40005BB2013365D07378522B04D0572B02D03D
:106D5000502B5BD137E09DF80000FDF787FF04461C
:106D600008B9462053E07378522B2C4B17D1017F82
:106D7000702202FB01339B6B9DF802201E6A9DF876
:106D80000330B0472B78422B04D101236371236871
:106D90001B7802E000236371FF23237139E02A7816
:106DA000422A03D14179026801391170217F702292
:106DB00002FB01339B6B20465D6A9DF802209DF823
:106DC0000330A84725E09DF80000FDF74FFF00289D
:106DD000C7D0437F012B15D09DF800109DF80230DD
:106DE000C1F163028271006A013BDBB2FF2B04D068
:106DF000426A02B9026A1046F6E7037B81716FF3BB
:106E0000410303739DF80130437102E01F2002F03B
:106E100009FA03B0F0BD00BFFA170010C419001042
:106E20002DE9F84FDFF85C80134EB8F80090134D51
:106E3000C0EB0900C3B237882A68DFF84CA0C91A32
:106E40009AF800B01068B942B4BF0C463C46E4B2B0
:106E50000B4958442246A344A1443C1B1944A4B204
:106E6000FDF7DEFB8AF800B0A8F80090348004B982
:106E70002C60BDE8F88F00BF680F0010600F001095
:106E800000180010660F0010640F001070B51E4C43
:106E900005462378ABB91D4809F099FD280A09F089
:106EA0006DFD1B4EE8B209F069FD1A4809F08FFD2F
:106EB0003088000A09F062FD307809F05FFD09F0C2
:106EC00088FD23781BB9144B1A780F4B1A70207861
:106ED000124B13F80A2CA3F10C015AB1904207D1BE
:106EE00033F80C2CAA4203D14B68087A984701E08A
:106EF0000C33EEE7064B4FF6FF721A802278064BF2
:106F00001A700023237070BD7519001074210100E0
:106F10000400001082210100650F00101420010000
:106F200010B590B001A96A46012304460AF0C4F9DD
:106F300048BB164A009910700B78C3B15F2B03D180
:106F400004A8FDF783FC05E001A8202204AB0AF0A9
:106F50008BF9C0B99DF804300D4A702101FB032361
:106F60009B6B01A89B6B04A9984760B908E0204679
:106F70002F21FDF7F1FB18B9272002F053F902E0A9
:106F800001A80AF077F810B010BD00BF88190010F2
:106F9000C41900102DE9F04FAA4EA9B0002002F04C
:106FA00041F93278FA2A04D1202002F03BF901F0AD
:106FB000BCB9A54F397811B9A44809F013FD31784F
:106FC000A34B197041B1A14B0B4413F8013C0D2B9D
:106FD00002D19C4B4A1E1A70327822B91F2002F04F
:106FE00021F901F0A2B9994D28782C46582801F0D2
:106FF000D2806B78442B40F0B880FFF755FE2B7899
:107000004D2B05D0522B32D0432B40F0A98020E0ED
:1070100028463A21FDF7A0FB20B9222002F002F910
:1070200001F083B9A81C1CA910AA00230AF044F996
:10703000002841F07A819DF87030864A702101FB6A
:1070400003239B6B0DEB01005B6B1099984701F0DC
:107050006CB9A81CFFF764FF7F4B1B78580741F100
:10706000648100207D49FFF70FFD01F05EB92846DD
:107070002F21FDF771FB20B1222002F0D3F801F09F
:1070800054B9023528A840F8885D0AF019F8069B23
:1070900005461A783A2A04D0222002F0C3F801F0FB
:1070A00044B96C4F702606FB007208AC30328DF884
:1070B0001C0092E80300062284E80300591C07A87C
:1070C00010AB0AF0D1F8002841F02F819DF81C3058
:1070D00007A806FB03739B6B10A99B6B98470028BE
:1070E00041F023819DF81C300AA806FB0376B36BA0
:1070F00007A9DB6A9847002841F017819DF82830DE
:107100007026B84606FB0377BB6B0AA81B6B0DEB1A
:1071100006019847013009D0514B1B78002B41F0F4
:1071200004813F2002F07EF801F0FFB89DF81C308A
:1071300006FB058506FB0386303595E8030084E8E9
:107140000300B36B10A9DB6807A89847FF28014626
:1071500001F0EB800120002201F082FF01F0E5B890
:107160001E2002F05FF801F0E0B84238132801F267
:10717000D280DFE810F0140018007501D008D008A4
:10718000EB01D0087402D008D008D0088402E703CD
:10719000D0081004D0085A04BD042805A707FFF73B
:1071A00091FD01F0C2B8502B05D0D02B28D1A0788A
:1071B0000138C0B207E0FFF777FD2A4B28A840F856
:1071C000303D09F07DFF284B441C1B78834206D8D4
:1071D0004D20E1B2002201F043FF01F0A6B8234B9D
:1071E00018701D4B1B78590703D500201B49FFF76A
:1071F0004BFC0220E1B2002201F032FF01F095B811
:10720000FFF752FD11483D21FDF7A6FA059020B980
:107210001E2002F007F801F088B8431C05930023F4
:10722000037010A9124806AA0AF046F8002841F097
:107230007C8006980378EBB9222001F0F3FF01F07F
:1072400074B800BFF117001075190010FA1700107C
:10725000F2170010C4190010F31700104A2401009F
:1072600072190010FC170010C1190010C01900108D
:10727000FB17001009F010FF04460028C8D110A821
:10728000069920221CAB09F0EFFF002804D13F2013
:1072900001F0C8FF01F049B801F34780204601F032
:1072A000C1FFFDF70FFC0446FDF70CFC0546002C62
:1072B00001F03B80002801F0388005982C2107AAB6
:1072C0000AF02AFDDFF814830590002605980028AF
:1072D00000F0BE800AA905AA002309F0EDFF0028EE
:1072E00040F0B6800AA8059920221CAB09F0BCFF2B
:1072F000002840F0AD809DF8813003F00703042B97
:1073000014D116F0030303D0402001F08BFF9FE05F
:107310009DF82820702101FB02820121926B0091CF
:1073200097680AA81CA92246B8470DE0042EEBD0A6
:107330009DF82830702202FB03839B6B0DEB02014A
:107340001B680AA8224698479D4B1F78002F7FD1C3
:1073500036BB9DF88160394630221CA8FDF7B2F992
:1073600010221CA80699FDF7FFFA06F007069DF803
:1073700040307022042E02FB038309D19A6B012155
:10738000E3790091976810A81CA92A46B84707E03E
:107390009B6B00975F6810A81CA932462B46B84724
:1073A0006B7922796179042E14BF5F42E779C1EBD2
:1073B000020018BFFFB20130874202DD571C7F1A5E
:1073C000FFB2C3F580729742C8BF5F422268286847
:1073D000C8BFFFB2184411443A46FDF721F92846C8
:1073E000FDF75AFC6379013B3B4463716B791F44A1
:1073F000FFB26F71013F2F71237B9A0603D562792B
:1074000023799A4217D0E37923B1636920469847DC
:1074100030B11DE063795A1C627122799A42F4D02E
:10742000EB7913B96B79002BBAD16B692846984771
:107430000028B5D00CE02046FDF7D4FBFDF742FB59
:107440002C21044607AA00200AF066FC05903DE7BF
:10745000A369204698472846FDF7C4FB00F065BFA6
:10746000A078FDF703FC054620B9462001F0DAFEBE
:1074700000F05BBF437F012B05D98379056AC3F117
:1074800063028271AB71FF2300266E712B716378EA
:10749000E778522B626817D0572B33D0492B50D145
:1074A00031464FF480722868FDF70CF9454B384699
:1074B00019792A680AF028FB002800F036874A204C
:1074C00001F0B0FE00F031BF6B7F012B04D84E20DD
:1074D00001F0A8FE00F029BF2968384601230AF010
:1074E00033FA0146002800F02087012804D1142037
:1074F00001F098FE00F019BF4A20324601F0B0FDBD
:1075000000F013BF6B7F012BE1D9296838460123B6
:107510000AF086FA0128014608D0C0F00687022842
:1075200009D11A2001F07EFE00F0FFBE192001F003
:1075300079FE00F0FABE4A20324601F091FD00F0DB
:10754000F4BE1F2001F06EFE00F0EFBE022A40F2F2
:10755000EC862D2B02D1A378502B04D01E2001F0F5
:1075600061FE00F0E2BE032A03D0164BDD78FF2D4A
:1075700003D1154B1D780135EDB2144B144E00218B
:107580001E2283F83D1483F83C243046FDF79AF818
:107590000D23B3770F4B34461B78AB42C0F0C58642
:1075A000F5B90D4B03F11C0253F8041B934246F846
:1075B000041BF9D11A889B783280B37000F0B5BEF5
:1075C00072190010FA170010C019001024130010CF
:1075D0000E190010C11900101E1F0100C41900105F
:1075E000A84A6E1EF6B2702303FB0623A6499F6BC2
:1075F00090468F420ABF93F86030012303F07F0367
:107600002370E2236370A021A570A0481022FDF72B
:1076100059F83B6930469E499847002840F08586D6
:107620009B49034601335A1812F8012C12B1E01895
:107630008270F7E7702303FB0686F3681A0CE27486
:1076400063751A0AB368227596F82A20013B5343E2
:107650001A0CE2761A0A2277637700F066BE8D4B29
:107660001B78022B06D015201221002201F0F8FC15
:1076700000F05BBE0520FDF7BFFA00F056BEA17812
:10768000854B572940F0A580052A40F24E861D798A
:10769000DA785E7902EB0525ADB2772D06D19A79BD
:1076A0007E4B02F01F021A7000F03FBEA5F5E052BB
:1076B000063A92B2012A40F2388641F60202954219
:1076C00000F03386764A4FF00009DFF808B29A4698
:1076D00082F8009043F6A2036279DFF8F8814A4508
:1076E00018D909F106081AF80810BBF8000003932E
:1076F000FCF758FD039BABF80000984205D11AF83F
:107700000820602A04BF08223A7009F101095FFAD3
:1077100089F9E1E7B8F80010624B13F8024C1A1F20
:107720008CB1043333F8080C8842F6D1D3783C701E
:107730004BB15D4A5D4852F8331002EBC3035A68FF
:107740005B4B01601A605B4B1A689A461AB1284677
:107750003146FFF765FB44B3DAF800302BBB564BDC
:1077600013F8062CA3F10609A2421BD133F8042C0E
:10777000524B1A8099F80420514B01321A80514B18
:1077800000221A70FDF786F9CAF80000002800F000
:10779000C685037B43F04003037399F8053083717A
:1077A00000F0BDBD0633002ADAD13B78002B40F053
:1077B000BC85454809F00BF9B8F80000000A09F04B
:1077C000DDF898F8000009F0D9F809F002F900F0A6
:1077D000ACBD45290BD1042A40F2A7851879DB7886
:1077E00003EB002080B2FFF751FB00F09EBD522951
:1077F0007FF4B4AE052A40F298851D79DB7803EB5F
:107800000525ADB22B0440F18280304E3378002B39
:107810007DD0DFF8C4A01B4F9AF800004FF070092C
:1078200009FB0070036B2A4983613246012305F08E
:1078300085FBDFF89C8058B9D8F80C30A5F50045D9
:10784000B3F5004FADB249D2C5F30D05ADB245E079
:107850009AF80000414609FB00704FF00009C0F89B
:1078600018903246012305F069FB0028E4D0C7F8E0
:107870001890384641463246012305F05FFB002848
:1078800045D1D9E7C4190010BC1E01001119001020
:10789000A4170010F0170010FA170010BD190010FF
:1078A000650F0010421F0100C42101008019001063
:1078B00078190010600F0010B8210100660F001049
:1078C000680F0010640F001089210100FD180010DE
:1078D0006C0F001004000010C0190010C3F30D035A
:1078E0000BB11D44ADB2AB48294605F077FD70B928
:1078F0006679A848642E28BF6426A74932461CAB87
:1079000005F0EAFB18B9BDF87030B3420DD0A34BB7
:1079100033F8042C191F42B1AA4203F10403F7D132
:107920008A789D4B1A70CA785A709D4B9A4AC3F850
:107930003824002283F83D246279013A83F83C24FC
:1079400000F0F3BC974DFFF7AFF928A840F8305D81
:1079500009F0B6FB3A210446681EFCF7FDFE431C05
:107960001C9320B9222001F05DFC00F0DEBC18461B
:107970002C21FCF7F1FE024610B1002302F8013B76
:10798000894B702101FB04339B6B20469B6A1C9939
:10799000984700F0CABC3170FFF786F93378012BA5
:1079A0007FF663AD6078814D00F00F00FDF75EF962
:1079B000064600283FF459AD0469002C3FF40EAB95
:1079C000C3790BB37A4A1278012A09D9022AA97815
:1079D00007D0E878032A41EA002102D02A7901E0A1
:1079E000012101229A4204D9332001F01BFC00F04E
:1079F0009CBC09B1013989B20AB1013AD2B2304610
:107A00005943A04700F091BCAA78002162F3070116
:107A1000EA7862F30F212A7962F317416A7962F3F7
:107A20001F611A46A04700F080BCFFF73DF95F4890
:107A30003D21FCF791FE069020B91E2001F0F2FBDB
:107A400000F073BC431C06930023037010A9554833
:107A500007AA09F031FC0346002840F06684069826
:107A60000AA906AA09F028FC002840F05E840BA8A9
:107A700011A90822FCF7A0FD20B13E2001F0D2FBA5
:107A800000F053BC079809F007FB04460028D4D146
:107A900007990B7823B9222001F0C4FB00F045BC04
:107AA00010A820221CAB09F0DFFB002804D13F20E6
:107AB00001F0B8FB00F039BC00F33784204601F038
:107AC000B1FB0AA8069920221CAB09F0CDFB0028C7
:107AD00040F02B849DF82830334A702101FB0323AA
:107AE0009B6B0AA8DB6B6944079A984700F01DBCA2
:107AF000032A02D12D2B3FF471AAFFF7D5F82C21D0
:107B000007AA28480AF008F92A4B01210246196001
:107B100000241CAD002A51D0104610A90AAA002347
:107B200009F0CAFB204E9DF84030702202FB03632F
:107B30009B6B2148DB6A10A99847002840F0F58329
:107B400020270022009701951B480A99134609F047
:107B500041FB002817DB40F0E8839DF8813003F0FB
:107B60000703062BEDD09DF84030702202FB036323
:107B70009B6B10A8DB6829469847FF2800F0D58347
:107B80000444E4B2DCE707AA00202C210AF0C4F880
:107B90000246BFE76C0F00100E19001068210100AB
:107BA00024130010FB170010C4190010FA1700105E
:107BB000F1170010EC0338230C13001001202146AC
:107BC00001F04EFAB1E3BA4B197800293FF4C6AC84
:107BD000A378522B40F01681022903D01F2001F018
:107BE00021FBA2E31CA809F0D1FC9DF872200C2314
:107BF000B2FBF3F503FB152515F0FF0508BF1D4685
:107C0000E378413B082B00F2F980DFE813F009002C
:107C10005500F7008C00F700F700F700F700AE0002
:107C2000A44B192283F83C24A34BA44A03F114016A
:107C300053F8040B8B4242F8040BF9D119889B7856
:107C4000118093709DF876209D4B9E4C9DF874108A
:107C500053F822302046013140F8053BC9B20AF002
:107C600031F89DF8731004F108000AF02BF89DF824
:107C700075206423B2FBF3F103FB112104F10B0027
:107C8000C9B20AF01FF8294604F10E000AF01AF8EA
:107C90009DF8711004F111000AF014F804F11400B9
:107CA0009DF870100AF00EF89DF872300B2B94BFFF
:107CB00041235023E37538E37E4B082283F83C24AC
:107CC000804C9DF876309DF8752023706423B2FBBC
:107CD000F3F103FB1120C0B20AF015F860709DF8B3
:107CE00074000130C0B20AF00EF8A0709DF8730065
:107CF0000AF009F8E07028460AF005F820719DF8AE
:107D000071000AF000F860719DF8700009F0FBFF47
:107D10009DF87230A0710B2B94BF00230123E371F7
:107D20000D23237201E3634B082183F83C149DF873
:107D30007610644B0B2A19709DF8751098BF0022BD
:107D400059709DF8741088BF0122013199709DF817
:107D50007310DA71D9709DF871100D2259719DF868
:107D600070101D7199711A72DFE2524B172283F85D
:107D70003C249DF875106425524CB1FBF5F113318C
:107D8000C9B2204609F09EFF9DF87530B3FBF5F2AD
:107D900005FB1231C9B209F095FF2D2505709DF83C
:107DA000741001300131C9B209F08CFF05709DF8E3
:107DB0007310013009F086FF542303709DF8721090
:107DC000013009F07FFF3A2505709DF871100130F0
:107DD00009F078FF05709DF87010013009F072FF0E
:107DE000202303709DF87620354B03EB82031A881D
:107DF0009B78A282A3750D23E37596E21E2001F005
:107E000011FA92E2572B7FF4A9AB2F4BDB78413B61
:107E1000082B00F2E480DFE813F009002100E20003
:107E20005B00E200E200E200E2007F001A2A03D8D1
:107E30001F2001F0F7F978E2214F0025234807EBD6
:107E400085010222FCF7B8FB5FFA85F80646002898
:107E500000F0C9800135072DF0D1E9E70B2AE7D9F9
:107E6000237960798DF8763009F045FF8DF875003B
:107E7000A07909F040FF8DF87400E07909F03BFF2C
:107E80008DF87300207A09F036FF0C2814BF8DF8A6
:107E900072000023607A08BF8DF8723009F02BFF62
:107EA0008DF87100A07A09F026FF8DF8700029E0A6
:107EB000851B0010241300109A21010012190010D4
:107EC000142201000E190010FA170010FE170010FE
:107ED0000B2AADD923798DF8763063798DF875301A
:107EE000A3798DF87430E3798DF87330237A0C2BF5
:107EF00008BF00238DF87230637A8DF87130A37A51
:107F00008DF87030E37A002B00F0AD809DF8723070
:107F10000C338DF87230A6E0162A89D9BB4B28ACF9
:107F200044F8603D204609F079FA109B6C38013323
:107F30008DF875002046109309F070FA109B8DF8AB
:107F4000740001332046109309F068FA109B8DF8F5
:107F5000730001332046109309F060FA109B8DF8EE
:107F6000720001332046109309F058FA109B8DF8E7
:107F7000710001332046109309F050FA9DF87410F7
:107F80008DF870009DF87500022900F26C739CBF9B
:107F9000DAB200F26B734FF0170000FB01F188BFFB
:107FA0009A1E9DF8734088BFD2B20920224491FBEB
:107FB000F0F1D2B20A4404326421B3FBF1F102EBD6
:107FC0009302521A4FF4C871B3FBF1F31344072222
:107FD00093FBF2F102FB11338DF8763043E01E2063
:107FE00001F020F9A1E18A4B28AD45F8603D284613
:107FF0008DF8768009F012FA109B8DF87400013329
:108000002846109309F00AFA109B8DF8730001338B
:108010002846109309F002FA109B8DF87500013381
:108020002846109309F0FAF9109B8DF8720001337D
:108030002846109309F0F2F9109B8DF87100013376
:108040002846109309F0EAF9237F8DF870004D2B34
:1080500009D19DF872300C2BE37E08BF8DF8726059
:10806000502B3FF453AF9DF875209DF874304F2A84
:108070009CBF64328DF875209DF87320013B013A56
:10808000D2B2DBB21E2A8DF874303FF6D1AE0B2B84
:108090003FF6CEAE9DF87630062B3FF6C9AE9DF882
:1080A0007230172B3FF6C4AE9DF871303B2B3FF674
:1080B000BFAE9DF870303B2B3FF6BAAE1CA809F05E
:1080C00093FA32E13A2B4DD00AD8322B1FD004D884
:1080D000302B4ED0312B13D059E0382B27D81DE050
:1080E000482B06D8432B19D2412B09D0422B0ED056
:1080F0004DE04A2B36D01AD3CA2B48D108F046FBA4
:108100002D23237052236370FEF7DCFD0DE12D2338
:10811000237057236370FEF7D5FD06E1333B032040
:10812000584300F5A06080B2FEF7B0FEFDE0022AE1
:1081300003D1492001F076F8F7E0A3782B2B07D084
:108140002D2B0BD1334B1A7842F001021A70ECE060
:10815000304B1A7822F001021A70E6E0492001F053
:1081600061F8E2E00420FCF747FD492001F05AF8ED
:10817000DBE0A37803F01F031E2B08D1264BDB782E
:108180001A1FD2B21A2A02D8244A1370CDE01E2038
:1081900001F048F8C9E0FEF787FD6B78492B53D012
:1081A0000CD83F2B00F0A68003D82A2B00F0888043
:1081B000A7E0442B44D0452B11D0A2E0532B72D022
:1081C00005D8512B00F09A80522B56D099E0572BAE
:1081D0004AD05A2B40F0958002F006FDA5E0AB1C7A
:1081E0001093AB782B2B1FD02D2B04D1094B1A7871
:1081F00022F008021CE010A809F010F9C0B204280F
:108200000ED91E2001F00EF813E000BFFE1700107B
:1082100003180010F3170010FA170010BD19001012
:10822000434B0228187004D9424B1A7842F00802D6
:108230001A70414B03201978002200F011FF74E0FE
:108240001E2000F0EFFF70E028A8023540F8605DC6
:1082500009F0E4F8C0B2022802D8384B187064E084
:108260001E2000F0DFFF60E000F078FB324B0320BF
:108270001978002200F0F4FE57E0AB783A2B0ED1CB
:108280002F4B1B78132B03D9202000F0CBFF4CE0A1
:108290002C482D4929B0BDE8F04FFCF7D7BA294B3F
:1082A00000221A7041E0A81C1CA910AA002309F0A2
:1082B00003F8002839D11CA81099FEF7E5FB34E03B
:1082C000AB782B2B05D02D2B08D01E2000F0AAFF59
:1082D0002BE0184B1A7842F0100203E0154B1A7885
:1082E00022F010021A70144B03201978002200F0BB
:1082F000B7FE1AE0092000F095FF16E002F016FC28
:1083000013E03378012BABD10B4B032019780022FB
:1083100000F0A6FE09E01E2000F084FF05E02846DC
:108320003146FEF77DFDFFF740BA29B0BDE8F08F7A
:1083300085190010F3170010BD190010B8190010AE
:10834000F1170010FD180010FD170010234B13B596
:108350001A68044602609A889B7982808371204B58
:108360001B78022B37D1D020002107226B4608F062
:1083700003F880BB9DF8000000F07F0009F0BBFC13
:1083800020709DF8010009F0B6FC60709DF80200B5
:1083900009F0B1FCA0709DF8040009F0ACFCE0709D
:1083A0009DF8050000F07F0009F0A5FC0138207160
:1083B0009DF8030009F09FFC0138A0719DF80600AC
:1083C00009F099FC9DF905306430002BB4BF64239B
:1083D00000230344637102B010BD00BF53280100A5
:1083E000851B001037B5234D04462B78002B3ED05B
:1083F000007809F088FC8DF80000607809F083FCB3
:108400008DF80100A07809F07EFC8DF80200A079BB
:108410000130C0B209F077FC8DF80300E07809F074
:1084200072FC8DF8040020790130C0B209F06BFCB9
:1084300062796423B2FBF3F18DF8050003FB112090
:10844000C0B209F060FC6B468DF8060000210722DF
:10845000D02007F043FF0E210022D02007F050FF6C
:10846000D0200F21002207F04BFF02232B7003B016
:1084700030BD00BF851B001010B50E4C00230E4808
:10848000237008F0A4FAD0200F2107F087FF0028FE
:1084900001DA0A4808E0030603D5012323700848DF
:1084A00002E002230748237008F091FABDE810406B
:1084B00008F08FBA851B001031220100392201001B
:1084C00043220100B4270100064B03F1100253F8C8
:1084D000040B934241F8040BF9D11B7800200B7078
:1084E000704700BF5C2201000020704710B50446B1
:1084F000FCF70AFAC2B2A018A021C2F11002BDE82E
:108500001040FCF7DFB81F2000F08CBE114614208D
:108510001A4600F0A5BD114614201A4600F0A0BD71
:1085200030B587B0054614220C4601A80021FCF79F
:10853000C9F8281D01A900F05FFB054620BB3022C9
:1085400020462946FCF7BEF80523E3760223637430
:10855000BDF804302846FF331B1263822A4601AB64
:10856000034499780130A02908BF9A701028F6D1E9
:108570000DF106030DF1160253F8041B934244F863
:10858000041BF9D1002000E0FF2040B207B030BD4D
:10859000034B00201A681B790A600B71704700BFFB
:1085A000B0220100054B03F1100253F8040B934273
:1085B00041F8040BF9D10020704700BF4B220100A5
:1085C00008B50B7800F8043B00F012FB002008BD52
:1085D00000F0ECBA08B500F005FBC0F3870008BD59
:1085E0000146062813D8DFE800F00406090B0B0E3D
:1085F0001000002000E03E2000F014BE3F20FBE70A
:108600004820002205E01F20F6E71E20F4E71F2087
:10861000632200F025BD38B5084614460D46FFF725
:1086200065FF2046FFF762FF2846214600F084FCE4
:10863000BDE83840FFF7D4BF0A4B012210B5084609
:108640000C461A60FFF752FF204600F097FC0446E4
:10865000FFF7C6FF06F0F8FDD4F1010038BF002097
:1086600010BD00BFEC03382313B501680DF10603FC
:10867000044602311C30FE2200F0ECFB034630B110
:10868000FFF7AEFF2046FCF791FA012015E0022229
:108690006271BDF80620511CFD2A2171227B03D98D
:1086A000E08BA18B884204D142F02002227300208B
:1086B00003E063F345122273184602B010BD0000B8
:1086C00038B508460D461C46FFF710FF9DF81030E0
:1086D00004F11C0128460BB1022200E0012200F047
:1086E000B1FA0546FFF77CFF6DB9237B0D2243F0FD
:1086F0004803237302236371237123689A70024B2A
:108700006361024BA36138BD7D8700004D87000087
:1087100038B508460D461446FFF7E8FE284604F132
:108720001C01002200F08EFA0546FFF759FF55B9EB
:10873000237B054A43F04403626123732046BDE86E
:108740003840FFF791BF38BD6986000038B5037B1C
:10875000044643F300036BB143699847054638B9B3
:1087600004F11C0000F0D6FB034B2846A36138BD82
:10877000012038BD184638BDF949000073B5037BA8
:1087800004469B0702D44379013B03712279216897
:1087900004F11C05013A2846023192B20DF106039C
:1087A00000F0BEFA064648B1FFF71AFF284600F06F
:1087B000B1FB2046FCF7FAF901200AE02046FCF75D
:1087C0007DFA237B304666F34103237302236371F2
:1087D000237102B070BD000009490A4AFF230B70E3
:1087E0001378032B0AD80B700749702000FB031184
:1087F000064801338863137000F09EB9704700BFCC
:10880000FC180010C1190010C419001070220100DA
:108810000D4A0E4B1B681068002B14BF0823092358
:1088200000280CBF022000201844094B1B68002BB5
:108830000CBF042300231844064B1B68002B0CBFFD
:108840000823002318447047F0123823F412382309
:10885000E80E3823E40E38232DE9F0412F4C304D3B
:108860002378112243F0100323702E4801230021A6
:108870002B70FBF727FF2C4B2C4A5B69274613F024
:10888000807F5269A84604D1294B80221A70BDE826
:10889000F081284806F026FD4FF6FF739842044603
:1088A00039D000260225A54206D2284606F0FEFC55
:1088B0003044C6B20135F6E71F4806F0F7FC8642A1
:1088C00029D11E4806F0F2FC3B7823F01803184328
:1088D00038701B4806F0EAFC0546FFF799FF854211
:1088E00004D1184806F0E2FC174B1870174806F040
:1088F000DDFC0D2C88F800000DD9154806F0D6FCDB
:10890000144B1D2C187006D9BDE8F04105481249DA
:10891000102206F003BDBDE8F08100BFF317001080
:1089200085190010FD18001020C0092000C0092082
:108930008C1B0010020000800100008005000080F8
:108940000700008006000080BD19001008000080AC
:108950000D000080B81900100E00008038B52048C6
:108960001E2106F039FD1F4B1F4819781F4C01F0DE
:10897000180106F0E9FC1E4B1E48197806F0E4FCCD
:10898000FFF746FF01461C4806F0DEFC1B4B1C4867
:10899000197806F0D9FC1B4B1B48197806F0D4FC5B
:1089A0002046FBF7B1FF024600212018C2F1110258
:1089B000FBF788FE20461549102206F0E1FC002551
:1089C0000224204606F072FC013428441E2CC5B255
:1089D000F7D129460E48BDE8384006F0B5BC00BFC7
:1089E00002000080F317001005000080FD18001041
:1089F000BD190010060000800700008085190010D6
:108A000008000080B81900100D0000800E000080E2
:108A10000100008000F1100149010248202206F007
:108A20007DBC00BFA4170010F8B50C4F064600240B
:108A30002046FFF7EFFFBB7F651C9B07EDB205D11A
:108A4000074831461022FBF7B7FD18B1102D03D0AF
:108A50002C46EDE72046F8BDFF20F8BDA417001016
:108A6000B01700102DE9F843103000AF46018AB06E
:108A70006846314620220024DFF8548006F04EFC80
:108A8000E9462346E1B219F804205BB118F8041056
:108A900091420FD108EB0500A919621B06F070FC8A
:108AA000002307E018F80430934218BF0D460CBFAE
:108AB000002301230134202CE4D133B10448A91947
:108AC0002844C5F1200206F05BFCBD46BDE8F883F2
:108AD000A4170010CB08012201F0070102FA01F1EE
:108AE000C25C1143C154704738B50D4D0446012195
:108AF000E308EA5C04F0070301FA03F31A4208D022
:108B00000134E4B2102C08BF00248442F0D1FF20CD
:108B100038BD03482146FFF7DDFF204638BD00BFC2
:108B2000900F0010034B9B7F13F0020F14BF1E2009
:108B30000C207047A41700102DE9F041174E702348
:108B4000174800210E223370164FFBF7BBFD164B62
:108B500000241C705C70B8462046FFF75BFFBD7FA9
:108B600015F0010505D00134E4B2102CF4D1BDE8B4
:108B7000F0810D482146FFF7ADFFFFF7D3FF854297
:108B8000F1D218F80510FF2905D00548FFF7A2FF1C
:108B90003378013B33700135EDB2EEE7920F0010F0
:108BA000930F0010A4170010900F001037B54FF46A
:108BB00000744FF0FF3501A82146042206F0AEFBF9
:108BC000019B013305D001A821460422019506F03E
:108BD000D7FB0434B4F5005FEDD1FFF7ADFF03B070
:108BE00030BD0000014B1878704700BF920F001095
:108BF000002303707047000070B5114E05460C4607
:108C000028780F280ED8421C2A70FFF703FFB37F85
:108C100013F0030F0A4BF3D103F10C02A11C03F173
:108C20001C0001E0012070BD52F8045B824241F853
:108C3000045BF9D19A7F0020E2749B8B238070BD86
:108C4000A4170010F8B50746164608460A220C4637
:108C50000021FBF737FD3846FFF7E6FE012E0546FB
:108C600022D1FF2852D10020FFF73EFFFF282071BC
:108C70004ED0E07120222572667227482946FBF704
:108C800021FD264B384607F1100250F8041B904294
:108C900043F8041BF9D1204B00251D775D779D77A4
:108CA0002079FFF7DFFE29E0FF2833D01A4B20712F
:108CB0009A8B022E22801E4622D1F77FFF2F04D0EE
:108CC0003846FFF7A7FE3D46F7E7FFF72BFF0023E7
:108CD0001A4600E00A46D9B2814205D20133F7189C
:108CE00017F8017CFF2FF5D1B35CE5716371238820
:108CF000638003F03F03A371012363720020F8BD7A
:108D00001B78E071002063716072F8BD0220F8BD2D
:108D10000320F8BD0120F8BDA4170010B017001003
:108D20002DE9F74F9846437A0446012B0F46164625
:108D300040F081800023DFF81891A8F80030002E61
:108D400077D0A379002B4ED162790121154605F029
:108D5000070B01FA0BFB3C48EB08C35C13EA0B0B57
:108D6000CDF804B007D00135EDB2702D08BF002555
:108D70009542ECD161E0FF2D5FD0E0796571FFF79E
:108D800049FE237A01335FFA83FA84F808A0FFF7DB
:108D9000C9FE824518D3E079FFF7A6FEFF28824678
:108DA0004DD0DFF8A8B08BF81F00E079FFF75AFE2E
:108DB00020225846FF21FBF785FC019B02228BF8FD
:108DC0001E2084F807A023721F482946FFF782FE61
:108DD00099F800301D4A013B89F80030237AD554B8
:108DE000E079FFF73FFEA1796379C1F14005ADB2AB
:108DF000AE4238BF3546EDB201F580612A463846AD
:108E000001EB831106F0BCFA2288ABB21A4422802F
:108E100062882F441A446280A279F61A154405F03C
:108E20003F05A571B8F80020B6B21344A8F8003089
:108E300085E7304604E0052002E0042000E003203E
:108E400003B0BDE8F08F00BF930F0010A41700100F
:108E5000920F00102DE9F0479846437A04460F46DA
:108E60001546002B50D1A8F8003002884388DFF85F
:108E7000A090D31A9D42C8BF9DB2002D41D0A179C8
:108E80006379C1F14006B6B2B54238BF2E46F6B29C
:108E900001F580613246384601EB831106F03EFA57
:108EA000B8F80020B3B21A44A8F800206288ED1A7E
:108EB0001344A2793744164422889BB206F03F0639
:108EC0009A42ADB26380A671D7D0002ED5D1E07999
:108ED000FFF7A0FD94F808A00AF1010A5FFA8AFAE8
:108EE00084F808A0FFF71EFE824505D399F81F00FD
:108EF0002672E071FFF78EFD237A19F80330637153
:108F0000BBE72846BDE8F0870520BDE8F08700BF35
:108F1000A417001010B5437A044643B10079FFF757
:108F200079FD2288034B9A832079FFF79BFD00236C
:108F3000637210BDA417001038B5054608460C46EC
:108F4000FFF772FDFF2812D12846FFF76DFDFF28BD
:108F50000FD0094B214604F1100251F8044B914205
:108F600043F8044BF9D1FFF77DFD002038BD022006
:108F700038BD012038BD00BFB01700102DE9F04703
:108F8000FFF752FDFF28054630D01B4E1B4FB14660
:108F9000DFF86C8000244FF0010AFFF7C3FD844224
:108FA00013D2335DFF2B10D0DA0803F007030AFA5F
:108FB00003F3B95C013421EA0303BB5498F8003091
:108FC000E4B2013388F80030E7E799F81F40FF2149
:108FD00020220948FBF776FB2846FFF743FDFF2CCC
:108FE00007D02046FFF716FD2546D1E70120BDE852
:108FF000F0870020BDE8F087A4170010930F001041
:10900000920F001070B580320C4600214B1C615C41
:10901000DBB2914203D0FF2903D01946F6E7FF2ABD
:1090200003D13F230370013070BDE256002A09DAF4
:109030000133DBB2F9E7002DA4BF02700130002D2F
:109040000ADB3346E25C5E1C1F2AF6B255B2F2D848
:109050000249FFF7D7FFF2E770BD00BFB12301005F
:109060002DE9F84F634B644FDFF8AC810025187091
:1090700004468946164629466422C7F8388487F88C
:109080003C5487F83D544046FBF71CFB40462146C4
:1090900008F018FE2C22032C0346027051D1012E39
:1090A00000F1020036D045225A70544B4FF03A0A74
:1090B000197808F007FE524B1A7812F0080F18BF03
:1090C0002B211A4608BF2D21431C017083F800A0F4
:1090D00012782A2112F0100F597003F1030214BF05
:1090E0002B212D2199701046492300F802AB5370B3
:1090F000444B197808F0E6FD054605F802AB52230B
:10910000437041492846FBF7A1FB3F48FBF7FCFBB6
:10911000284448E044225A704FF03A0B4FF03D0A81
:10912000294680F800B0013008F0CCFD2946013511
:1091300080F800A0EDB2013008F0C4FD082DEFD199
:1091400031E004F0BF03092B00F1010027D12F49C2
:1091500005462A1AD2B28A5C2B4603F8012B0AB1C3
:109160001D46F6E7092C284617D1DFF8B0E0DFF8F6
:10917000B0C06B1C2D1AEDB21EF80520DCF80010F3
:109180001144497801F00301022908BF203AD2B204
:1091900003F8012C0AB11D46EBE7581E03E01C49F9
:1091A0002246FFF72FFF2C2505704946013008F0B5
:1091B00089FD31460570013008F084FD0D230370F0
:1091C000144B132C05461A7805D9492C03D042F0CC
:1091D00001021A7008E002F0FE021A701A7802F01A
:1091E000FE021A7006F030F8C8EB050887F83C84D8
:1091F000BDE8F88F721900102413001085190010B3
:10920000F3170010B8190010FD1800100724010012
:10921000B6220100BE1900100E190010272401000B
:109220000000001000210A46FFF71ABF08B5002011
:10923000FFF7F8FF002008BD30B572B60E490F4B9E
:10924000042201240D68002DFCD110F0010514BF8B
:109250001C601D6040080D68002DFCD010F0010559
:1092600002F1FF3214BF1C601D6012F0FF024FEAD2
:109270005000E7D162B630BDE806382384070842C3
:1092800070B54C1E204472B60B4A1368002BFCD1FB
:109290000A4B0122091A0A4E1A6004468DB263195C
:1092A0009BB223B13368984704F80109F7E7034AF2
:1092B000136062B670BD00BFE80638238407084219
:1092C0008019001070B54C1E204472B6104A136805
:1092D000002BFCD10F4B0122091A0F4E1A600446D5
:1092E0008DB263199BB223B13368984704F8010922
:1092F000F7E70A4B1B78123BDBB2012B03D8044A79
:109300001368002BFCD0034B00221A6062B670BDBC
:10931000E8063823840708428019001075190010E8
:10932000F8B5EFF3108772B6094B1D68002DFCD11C
:10933000084C0126084B26601B689847074B1E60A7
:10934000256087F310881920BDE8F84006F0B4B80E
:10935000E80638238407084278190010800708427D
:1093600008B572B60120FFF7DBFF064B1B780BB97F
:10937000012003E01A2B0CBF08200220FFF7D0FFCA
:1093800062B608BD7219001070B572B60E4A136845
:10939000002BFCD14C1E0D4B04440122091B0C4E2A
:1093A0001A608DB263199BB223B114F801093368B6
:1093B0009847F7E7074A012111600F20536006F034
:1093C0007BF862B670BD00BFE80638238407084208
:1093D000781900108007084270B51A4C02462478AC
:1093E0000B46132C184D26D172B629680029FCD1E2
:1093F0005C1E1649144401201B1B154E08609DB2CB
:1094000063199BB223B114F8010932689047F7E75A
:10941000104A0E4C012313600520236006F04CF81F
:10942000094A1368002BFCD0002323600F2006F0AC
:1094300043F862B670BDFFF7A7FF2B68002BFCD086
:1094400070BD00BF75190010E80638238407084274
:109450007819001080070842F8B5054652200C46DE
:10946000174607F03BFA284607F088FA2F2007F046
:1094700035FA204607F082FA07F0ABFA064B702265
:109480001978064B384602FB01339B6B2A461E6A4D
:109490002346B047F8BD00BFC0190010C419001022
:1094A00070B5064672B600231D46F25C0133B3F573
:1094B000807F85EA0205F8D1002006F043FC0024F5
:1094C000305D013406F03EFCB4F5807FF8D12846CB
:1094D00006F038FC024A01231360536062B670BD87
:1094E000800708422DE9F84F05460F469146FBF7E5
:1094F000E9FA044628B9FF2006F0EEFC0020BDE89A
:10950000F88FDFF8DCA04FF001089AF80010334A1A
:10951000702303FB01239B6BDFF8C8B01E6A204653
:109520003B462A46B0479BF80030002BE3D1236826
:109530001A781AB95E78013EF6B200E0FE2630468F
:1095400006F0CAFCB9F1000F01D14D462CE0B8F18C
:10955000000F15D023684FF00208987806F0BCFC85
:109560002368D87806F0B8FC0AE006F083FC0028EF
:1095700030DB2368434408F1010898705FFA88F8EB
:10958000B045F2D3164B70221978144B204602FBDB
:1095900001339B6B2A465E6A3B46B0479BF800301E
:1095A000002BA8D1984609E0EBB2B34206D223685B
:1095B0002B44987806F090FC0135F5E723681D7878
:1095C0005F78002DA1D1284606F086FC2046FBF7E7
:1095D000EDFA93E70120BDE8F88F00BFC419001031
:1095E000C01900107219001010B5054C06F02EFDC0
:1095F0000023237006F040FD2378002BFCD010BD23
:1096000074190010094B1A6822B9094A1368002B13
:10961000FCD006E0074A002111601A68002AFCD03D
:1096200001E0012070470020704700BFC8063823C2
:10963000E8063823800708422DE9F041064672B655
:10964000134A012313600320536005F035FF114FC7
:10965000DFF8488008250024FFF7D4FFA8B13B6855
:10966000002B14BF8023002343EA5404D8F80030B1
:10967000002BFBD1013D15F0FF05EDD1044B064A4F
:109680001D60012313601846347062B6BDE8F08196
:1096900080070842EC06382384070842E80638238E
:1096A00070B5174B02461B78164C132B1FD1EFF3E6
:1096B000108672B62368002BFCD1134C0125134B86
:1096C000256010461B689847114B05201D602560DA
:1096D00005F0F2FE0B4A1368002BFCD00023236038
:1096E00086F310880F20BDE8704005F0E5BEFFF757
:1096F00017FE0F2005F0E0FE2368002BFCD070BDA4
:1097000075190010E80638238407084278190010FC
:109710008007084208B572B6064B1B780BB90120CA
:1097200003E01A2B0CBF08200220FFF7B9FF62B636
:1097300008BD00BF72190010F8B5064652200D464C
:1097400014461F4607F0CAF8304607F017F92F20D5
:1097500007F0C4F8284607F011F907F03AF90B4B67
:1097600070211A780A4B204601FB02339B6B11468D
:10977000D3F820C032462B46E04720683946FFF731
:109780002BFEBDE8F840FFF7C5BF00BFC0190010B1
:10979000C419001010B50E4C23785A0701D0FDF7FC
:1097A00077F922780A4B02F0080202F0FF006AB152
:1097B0001A7802F0F7021A70064A01231360A2F524
:1097C000E962136023781B06FCD4012010BD00BFA2
:1097D0008C1B0010340B3823F8B5164E164F042599
:1097E0000024336833B9FFF7D5FF0028F9D04FF6CE
:1097F000FF701DE0032005F05FFE3B68640833B195
:1098000044F0800403E0FFF7C5FF0028EFD1336880
:10981000002BF8D1032005F04FFE3B68640813B11C
:1098200064F07F04E4B2013D15F0FF05D9D1204674
:1098300000B2F8BDE8063823EC063823F8B5174E19
:10984000174F04250024336833B9FFF7A3FF00281E
:10985000F9D04FF6FF701EE0032005F02DFE3B68A7
:109860006400E4B233B144F0010403E0FFF792FF77
:109870000028EED13368002BF8D1032005F01CFE40
:109880003B686400E4B20BB144F00104013D15F003
:10989000FF05D8D1204600B2F8BD00BFE806382346
:1098A000EC063823F8B5134F134C064604253B68E5
:1098B0002BB1FFF76FFF0028F9D00120F8BD30066B
:1098C00048BF012323603B6823B9FFF763FF0028EB
:1098D000F9D0F2E77600F6B2310605F1FF354CBF5C
:1098E00001230023760015F0FF052360F6B2DED1D8
:1098F0002846F8BDE80638238407084270B5154E9F
:10990000154D0446336843B12B682BB9FFF742FF6E
:109910000028F7D0012300E000230F4A126802B9A3
:109920001BB100232370637070BD72B60B4D012311
:109930002B600B4B1B689847002301462B6062B6D7
:109940002046002908BF4FF48071BDE87040FFF742
:1099500097BC00BFE8063823C806382384070842AE
:109960008019001008B5064B012018605860FFF7F9
:1099700099FF20B91120BDE80840FFF793BF08BD4B
:109980008007084238B5354B00241C6007F00AF800
:10999000334923464A7AD8B2904204D2C818807A12
:1099A000C8540133F7E700242E4B20468C541A701C
:1099B00004F08EFB2046FBF759F9044648B972B60D
:1099C000FF2006F06BF8254A01231360536062B64E
:1099D00038BD72B60125237B9B064CBF00200120B9
:1099E00006F05CF865B165792368585D06F056F8B5
:1099F0006A1C2368D2B2985C023506F04FF8657194
:109A0000237B13F0200F637911D022790232D01A10
:109A1000C0B206F043F865792368585D06F03EF859
:109A200022796B1CAA42DBB20FD91D46F4E72068ED
:109A3000FE21184406F05EF863692046984708B98D
:109A40000546C8E7FF2006F029F862B62046FBF776
:109A5000C9F8024B01221A6038BD00BF80070842D6
:109A6000FA170010F11700102DE9F7430646002001
:109A7000FBF7FCF8044620B92A4B186043F8040CA5
:109A80004DE0142005F02CFDDFF89C80002506F049
:109A90007DF8237B8DF8055043F3401313F0FF0F3F
:109AA00018BF23796F1C8DF806302368FFB29B78AE
:109AB0008DF8073016B9BE2005F0FEFC01A806F0AF
:109AC00083F800254FEA8509D8F8003009F1030929
:109AD0005FFA89F903BB16B106F058F802E0BE2020
:109AE00005F0EAFC206801354844EDB206F06CF858
:109AF000402DE7D1257B45F340151DB1094B0022D0
:109B00001A6009E063692046984708B93D46BEE7F8
:109B1000044B1D6043F8045C2046FBF763F803B078
:109B2000BDE8F08384070842C80638232DE9F84FC2
:109B30000120FBF79BF8044600283CD0037B190763
:109B400039D5052005F0CCFCDFF870804FF0000916
:109B5000C8F8009006F078F818B10138C7B20126AD
:109B600001E00646FE270025BD421DD0237B9A0753
:109B700002D563692046984794F805B0D4F800A050
:109B800006F062F80AF80B00637922799A4238BF2E
:109B900023710133DBB263711BB9237B43F00203F2
:109BA00023730135EDB2DFE7002ED1D02046BDE8AA
:109BB000F84FFBF717B8BDE8F88F00BF84070842DD
:109BC0001B4A002370B513601A4A012010605360CD
:109BD00005F072FC642005F099FC174C23682BB942
:109BE0000020FBF743F8044628B970BD05F09CFC43
:109BF0000028F3D0F4E7114E02252379AB420CD3B1
:109C00002368585D3368984720B12046BDE870400E
:109C1000FAF7E8BF0135ADB2EFE7237B9806F4D43D
:109C20006369204698470028EFD10225E5E700BF89
:109C30008407104280070842E8063823781900108C
:109C40002DE9F04F8DB072B64FF040239A6A22F0A2
:109C500007029A6203F580439A6A22F007029A6229
:109C6000534A012313605360524B1C68002CFCD1F3
:109C70004FF4806506F09CF8013D6040ADB2C4B27F
:109C8000002DF7D1AC2C01D0DC2C08D14A4B9A6ABC
:109C900042F007029A62494B02221A7005E04FF027
:109CA00040239A6A42F007029A62454BFF221A70DB
:109CB00062B6FAF7EFFE424D0446002866D0414FE7
:109CC000414E3B7870228DF80C3002FB036303F1A8
:109CD00030019B6B04AA03C9DB6A82E8030006A873
:109CE00003A99847DFF8F0A0B046A946D3462B78E1
:109CF000FF2B08D1FFF74EFD0028F8D0334A002390
:109D000089F800301370324A0123136028782F4EEF
:109D1000019306F033FE2F2006F0E0FD307806F0C8
:109D20002DFE06F056FE2A78019BF2B9327812B960
:109D3000284A13602AE03278012A13D1DAF8002089
:109D40006432DBF800309B1A002BFADB3978702381
:109D500003FB01839B6B20461E6A9DF81C209DF827
:109D60001D300CE01B4A13600DE03978702000FBB9
:109D70000180806B99F800203378066A2046B0474E
:109D80002068FFF78DFBFF232B70B0E72046FAF722
:109D90000DFF4FF040239A6A22F007029A6203F502
:109DA00080439A6A22F007029A620DB0BDE8F08FF4
:109DB00080070842E806382300800040751900102B
:109DC00084190010C0190010C41900107C1900106B
:109DD000B40B3823340B3823941B001030B51F4BC1
:109DE00070211A781E4B8BB001FB023303F1300156
:109DF0009B6B8DF8042002AA03C9DB6A82E803008A
:109E000004A801A9984706F035F8041E24DB012CAC
:109E10001EDB022C09DD242C1AD19DF814009DF8BC
:109E200015100022FFF75EFBEDE706F023F800288F
:109E300012DBC5B206F01EF8011E0DDB023C6242C9
:109E400062412846C9B2FFF74DFB0028DBD003E092
:109E5000FF2006F041F8D6E70BB030BDC019001066
:109E6000C4190010F8B51C4D06F004F8002831DBC9
:109E700001282BD10020FAF7F9FE044658B9164BF9
:109E80001B683BBBFF20BDE8F84006F025B86369BE
:109E900020469847D0B926792B68701EC0B2CBB93E
:109EA000013606F019F8F6B20223B34209D02A6847
:109EB00082B922685F1CD05CFFB206F00DF83B4609
:109EC000F3E7237B9E06E2D5002000E0FF2006F0AA
:109ED00003F8C9E7F8BD00BFC80638232DE9F047ED
:109EE000484A0123136042F8043C474B0A209A6A0F
:109EF00022F007029A6205F0F3FA444A444B1168D3
:109F00000029FCD11F68002FF9D1424DDFF8FC90E9
:109F1000B846C5F80080D9F8003023B9FFF73AFCFD
:109F20000028F8D06CE001262E6006F03BFDFFF71C
:109F300053FC002864DBFFF74FFC374CB24620701F
:109F4000FFF74AFC2A2360702F60A370334B032273
:109F500000201A70E77004F0BBF806F023FD002023
:109F6000FAF784FE044668B92E60FE20FFF764F914
:109F7000FE20FFF761F9AC20FFF75EF9F720FFF74D
:109F80005BF9C6E766790220C5F800A005F094FAEF
:109F90002368985DAC2801D1FFF74EF92368985DDE
:109FA000FFF74AF92279731CB242DBB201D91E468F
:109FB000EEE7267BAC2046F340161EB1FFF73CF9D6
:109FC000FF2017E0FFF738F9C320FFF735F93220FB
:109FD00005F072FA2E606369204698470028D1D0B8
:109FE000FE20FFF729F9FE20FFF726F9AC20FFF746
:109FF00023F9F720FFF720F92046FAF7F3FD88E769
:10A00000BDE8F0878407084200800040EC06382352
:10A01000E806382380070842FA170010F1170010ED
:10A020002DE9F04106F0BEFC414B01221A600022EE
:10A0300043F8042C3F4B40499A6A22F007029A6287
:10A040003E4A13681BB90B68002BFAD06EE03C4BFC
:10A05000012200241A602546FFF7BEFB002865DBBD
:10A0600023B2EC2B04F10104D8BF4540A4B2D8BF01
:10A07000EDB2B4F5807FEFD1912D01D05B2D55D19C
:10A08000FFF7AAFB041E51DB2E4B2F4D1C70FFF770
:10A09000A3FB00284ADB013CA4B223B2002BE85406
:10A0A000F5DC274D002420462C6004F011F82046F2
:10A0B000FAF7DCFD044618B901232B60BDE8F081F6
:10A0C00072B61F4EDFF8688001273760C8F800704D
:10A0D00020790138C0B205F039FF80B9022501E0CE
:10A0E0000135ADB222792BB2934205DC2268D05CF7
:10A0F00005F02CFF0028F3D00F4B1B6853B162B65C
:10A100000F4A01231360043213602046BDE8F0417A
:10A11000FAF768BD237B43F34013002BEFD1336084
:10A120006369204698470028CFD0E8E7BDE8F08172
:10A130008407084200800040C8063823EC06382314
:10A1400080070842F1170010FA1700102DE9F047B8
:10A15000FAF7A0FC0546FAF79DFC0446002D00F036
:10A160001D81002800F01A812D6806F01BFC0120DB
:10A1700005F0B6F98A4B00221A608A4A1368002B50
:10A18000FCD04FF00108DFF83C92C246864EC9F879
:10A1900000A02846FFF7B2FBC6F800806A782B784B
:10A1A00043EA022340F27C42934200F0C28031D85D
:10A1B00040F21242934200F0988015D8B3F5487FE0
:10A1C00000F08B8007D8002B00F08F8040F21F3208
:10A1D000934272D0D8E040F22532934200F0828060
:10A1E000063293427ED0CFE040F23942934200F0F3
:10A1F000928007D8B3F5846F77D040F23242934211
:10A200007CD0C1E040F2574293426ED01E3293425E
:10A210006BD0B9E040F2DC429342B8D014D840F29F
:10A22000AF42934254D007D840F29B429342AED003
:10A230000A3293426FD0A7E040F2B9429342A6D0CF
:10A24000133293426DD09FE040F27E5293429ED0F3
:10A250002BD840F20452934299D07832934240F086
:10A260009380AF785720EE7806F038FB384606F03A
:10A2700085FB2F2006F032FB304606F07FFB06F010
:10A28000A8FB2046FAF708FD2068FFF737FB474B8D
:10A2900070221978464B204602FB01339B6B3A46ED
:10A2A000D3F824C03346E0476AE040F28E5293422E
:10A2B00037D0703293423CD066E03E4B1B780E2B79
:10A2C00010D195F90230002B07DA2068022107E04F
:10A2D000A878E9782246FFF7BFF820684FF480712C
:10A2E000FFF752F8FFF73CF850E72E4A1368002BAF
:10A2F000FCD12B4B01221A60BDE8F0872E4B187859
:10A300000028EFD12668FFF70BF830464FF4807134
:10A31000FFF73AF83AE7AA78284B02F01F021A70C2
:10A3200034E7A878E97800F07F002246FFF794F838
:10A330002CE7AF785720EE7806F0D0FA384606F0D2
:10A340001DFB2F2006F0CAFA304606F017FB06F078
:10A3500040FB2046FAF7A0FC20684FF48071FEF71E
:10A360008FFF124B70221978114B204602FB0133EC
:10A370009B6B3A46D3F824C03346E047FEF7F0FF24
:10A380002046FAF79BFC01E70D4806F020FB284623
:10A3900000210422BDE8F04706F024BBBDE8F087A9
:10A3A00084070842E8063823B40B3823C01900108C
:10A3B000C41900107519001072190010BD19001091
:10A3C00040240100340B38232DE9F04F044685B0BA
:10A3D0006620FAF74BFC0746FAF774FB0646002F97
:10A3E0005DD000285BD02F4B2F4D002C08BF1D46A1
:10A3F00006F0D8FA012005F073F82C4B00221A6001
:10A400002B4A1368002BFCD0DFF8A890DFF8A8A037
:10A4100002354FF0000815F8024C002C39D015F821
:10A42000013C4FF0700B99F8001030460BFB01A275
:10A43000926BD2F820C02246E047B8F1000F05D158
:10A440003268147853786CB1FE210DE03468002333
:10A45000E21818F80310907801334140FE2B9170F8
:10A46000F6D1EDE7591EC9B2084601930291039255
:10A47000FEF756FF039A0299901CFEF785FF019B99
:10A48000002CD0D12046FEF74BFF0235D7F80080D4
:10A49000C1E73846FAF78AFB044B01221A6005B07F
:10A4A000BDE8F08F392401006A24010084070842C6
:10A4B000E8063823C0190010C419001010B504466E
:10A4C00006F070FA022005F00BF81D4A1368002B05
:10A4D000FCD01C4B00221A601B480CB91B4900E041
:10A4E0001B49FAF7B3F91848FAF70EFA194B187026
:10A4F000002003F0EDFD0020FAF7B8FB044630B968
:10A500000F4A0DE06369204698470028F8D120687B
:10A510004FF48071FEF760FF237B9B06F0D4F1E7D8
:10A520001368002BFCD1074A01231360043A13601F
:10A5300024B12046BDE81040FAF754BB10BD00BF5F
:10A54000E806382384070842FA1700104E24010059
:10A550004B240100F1170010F7B5FAF79BFA0446F7
:10A56000002800F0FB8006F01DFA012004F0B8FF7F
:10A570007B4A1368002BFCD07A4B00221A60012220
:10A5800043F8042C032004F097FF754D2B683BB172
:10A59000754B1B6823B9FFF7FDF80028F6D0DDE006
:10A5A00001A80421FEF78EFE704B01221A609DF86F
:10A5B0000430033B182B00F2B880DFE803F00DB63F
:10A5C000B615B6B642B6B64AB6B663B6B653B6B662
:10A5D00066B6B67CB6B69400614A1368002BFCD10F
:10A5E000604B01221A60B9E09DF8067057209DF873
:10A5F000076006F073F9384606F0C0F92F2006F020
:10A600006DF9304606F0BAF906F0E3F92046FAF79C
:10A6100043FB20684FF48071FEF754FE544B7022C8
:10A620001978544B204602FB01339B6B3A46D3F812
:10A6300024C03346E047FFF76DF82046FAF73EFBAB
:10A640007CE09DF806009DF8071022464FF48073C9
:10A6500005E09DF806009DF8071022460223FFF74B
:10A660006BF86BE0424B70221878424B02FB0033D0
:10A670009B6BDB69984702AB23F8080D0221684603
:10A68000FEF7AAFEFFF746F858E0394B394A1B7827
:10A69000702101FB032292F83410303252798DF888
:10A6A00000100133684603218DF801208DF8023037
:10A6B000FEF792FE42E068460321FEF703FE9DF896
:10A6C00002202B4B0AB1013A1A702A4A1B787021DA
:10A6D00001FB03239DF8002083F834209DF801201E
:10A6E00083F835202AE072B6234E33780BB103206D
:10A6F00012E0224B1B78122B0DD11D4B1D4A1B78EB
:10A70000702101FB032393F8603003F07F03032BD8
:10A7100001D1802000E00020FEF7C2FF002333704B
:10A720002B68002BFCD062B608E0154806F04FF904
:10A7300001A80021042206F055F90FE0114B012277
:10A74000094E1A602B68002B7FF420AF3368002B72
:10A750007FF41CAFFFF71EF80028F3D003B0F0BD64
:10A76000E806382384070842C8063823B40B382388
:10A77000C0190010C4190010841B001075190010B6
:10A7800040240100340B38232DE9F04F644885B094
:10A7900006F01DF9634B9A6A22F007029A62FAF7F3
:10A7A00079F9044620B1012700255F4EB8461EE026
:10A7B0005E48ADE0FEF7EEFF0546002840F0A480BD
:10A7C000D9F800205A4B002AF4D0002D40F09C808C
:10A7D000584A1560584A17601D68002DFCD10DF1CC
:10A7E0000E00FEF729FF90B94FF0000B5D46514B6C
:10A7F000C6F80080C3F80080504BDFF83491C3F8EE
:10A80000008006F0E6F84C2006F068F8D8E75420FF
:10A8100006F064F89DF80E0006F0B0F89DF90E30D1
:10A82000002B71DB0DF10F00FEF706FF0028DBD0D7
:10A83000532006F053F89DF80F0000F07F0006F05B
:10A840009DF89DF80F301A0643D503F07F03522080
:10A850008DF80F3006F042F8394B70221978394BD9
:10A86000204602FB01339B6B9DF80E20D3F820C0DD
:10A870009DF80F30E047DFF8BCA022685FFA85FB47
:10A8800012F8059072B60320CAF8008004F014FE96
:10A8900008220192FEF7B6FE019A90B119F001016B
:10A8A00014BF376031604FEA5909274B19680029F6
:10A8B000FBD1013A12F0FF02EBD1CAF800200120CF
:10A8C000376062B6002891D00135B5F5807FD4D1CC
:10A8D0008AE7572006F002F820682844FEF7ACFE0D
:10A8E00090B10135B5F5807FF6D1154B70221978FE
:10A8F000144B204602FB01339B6B9DF80E205D6AD2
:10A900009DF80F30A8476FE72046FAF74FF90F4838
:10A9100006F05DF806F05DF805B0BDE8F08F00BF09
:10A920005624010000800040840708425D24010095
:10A93000C806382380070842B40B3823340B382369
:10A94000C0190010C4190010E8063823652401005E
:10A9500038B50020FAF78AF9044650B3154B0022A7
:10A9600001201A60586004F0BBFD207902250138EF
:10A97000C0B205F097F92379AB4206D32368585D3E
:10A98000013505F08FF9ADB2F5E7237B99060AD5BD
:10A99000002005F087F9012004F0A2FD054A0123FB
:10A9A0001360536038BD6369204698470028DCD0A7
:10A9B000EEE738BD80070842F8B50120FAF756F9EE
:10A9C000044638B3144B002501201D60586004F084
:10A9D00087FD2E462046FAF75FF90025276805F027
:10A9E0008BF978550135B5F5807FF7D123681A7852
:10A9F00012B95B78637100E066716369204698471D
:10AA000018B923681B78002BE4D12046BDE8F84034
:10AA1000FAF7E8B8F8BD00BF80070842014B0122F1
:10AA20001A7070477419001038B572B6204C23683C
:10AA300033B103F04FFF0028F9D04FF6FF701CE050
:10AA40001C4B01221A60562004F060FD184C03F0E4
:10AA500041FF05460028F0D104F066FD10F0FF0F1D
:10AA60000ED12368002BF2D005F0EAFA044605F077
:10AA700003FB104B00221A60204662B600B238BDBC
:10AA80000C4C3920256004F017FD0123236045207C
:10AA900005F024FF084B064C1A7842F001021A70A8
:10AAA0002368002BE0D103F015FF0028F8D0C4E79D
:10AAB000E806382384070842B9190010194B70B50D
:10AAC0000122194E04460D461A6033682BB103F07B
:10AAD00001FF0028F9D0FF2070BD4DB9204605F0D8
:10AAE000B5FA05F0C9FA0F4B00221A600E4C14E0BB
:10AAF0000D4D2B6823B903F0EDFE0028F9D0EAE7ED
:10AB0000094D2B68002BE9D003F0E4FE0028F8D0B3
:10AB1000E1E703F0DFFE0028DDD12368002BF8D049
:10AB2000002070BD80070842EC06382370B5002075
:10AB3000FAF79CF8044600284DD0022343716420A4
:10AB400004F0BAFC012005F08DFA234A00231360BB
:10AB5000224A6420137004F0AFFC05F08DFA05F072
:10AB600021FF642004F0A8FC1D4E237B980615D419
:10AB7000236875699878FEF737FD2D0126D50325E2
:10AB80002368585D0135FEF72FFD15F0FF05F7D15D
:10AB90006369204698470028E7D017E0022523681C
:10ABA000585DFEF721FD22796B1CAA42DBB201D968
:10ABB0001D46F4E7084B01221A600A4B1D68002D60
:10ABC000FCD105F059FA284605F04CFA2046BDE8BC
:10ABD0007040FAF707B870BD80070842741900107A
:10ABE00020C00920EC0638232DE9F8430120FAF7AC
:10ABF0003DF8044600283CD00223437103716420D1
:10AC000004F05AFC002005F02DFA1B4B00251B4ECA
:10AC10001D60357005F030FA05F0C4FE184F237B37
:10AC20009B0703D563692046984710BB3378002BF8
:10AC3000FCD094F80590D4F8008005F001FA08F8EB
:10AC400009002046FAF728F8637922799A4238BF3A
:10AC500023710133DBB263711BB9237B43F0020321
:10AC60002373D7F80080357005F006FAB8F1000FAD
:10AC7000D5D1BDE8F88300BF8407084274190010DD
:10AC8000E80638232DE9F74FF9F704FF06460028B8
:10AC900000F0D080694B01259A6ADFF8AC8122F080
:10ACA0000702674C9A620827A9460023C8F800905B
:10ACB00040F20550236004F0FFFB013F256040F2A5
:10ACC0000A5004F0F9FB17F0FF07EED15D4C636901
:10ACD000DB4303F04063B3F1406F04D0FEF75AFD4D
:10ACE0000028F4D0A6E00124574D554F4FF000083E
:10ACF000A346564B00222A600320C7F800B0C3F8D1
:10AD000000B004F0D9FBDFF85891D9F8003023B92E
:10AD1000FEF740FD0028F8D00AE02C60FEF78EFD1B
:10AD2000002805DB5FFA80FAFEF788FD002803DAC9
:10AD3000464B01221A607DE05FFA80F9FEF77EFD46
:10AD40000028F5DB424BC0B230281C60C5F80080FB
:10AD500004D040283AD0202866D1E9E73D4B702244
:10AD600019783D4B304602FB01339B6B5246D3F8BA
:10AD700020C04B46E047394B1B78002B54D12C6048
:10AD800003203C6004F098FBD6F800A00AF5807917
:10AD90001AF8010B012805D01AF8010CFEF782FD04
:10ADA00028B1C5E7FEF77EFD0028F5D0C0E7CA450B
:10ADB000EED10120FEF776FD0028B9D18120FEF703
:10ADC00071FD0028B4D128603C6092E72C6003201C
:10ADD0003C6004F071FB336830460193F9F75CFF87
:10ADE00000230093FEF72AFD0028009BA0DB019AB8
:10ADF000D0540133B3F5807FF3D1164BC5F80080F2
:10AE00001978154B702202FB01339B6B3046D3F847
:10AE100024C052464B46E0473046F9F74FFF0F4BF0
:10AE20001B78002B3FF465AFFEF79CFD00283FF434
:10AE300060AF7DE703B0BDE8F08F00BF0080004049
:10AE40008407084220C0092080070842340B3823B9
:10AE5000B40B3823C0190010C41900107219001067
:10AE6000EC06382310F8013BA3B103F13F02D2B244
:10AE7000192A01D8803B05E0A3F14102D2B2192A78
:10AE800002D82033DBB202E0FF2B08BF7E2300F89C
:10AE9000013CE7E7704700000378124A702000FB8E
:10AEA000032393F82930022B06D0032B0AD0012B61
:10AEB0000FD10B46312207E031220B4603F8022B5B
:10AEC000362204E00B46332203F8022B32224A706A
:10AED000194620230B7032234B7041238B700020C6
:10AEE000704700BFC41900101E20FEF79BB9000078
:10AEF00010B50C462E21F9F76BFD2060002835D0E7
:10AF0000431C236043788278502BC17806D0552BA0
:10AF100004D0A3F15200C0B2012825D8144800681B
:10AF200084186478640703D508444078400719D42E
:10AF3000502B05D1522A19D1472917D1022010BD13
:10AF4000532B03D1452A11D15129F6E7522B03D1B6
:10AF5000452A0BD14C29F0E7552B07D1532A05D1AF
:10AF60005229EAE7012010BD522BF1D0002010BD7C
:10AF70000000001013B50B4B70224FF6FF7402FB5C
:10AF80000030094901AA234602F06AFB20B9019862
:10AF9000A04203D880B202E0002000E0204602B0C8
:10AFA00010BD00BFC41900104A2401000A4B1B68E1
:10AFB00003445B785B070DD121280BD0A0F123035C
:10AFC000DBB2062B06D9B0F12D0CDCF1000050EB02
:10AFD0000C007047012070470000001003460A462D
:10AFE000112831D8DFE800F009140C0F11142721C3
:10AFF000171E14142C302A2A240F0020FEF712B931
:10B000003E2002211EE0272003E02120042119E038
:10B010004A20194616E012B11420082112E0192026
:10B02000082114E01A2009210CE03F20072109E043
:10B030003F20102106E04820062103E03F20E8E7FA
:10B040004A200C21002202E01F2019466322FEF74D
:10B0500007B873B504462F2005F040FC237B9A0700
:10B0600002D46379013B23712079E379984208DCAB
:10B070002168C0F10102013008441A440021F9F7A7
:10B0800021FBE3790BB1013323712279216804F1AB
:10B090001C06013A3046023192B20DF1060302F06D
:10B0A000B3F8054638B1722005F018FC2846012196
:10B0B000FFF794FF0BE02379BDF80620013B9A428D
:10B0C0000DD06C2005F00AFC4820FEF7ABF83046A6
:10B0D00002F07DF92046F9F769FD01200FE02046D6
:10B0E000F9F7ECFD237B94F8402065F341032373CB
:10B0F000022363712371636A28469B1AA36002B01E
:10B1000070BD2DE9F84390F84010866A8368761A7E
:10B11000B34204460BD000F11C052846194402F046
:10B120005DF920B10121FFF759FF28464DE0A568E0
:10B130002046B5428CBFC6EB05050025FFF789FF09
:10B140008046002846D1002D4CD094F8401004F1E0
:10B150001C073144384602F041F9237BE27968F359
:10B16000410323732368003A18BF6FF00002A66002
:10B170009A708146206841460330FD22F9F7A2FA11
:10B18000B9F1000F19D03846A16A02F027F9054637
:10B1900018B3722005F0A2FB28460121FFF71EFF1D
:10B1A000384612E0237123792046ED1A0233637189
:10B1B000FFF74FFF70B9002DE5D0E379002BF1D1F7
:10B1C000FE2D94BFEBB2FE23ECE702F000F920461F
:10B1D000F9F7ECFC0120BDE8F88394F84020636A9D
:10B1E0009B1AA3602846BDE8F88337B504462320A0
:10B1F00005F074FB94F84020636A21689B1AE27999
:10B20000A36004F11C000231002A08BFFE220DF1E8
:10B21000060301F061FF38B10121FFF7DFFE204690
:10B22000F9F7C4FC012030E0BDF806304BB901232A
:10B23000E279ADF806302368002A0CBF0D22FF2208
:10B240009A7002236371BDF80630E0795A1C2271AE
:10B2500018B9FD2B237B0BD80FE0216822798D5C78
:10B26000002DF6D1013AD2B2012A2271F6D8F0E7C8
:10B27000A16A626A914200D020B143F02003237397
:10B28000002002E060F34513237303B030BDF8B52E
:10B2900090F84070037B0E460F44D90604461546CD
:10B2A00003D4A36ABB421CD304E0FFF72AFF0028A3
:10B2B000F7D00FE004F11C063046394602F08EF854
:10B2C00050B10021FFF78AFE304602F080F8204698
:10B2D000F9F76CFC0120F8BD2046FFF786FF68B146
:10B2E000F8E7E2792368002A0CBF0D22FF229A704A
:10B2F00002232371A6603220FDF794FFAB1C63711B
:10B30000237901359D42A8BF63710020F8BDC17942
:10B31000836800221944FFF7BABF00002DE9F0410D
:10B320000D460646084614468846FFF79BFD95F8ED
:10B3300020300BB105F12008174B3078702202FB4A
:10B340000030716804F11C0781613078394602FBD6
:10B3500000304246012301F0F1FD20B10121BDE89A
:10B36000F041FFF73BBEEB7E022B06D138461A2197
:10B3700002F034F81A2384F84030084A237BA26193
:10B38000074A43F044036261064A23732261204660
:10B39000BDE8F041FFF729BFC4190010A9B30000B0
:10B3A000EBB100008FB2000038B5027B044642F3D7
:10B3B0000003ABB115070DD404F11C0002F007F82F
:10B3C00001210546FFF70AFE064B281CA36118BFA2
:10B3D000012038BD436998470028EDD0012038BDD1
:10B3E000184638BDF949000038B50A4B0A780546B9
:10B3F000702000FB02300C462A1D496802F074F8E8
:10B4000023782B7020B10121FFF7E8FD012038BD22
:10B4100038BD00BFC41900102DE9F043934B8DB027
:10B4200006460C460B9300F1040842F62E67404690
:10B4300003A902F073F850B10C2803D14720FDF79F
:10B44000F1FE02E00121FFF7C9FD012009E19DF8AD
:10B450001C501DB19DF814301A07E8D4BDF81C30FB
:10B460002E2BE4D0079B23F07F43BB42DFD0204646
:10B4700000213022F9F726F9002D00F0F180012398
:10B4800007AFE37604F120003946F9F7DFF90B9DA9
:10B490002B7843B12846F9F737FA142803D8284601
:10B4A00006F053FC00E03D469DF8143003F0100315
:10B4B00003F0FF0733B1062363742B782E2B79D169
:10B4C000262376E007A802A9FFF712FD012850D134
:10B4D0003078069905F070FD029B93F8008048B122
:10B4E000234600F1100250F8041B904243F8041B5D
:10B4F000F9D138E030784FF0700909FB00F05C4F6B
:10B50000069A391808463C3101F0D8FD00283FD191
:10B510003378564909FB03701A223C300DF10603BB
:10B5200001F0DAFD002833D1504852490722F9F7DB
:10B5300043F8074660BB20464F49F9F787F9029464
:10B540001023029A013B1178A02908BF1770029AB4
:10B5500013F0FF0302F101020292F2D13078069952
:10B56000224605F049FD039B1A3B03930223E37631
:10B570000EE0022816D1414B1B781B0712D5029B07
:10B58000284693F80080F9F7BFF90438C0B22F5469
:10B59000A8F15008B8F1050F0CD8DFE808F0030B4C
:10B5A00009050B07022304E0012302E0032300E066
:10B5B00004236374E37E022B06D1039B304A93423B
:10B5C00019D94FF6FF121BE02846F9F79DF910280C
:10B5D0008CBF07A929462046F9F738F90294FF21C4
:10B5E000029A1378002BE8D07E2B08BF1170029BC3
:10B5F00001330293F4E703F1FD01FE22B1FBF2F205
:10B600006282FE22B3FBF2F102FB113323759DF837
:10B610001430DE0703D5627C42F04002627413F0FE
:10B62000060F03D0637C43F020036374069B002065
:10B63000E361BDF810305A0A50326275C3F3431209
:10B6400003F01F03E375BDF81230A275DA0A227603
:10B65000C3F3451203F01F035B006276A37600E09C
:10B66000FF2040B20DB0BDE8F08300BFA41700106A
:10B67000C4190010C1240100AC170010F31700100A
:10B68000020BF80038B5164B01221A6091F82030F1
:10B69000044623B101F1200505F082FC03E00846D1
:10B6A0000D46FFF7DFFB0F4B2078702202FB0030C6
:10B6B000616881612078294602FB003002F032F88F
:10B6C000044603F0C1FD20460021FFF787FC24B1AA
:10B6D000022C14BFFF20002038BD012038BD00BF60
:10B6E000EC033823C4190010F8B50B4E027870270C
:10B6F00007FB026243680446936108460D46FFF764
:10B70000B1FB2078294607FB006002F0A3F8BDE8F2
:10B71000F8400021FFF762BCC419001070B5002486
:10B720008EB00646112208460D4621460D94F8F7C4
:10B73000C9FF194B702000FB063021466A4601F014
:10B74000D3FE20B12146FFF749FC012021E06846E5
:10B7500005A901F0E3FE10B99DF824300BB90020D3
:10B7600017E09DF81C3003F00E03082BEFD10122E7
:10B770000446531EDBB20EA90B4413F8143C002BF5
:10B78000EDD02E2B02D0611C2B55CCB20132D2B29F
:10B79000EFE70EB070BD00BFC41900102DE9F043F3
:10B7A000DFF8C8808FB00546102208460E462021DB
:10B7B000CDF834802C4FF8F785FF2B78702000FBF4
:10B7C000037069686A4601F08FFE0446002841D183
:10B7D00042F62E69684605A901F0A0FE044658BB52
:10B7E0009DF824302E2B05D028782049FFF796FFAE
:10B7F000044621E0099B23F07F434B45EAD12B7897
:10B80000702000FB037008996A4601F06DFE044643
:10B8100090B9684605A901F081FE044660B99DF81B
:10B8200024304BB16B68089A9A42F2D198F80030F4
:10B8300023B10E4806F089FA0C4D00E009AD2B78D3
:10B840003BB12846F9F760F8294602463046F8F73A
:10B85000E7FE2CB120460021FFF7C0FB012000E0ED
:10B8600020460FB0BDE8F083C4190010A4170010E3
:10B8700073B5002A0CBF12230123144670225143D2
:10B8800006461348134A45183C350844294601F03A
:10B8900055FBC0B9284631684FF480720DF106039C
:10B8A00014B101F019FC01E001F0AEFC20B9BDF8C3
:10B8B0000630B3F5807F02D02146FFF78FFB284684
:10B8C00001F085FD10B12146FFF788FB02B070BD85
:10B8D000C4190010B4240100012A00D123B111467B
:10B8E00014201A46FDF7BCBB1A46FFF7C1BF012A58
:10B8F00010B5144600D133B1214614201A46BDE8D4
:10B900001040FDF7ADBBBDE81040FFF7B1BF000030
:10B9100010B52E21F9F75CF800283AD01D4A43787B
:10B920001268D118497801F00301022908BF203BB1
:10B93000D9B28378C078D41864780244527804F07D
:10B940000304022C02F0030208BF203B022A08BFB6
:10B9500020384D29DBB2C0B206D1322B18D1B0F15C
:10B9600049014842484110BD442911D1362B03D129
:10B97000342807D1022010BD4E2B01D1502806E0FB
:10B98000342B03D0373BDBB2012B01D83128F1D067
:10B99000002010BD000000102DE9F041394B0D468C
:10B9A000044641680078702202FB003081612988DA
:10B9B0008AB05F291F4612D133492E200870487083
:10B9C00000208870207802FB003001AA01F020FEE0
:10B9D000002838D1049BEB6106236B7403E02878C0
:10B9E00008B960604BE06B7C03F00703062B03D1C2
:10B9F000EB696360002042E020352846FFF788FFAE
:10BA000000283CD00520F9F7F7F820784FF07008AF
:10BA100008FB00F0391808462A463C31032301F0A0
:10BA20008DFA0628064601D009280AD123782A462D
:10BA300008FB03F03918084601233C3101F07EFA77
:10BA4000064626B130460121FFF7C8FA16E028461F
:10BA5000FFF75EFF012805D12378702202FB0377F0
:10BA60000A4B09E020462946FAF7A2FD30B92378AF
:10BA7000702202FB0377064BBB63BBE701200AB0D1
:10BA8000BDE8F081C4190010A4170010F0270100D0
:10BA9000BC1E010070B505463148FFF7E3F90F2DD4
:10BAA0002F4C3BD0022D04D12046FFF731FF002858
:10BAB00034D12C4B1E78012E02D1022D12D101E07F
:10BAC000022E0FD02378202B0CD0274B58785C1CEB
:10BAD00020B1FFF76BFA28B12346F7E714F8013CD1
:10BAE000202B02D11E4C5F2608E02E2B18D1F9E73F
:10BAF000FFF75CFA631C00B926701C46207800280A
:10BB0000F6D12E23237003235D43184B2071EB5C89
:10BB1000E01C63703023A370E37070BD002070BD23
:10BB2000032E03D1022D19D00F4A02E0042EFBD0C0
:10BB300070BD5078531C1A460028FAD12E2102F805
:10BB4000011B0A49032405F00F0504FB051529888C
:10BB5000A3F80110A9789170187170BD70BD00BF75
:10BB6000A417001085190010A31700103C25010030
:10BB70002DE9F34790463A4D0278702707FB0252B1
:10BB800043680646936191F81BA00C46BAF1020F78
:10BB900001F120093AD105F003FA30784A4678439A
:10BBA0002918084653463C3101F0C8F9814600285F
:10BBB0004FD13078082107FB00503C3001F00EFCDB
:10BBC000014608B1494645E010222046F8F77AFDC3
:10BBD00020464146F8F73AFE3078214607FB0050F0
:10BBE00010223C3001AB01F00FFB044618B9BDF840
:10BBF0000430102B01D020462BE0337807FB035094
:10BC00003C3001F0E4FB38B3214623E0484601A96B
:10BC1000FFF76EF902280ED141461248F8F716FEDA
:10BC2000607C00F00700FFF735FF3078494607FBDE
:10BC300000500C4A0AE02046FFF714F94046FFF78F
:10BC400011F93078214607FB0050424601F0D8FE3A
:10BC500010B10021FFF7C2F902B0BDE8F08700BFC4
:10BC6000C4190010A41700102DE9F04F1E4691F8DA
:10BC7000203085B080460F4614469DF838501BB1E1
:10BC800001F1200A002408E03448F8F7DFFD2046DF
:10BC9000FFF700FFDFF8C4A00446314B98F800100E
:10BCA0004FF0700C0CFB0131D8F804209B468A61E0
:10BCB00006F11C0998F8000049460CFB00B0002D65
:10BCC0000CBF062307235246CDF804C001F036F915
:10BCD00007280146DDF804C013D1002CEAD02378F0
:10BCE0000133DBB23A2B2370E4D14FF030032370E1
:10BCF00014F8013C0133DBB23A2B04F8013CD9D1F2
:10BD000028E038BB14B9BDB9284624E01A221348EC
:10BD1000F8F7D8FC11481349F8F798FD124B07F1D2
:10BD2000100257F8041B974243F8041BF9D10DB1D8
:10BD30000A4B5D761A2302E0084B1D70012386F83A
:10BD400040304846054996F840200DF10E0301F0B9
:10BD50005BFA00E0084605B0BDE8F08FA4170010BC
:10BD6000C4190010C1240100AC170010F7B59DF8EC
:10BD7000206005460F461C4616B341681E4B0078EE
:10BD8000702202FB00308161287804F11C0602FB5E
:10BD900000303146022307F1200201F0CFF8FB7E8C
:10BDA000022B04BF1A2384F8403018B93046A16A28
:10BDB00001F014FB94F84020A36A9B1AA36002E0F0
:10BDC0000096FFF751FF28B1002103B0BDE8F04015
:10BDD000FFF704B9237B0D2243F0480323730223AA
:10BDE00063712371054BA361054B6361054B2361AF
:10BDF00023689A7003B0F0BDC4190010A9B3000005
:10BE000003B100008FB200002DE9FF411D469DF8EF
:10BE1000283007468846144653B923460095042225
:10BE2000FFF722FF0123ADF80E30284B1D7027E0ED
:10BE30004168274B0078702202FB0030816138781E
:10BE400004F11C0602FB0030314608F120020323F6
:10BE500001F074F8C8B998F81B30022B07D03046AF
:10BE60001A4901220DF10E0301F036F905E03046C2
:10BE7000192101F0B3FA0028F1D00DB9134B1D7848
:10BE800018B9BDF80E30012B03D00021FFF7A6F83A
:10BE900018E0636AE57184F84030237B204643F064
:10BEA0004C0323730B4BA3610B4B63610B4B23615F
:10BEB000FFF79BF930B9054B1B78AB4202D032201B
:10BEC000FDF7B0F904B0BDE8F08100BFA417001081
:10BED000C4190010A9B300000FB300008FB2000016
:10BEE0002DE9F84F224F0024DFF89480DFF894B05A
:10BEF00005463C702646BA463978032929D8072ECC
:10BF000027D84FF0700909FB018104EB0610C1F836
:10BF100038B0C0B201F00AF825B99AF8003009FB30
:10BF200003831D6330B93B780E2C03F101033B7092
:10BF300005D90AE0012808D00C2806D003E024B176
:10BF40000134E4B2D8E70E2CFAD90136F6B2002457
:10BF5000D2E73DB9074B284607491D70FAF794FD13
:10BF6000064B1D70FAF7FEFBBDE8F84F05F018B858
:10BF7000C1190010C01900104A24010088190010CE
:10BF8000C41900107424010070B504460E4D05203C
:10BF9000F8F732FE702303FB0452916B0B4A1E46E6
:10BFA000914202D12046FAF7F3FB7443084A2B1959
:10BFB0009A6303F13C0001F00AFA20B10021FFF777
:10BFC0000DF8012070BD70BDC4190010BC1E010029
:10BFD000742401000B885F2B02D10078FFF7D4BFD7
:10BFE000012070471F20FDF71DB90000F7B5054679
:10BFF000481C17461C46104E06D0702000FB0560FA
:10C000003C3001F0EBF950B9702303FB0560394671
:10C010003C3022460DF1060301F05EF820B101210B
:10C02000FEF7DCFF022004E0BDF80600001B18BF8D
:10C03000012003B0F0BD00BFC41900102DE9F34189
:10C040004E1C074690461D469DF82040164E08D0CF
:10C05000702000FB07603C3001F0C0F908B10021FE
:10C060000DE0702303FB07663C36304641462A4606
:10C070000DF1060301F0C8F8074620B10121FEF7D3
:10C08000ADFF02200CE0BDF80630AB4205D134B163
:10C09000304601F069F9384602E0012000E0204610
:10C0A00002B0BDE8F08100BFC419001083680239F6
:10C0B000023B994205D290F82A20436902FB0130E5
:10C0C00070470020704730B500F1100300240A5D6E
:10C0D000202A07D00134052A08BFE522082C03F8DE
:10C0E000012BF4D10A7A202A0DD01A462E2402F808
:10C0F000044BCD1D013315F8014F202C03D003F85C
:10C10000014B9342F7D100221A70CB7A0372CB69AC
:10C1100003600B8B8380CB8AC3808A8A4B8B43EA74
:10C120000243C36030BD10B5036814461A782F2A45
:10C1300008BF013303600B688BB193F829200AB95B
:10C14000012010BD93F82C0005F024FBC307F7D4A1
:10C150003CB110F0040F0CBF0020092010BD0A20D4
:10C1600010BD204610BDA0F16103DBB2192BA0F178
:10C17000200301D8D8B27047DBB20A2B1ED9A0F138
:10C180004103DBB2192B19D9A0F13003DBB2092B23
:10C1900014D9020612D4602808D85E280ED22C28A2
:10C1A0000BD32D280AD93D2807D170477B2805D00D
:10C1B00003D3A0F17D03012B00D95F20704708B5A0
:10C1C00048B190F8293033B190F82C0005F0E2FA2C
:10C1D00000F0010008BD0C2008BD00002DE9F04171
:10C1E000224B07461D680E468D429C6801D1A04235
:10C1F00038D01B79DFF874800BB99EB325E094F832
:10C200002C0008F10C012A46012305F009FC10B1AD
:10C210000020BDE8F08188F804006268E3681344F8
:10C220009D42EAD294F82B80B8F1010FE5D96368FA
:10C2300094F82C001D440E492A46012308F1FF38CA
:10C2400005F0EEFB5FFA88F8EEE7084C97F82C0053
:10C2500004F10C013246012305F076FB0028D7D10A
:10C260002660A7600120BDE8F08100BFA40F001088
:10C27000B00F0010FFF7B2BF70B506460C46FFF7CF
:10C28000F9FF08B9022070BD134D54B996F82C007F
:10C2900005F10C012246012305F056FB0028F1D1DF
:10C2A0002860B5F80A224AF655239A420A4CE9D189
:10C2B00004F1420009490322F8F77EF958B104F16C
:10C2C0005E0006490522F8F777F918B994F83400AA
:10C2D000C00970BD012070BDA40F0010D62401005C
:10C2E00001292DE9F84306460C4651D98368994245
:10C2F0004ED290F82930C568022B2DD0032B38D0B0
:10C30000012B45D18BB203275F43C7F34F0705EBE2
:10C310005721FFF7AFFF00283AD0C7F30803DFF833
:10C320007C800137BFB24344304605EB572193F878
:10C330000C90FFF79FFF58B3C7F308074744387BBB
:10C34000E10749EA002002D50009BDE8F883C0F3FF
:10C350000B0080B2BDE8F88305EB1121FFF78AFFDF
:10C36000B0B10D4B640004F4FF741C44A088BDE818
:10C37000F88305EBD111FFF77DFF48B1064BA40010
:10C3800004F4FE741C44606820F07040BDE8F8833B
:10C390000120BDE8F88300BFAC0F0010A40F00100F
:10C3A00038B5058804460135ADB228071DD123698B
:10C3B000E16801332361606821B90388AB4214D876
:10C3C000002038BD90F82A30013B13EA15130CD138
:10C3D000FFF786FF01280146F2D960688368994219
:10C3E000EED2E160FFF762FE20612580012038BDBA
:10C3F0002DE9F84390F829308046022B0C4615466B
:10C40000C6683FD0032B49D0012B57D18BB24FF0D8
:10C41000030909FB03F9C9F34F0906EB5921FFF79B
:10C4200029FF00284AD014F00104C9F30802254F5F
:10C43000EBB206D0B918097B01F00F0141EA0313F2
:10C44000DBB209F101093A441FFA89F91373404636
:10C45000012306EB59213B71FFF70CFF70B3C9F3C1
:10C4600008091FFA89F914B1C5F3071507E0154B40
:10C47000C5F303254B441B7B23F00F031D434F449F
:10C480003D7316E006EB1121FFF7F4FEB0B1640036
:10C490000D4B04F4FF741C44A5800AE006EBD11197
:10C4A000FFF7E8FE50B1A400074B04F4FE741C44EF
:10C4B0006560044B01201871BDE8F8830020BDE8D9
:10C4C000F88300BFA40F0010AC0F00102DE9F0415D
:10C4D0000546D0F808800F4629B9C66976B14645A9
:10C4E00028BF01260BE0FFF7FBFE012802D8012040
:10C4F000BDE8F081404532D33E4600E00126344697
:10C500000134444505D3012E02D80020BDE8F08156
:10C51000022428462146FFF7E3FE20B10128E6D099
:10C52000B442EDD1F1E7284621466FF07042FFF7A3
:10C530005FFF0028DBD04FB92B6AEC615E1C0DD089
:10C54000013B2B62012385F8283007E02846394655
:10C550002246FFF74DFF0028EED1C8E72046BDE890
:10C56000F081F8B504460D460127012D1BD9A368BB
:10C570009D4218D220462946FFF7B2FE0128064602
:10C5800001D10020F8BD204629460022FFF730FFE8
:10C590000028F6D0236A5A1C03D00133236284F8A2
:10C5A00028703546E1E70120F8BD00002DE9F74F7E
:10C5B0000D231932876892FBF3FB80460191446892
:10C5C0001FFA8BFB3FB1C76039462046FFF76EFD6F
:10C5D000C8F8100001E0236903610026A8F8006094
:10C5E0000096B14635462046D8F81010FFF742FEB7
:10C5F00008B908207DE0B8F800203F4B02F00F0298
:10C60000520113441B7B0BB1E52B19D16B1CDBB220
:10C610005DB939490A4401990C320A60D8F80C20F6
:10C62000B8F80090D8F8106000925B450DD1009BDF
:10C63000A8F80090C8F81060C8F80C30002058E046
:10C640005D450CBF5D46002500E01D464046FFF7F6
:10C65000A7FE82460028C6D10FB9062049E0204631
:10C66000D8F80C10FFF732FF07460028F5D0012854
:10C67000BFD020465146FFF7FDFD0028B9D039460E
:10C680002046FFF713FD1C49834608604FF40072F3
:10C6900001F10C005146F8F715F894F82AA0BAF108
:10C6A000000F0FD094F82C0014495A46012305F0CE
:10C6B000B7F900289DD10AF1FF3A0BF1010B5FFA9F
:10C6C0008AFAECE70C4A0123137135B12046314652
:10C6D000FFF7D0FD00288CD0A9E7074BA8F8005041
:10C6E00053F80C2B0199C8F81020C8F80C70284694
:10C6F0000B6003B0BDE8F08FA40F0010B00F001066
:10C70000F8B51C4C0127002105462771FFF7B2FD43
:10C7100048B395F829300026032B26D195F8283008
:10C720002BB3204631464FF4007240F80C6BF7F7FC
:10C73000C9FF4AF65523A4F80A320F4B04F10C0145
:10C74000E3600E4BC4F8F0312B6AC4F8F431EB69A6
:10C75000C4F8F83195F82C006A6A3B4605F060F998
:10C7600085F8286001E00820F8BD3046F8BD18467D
:10C77000F8BD00BFA40F00105252614172724161B6
:10C780002DE9F04FD0F804900F46D9F8181085B075
:10C7900004469046039311B113782F2B0AD199F8D0
:10C7A0002930D9F81010032B04D00023A360E360D4
:10C7B000216105E0A160E1604846FFF777FC206158
:10C7C000002323800E9BC3F8049098F8000010B952
:10C7D000039B18604AE101260F9B0B22C3F80080DF
:10C7E00038462021F7F76EFF0822002318F8015B76
:10C7F0000DB12F2D04D1002B4CD00023FB724AE049
:10C800001F2D47D97F2D45D0202D41D02E2D0BD166
:10C8100023B3012B05D139782E291DD00B220823F3
:10C82000E4E7082B34D8F9E7222D33D0292D13D98A
:10C830002C2D2DD9392D0FD93F2D29D97C2D27D03D
:10C84000A5F15B01C9B2022922D9A5F16101C9B2E2
:10C8500019299CBF203DEDB2934219D2591CFD54B9
:10C86000CBB2C3E73A2D15D005F0F703222B11D038
:10C8700005F0BF033C2B0DD03E3DEDB2012D09D993
:10C8800018F8015B002D00F0E7802F2D00F0E48008
:10C890005C2DE7D10125109B4FF0000AA3F800A002
:10C8A000012D00F0D3804FF0000C4FF0010B4846F3
:10C8B0002169CDF808C0FFF7DDFCDDF808C00028CD
:10C8C00000F0C68066B1E3680E99CB6023690B6106
:10C8D00023880B80BAF1000F02D1109BA3F800A0AF
:10C8E0002388644E03F00F0362495B011E440B442E
:10C8F0001B7B0C3623B9002D40F0AC800220B5E044
:10C90000E52B7AD0F27A02F00F010F294BD1BAF160
:10C91000000F43D003F01F03013B4FF00D0E0EFB41
:10C9200003FE00235FFA8EFED9B201EB0E00C0B207
:10C93000BBF1000F2DD0504A13F802B016F80B20AF
:10C94000B3449BF801B012B9BBF1000F1FD00F998F
:10C950000133096811F800B0ABF16101C9B21929BE
:10C96000A2F1610198BFABF1200BC9B298BF5FFA89
:10C970008BFB19299CBF203AD2B2B2EB0B02D2F149
:10C98000000B5BEB020B0D2BCED1194601E04FF0F3
:10C99000010B8C441FFA8CFC00262FE0109A1388A0
:10C9A0000D331380F8E7BAF1000F11D0BBF1000F7F
:10C9B0001BD010990B8863451AD133683B607368AC
:10C9C0007B6033893B81B37ABB72337BFB7227E098
:10C9D000100712D4304639460B22CDF808C0F7F7BD
:10C9E000EBFDDDF808C040B91AE00126DC4602E0A4
:10C9F00001264FF0000CB34600E001262046CDF89A
:10CA000008C0FFF7CDFCDDF808C000287FF44FAF69
:10CA1000BAF1000F7FF46FAF109BA3F800A06AE794
:10CA20001DB9039B28461E6020E0F37AD90611D574
:10CA3000738BB18A484643EA0141A160E160FFF788
:10CA400035FB0223206123800026C5E604200DE08B
:10CA500008200BE0032009E00F99109A0B684FF0B3
:10CA6000010AC3EB0803013B138019E705B0BDE8D9
:10CA7000F08F00BFA40F0010C92401002DE9F04180
:10CA800005460C460846164600213022F7F71AFEE6
:10CA9000280984F82C0004F08FFEC70700F19A8063
:10CAA00016B1410700F1998015F00F0513D05F4FC3
:10CAB00094F82C0007F10C010022012304F044FF3C
:10CAC00020BB042D0DDC07EB051595F8BE3105F5EF
:10CAD000DD75DBB1AD6820462946FFF7CDFB78B1A7
:10CAE00017E0043DDFF85881EDB20646504B1A7945
:10CAF000052A75D00F2A73D010334345F7D18AE049
:10CB00004A4BB3F81720B2F5007F05D00B20BDE8E3
:10CB1000F081FF28FAD17EE05A8C02B91A6B62606C
:10CB2000197F84F82B104A43598B2944E160B3F8EC
:10CB30001D7093F819C02780B3F81F0084F82AC02D
:10CB400008B93A48C06A5E8B3F09861BB61AF61BC5
:10CB5000B6FBFCF6023640F6F6708642A66006D9B1
:10CB600000F5704086428CBF0326022600E00126B5
:10CB7000032E18BF501884F82960394408BF986BF9
:10CB80000A446261032E4FF0FF32206122621CD101
:10CB9000998F204629446162244FFFF76BFBA0B1B7
:10CBA000B7F80A224AF655239A420ED1FB68214A69
:10CBB00093420AD1D7F8F0311F4A934205D1D7F8F2
:10CBC000F831E361D7F8F431236284F8296000205A
:10CBD000BDE8F0810120BDE8F0810920BDE8F081C9
:10CBE0009F6894F82C00374414493A460123002EDC
:10CBF00008BF3E4604F0A8FE002887D1013D15F08D
:10CC0000FF057FF473AF0E49A1F140031A792AB9E9
:10CC100010338B42FAD10C20BDE8F081052AF7D001
:10CC20000F2AF5D09D683D4455E700BFA40F0010C2
:10CC30006E1100105252614172724161B00F0010CA
:10CC4000AE1100102DE9F04F87B002934368DDF874
:10CC500040B0039300238BF80B30C368164604934F
:10CC60000369B0F800800593029B04460D465846C0
:10CC700020210B225FFA83F9F7F724FD33782E2B5E
:10CC800025D04F4609F1FF3919F0FF0903D016F8F6
:10CC900009302E2BF5D1012F17D94FF0080A029B2E
:10CCA0009F4214D2BAF10A0F11D8F05D202809D0A2
:10CCB0000AF10103DBB20093FFF755FA0BF80A0003
:10CCC000009B9A460137FFB2E9E74FF006094FF0A3
:10CCD000000A57465FFA8AF34B4513D216F80A004A
:10CCE00020280AD02E2808D07B1CDBB20093FFF747
:10CCF0003AFA0BF80700009B1F46052F0AF1010ABC
:10CD0000E8D916E0022F3B4613D841220BF8072042
:10CD10007A1CD2B242210BF80210BA1CD2B24321C3
:10CD200003330BF802100437DBB24422FFB20BF8D6
:10CD300003207E230BF8073001373123FFB20BF8B5
:10CD400007309BF80030DFF8DC91E52B04BF0523AA
:10CD50008BF800304FF0000AA168676829B1E160E4
:10CD60003846FFF7A3F9206101E03B692361A4F88D
:10CD700000A038462169FFF77DFAF0B1238803F05F
:10CD80000F035B0109EB03004B441B7B0C30002BB2
:10CD900039D0E52B0BD0C37A03F00F020F2A06D04F
:10CDA0001B0704D459460B22F7F706FC28B120468E
:10CDB000FFF7F6FA0028DCD125E00823013BDBB2BF
:10CDC0001BF80320202AF9D0002030271BF803206D
:10CDD0000BEB0301392A08D10BF80370013B13F068
:10CDE000FF0300F09A800120F0E748B17E2A07D1C6
:10CDF00031200870002B00F0908001F8012CABE787
:10CE000001320A70A8E79BF8007000230BEB0302C5
:10CE100017F0010F52784FEA570714BF47F0800709
:10CE2000FFB2013317440A2BFFB2EFD1029BDFF8A8
:10CE3000F89003F10C0A0D239AFBF3FA049BA4F873
:10CE40000080E360059B5FFA8AFB23614FF00008D6
:10CE500003982169FFF70EFA00285AD02388314938
:10CE600003F00F0301EB43130C335FFA88FC2B60D4
:10CE7000CCEB0B0313F0FF034DD001220A7128689D
:10CE8000002120228DE80810F7F71CFC009B0D20E4
:10CE90005843DDF804C05B450CBF402100212A68DF
:10CEA000CCEB0A0C41EA0C0C0D3882F800C0C0B281
:10CEB0000023DAB21118DDF808E0C9B271450AD2D0
:10CEC00016F801E02A6813F8091001330D2B02F857
:10CED00001E0EED11A46531CDBB2FF210C2B2A686D
:10CEE0000CD819F803E009EB030002F80E100078E3
:10CEF0002A6801330244DBB25170EFE70F23D3728B
:10CF00002B6820465F73FFF74BFA08F101080028F1
:10CF10009ED1082002E0184600E0072007B0BDE8D7
:10CF2000F08F00BFA40F0010C924010011B100232D
:10CF300081F829300022FFF7A1BD0000F0B51E46A0
:10CF400097B0002305900C4604924B6004A805A9F5
:10CF500006F01E020793FFF7E6F8002840F0A980CC
:10CF6000059B09AF0D9311AB009308AB01930DF135
:10CF70001A0302930CA83946049A07ABFFF700FC8A
:10CF800016F01C0F06F01F0562D068B3022840F0AF
:10CF900090800CA807A9BDF81A20FFF707FB00280E
:10CFA00040F08780BDF81A30A3B9002120220798ED
:10CFB000F7F788FB079A3B4603CB1060516019884E
:10CFC0009B78118193729DF82F20079B45F00805EF
:10CFD0001A7330E000970CA807A9089AFFF732FEF1
:10CFE0000028E2D0082064E0700757D4079A002A8E
:10CFF0005CD0D37AD90653D413F0010352D137074A
:10D0000019D5518B968A53839382D36141EA0646A0
:10D01000294B0122059831461A711F68FFF7A1FAC2
:10D020000028DFD005983946FFF724F90028D9D029
:10D03000059B013EDE612E0715D5079B0022DA72A3
:10D0400004F0B2FA079B45F02005C3F80E000AE091
:10D0500000282ED1079B3BB3DB7AD80624D4B10736
:10D0600001D5DA0722D4144B05981B682570E361BB
:10D07000079B00262362998A5A8B15F01C0542EA09
:10D0800001422261DB69A660E3604FF00103637037
:10D0900060600DD0FFF734FB30460AE0072008E05F
:10D0A0000E2006E00F2004E0022002E0062000E04F
:10D0B000284617B0F0BD00BFA40F001010B5012422
:10D0C0000C700A6190F82A20034652020020CA60C0
:10D0D00088604C704B6010BD2DE9F84F466899464A
:10D0E00000230446A9F80030304688461546FFF76D
:10D0F00066F8002840F0848023781A067CD4DF0785
:10D100007DD5E268A368DFF8FCA0D31A9D4288BFF2
:10D110009DB2002D69D0A368C3F30802002A40D154
:10D120006278013AD2B262701AB1A36903F1010BBD
:10D1300014E00BB9216904E061693046FFF7D0F8CB
:10D140000146012954D9B368994251D261613046F0
:10D15000FEF7ACFF96F82A308346637060680021C2
:10D16000FFF73CF8002843D06F0AC4F818B018D075
:10D17000637896F82C009F4228BF1F46BFB24146F5
:10D180005A46FBB204F0E0FB002831D1637801334A
:10D19000DB1B6370A369013B3B447F02A361BFB209
:10D1A00017E06068A169A768FFF718F800B3C7F334
:10D1B0000807A368C7F50077BFB2C3F30803BD42F1
:10D1C00038BF2F460AEB030140460C313A46F7F7C9
:10D1D00027FAA368ED1B3B44A360B9F80030B844BC
:10D1E0003B44A9F80030ADB293E72846BDE8F88F7C
:10D1F000237863F07F0323700820BDE8F88F0620B2
:10D20000BDE8F88FA40F00102DE9F74F4668984647
:10D2100000230446A8F8003030460F461546FEF7B6
:10D22000CEFF002840F09B8023781A0600F19480FE
:10D23000990740F19380E368DD4280F09080DFF849
:10D2400024914FF0010ADDB1A368C3F30802002A5C
:10D250004FD16278013AD2B2627012B1A269013242
:10D2600021E03BB9216989B93046FFF72FF9014622
:10D27000206104E061693046FFF728F9014629B9C9
:10D28000A368E26893425DD9E3605BE001295FD067
:10D29000B36899425CD261613046FEF707FF96F8A9
:10D2A0002A3002466370606800210192FEF796FF03
:10D2B000019A00284CD05FEA552BA26119D06378FF
:10D2C00096F82C009B4528BF9B4639465B4604F0E8
:10D2D000A7FB00283CD163780133CBEB03036370D9
:10D2E000A369013B5B444FEA4B2BA3611FFA8BFB05
:10D2F0001BE06068A169D4F808B0FEF76FFF38B38F
:10D30000A368CBF3080BCBF5007BC3F308031FFA2C
:10D310008BFB09EB03005D4538BFAB460C3039464B
:10D320005A46F7F77DF989F804A0A368CBEB050509
:10D330005B44A360B8F800305F445B44A8F8003059
:10D34000ADB280E72378002043F02003237006E08D
:10D35000237863F07F032370082000E0062003B0E9
:10D36000BDE8F08FA40F001070B546680446304643
:10D37000FEF725FF014648BB237803F0200303F0A6
:10D38000FF001BB36068FEF729FF08B9082070BDD5
:10D390003046E169FEF76EFF0028F7D0256AEB7A88
:10D3A00043F02003EB72E368EB6123696B83638ACC
:10D3B000AB8204F0F9F8C5F816002378304623F064
:10D3C00020032370BDE87040FFF79AB970BD10B517
:10D3D0000446FFF7C9FF00B9606010BDF8B54668A4
:10D3E000044630460F46FEF7EAFE0146002878D193
:10D3F00094F90030002B75DBA368BB426AD06068EB
:10D40000FEF7ECFE002867D0E568AF4201D83D4644
:10D4100002E023789A07FAD4002D4FD096F82A70AC
:10D42000A3687F025A1EB2FBF7F2B5FBF7F19142F7
:10D4300003D1A56007FB115532E0012161703BB1BA
:10D440009D4205D907FB02F36169A360ED1A02E072
:10D4500000232169A36039B93046FFF737F8012866
:10D46000014639D02061D8B1BD42616115D9237818
:10D4700030469B0702D5FFF729F801E0FEF730FFA1
:10D48000014648B1012827D9B368984224D2A3683D
:10D49000ED1B3B44A360E7E73D46A3682B44A36034
:10D4A00030466169FEF702FE013D6D0A6BB2184419
:10D4B000A06196F82A305D1B657002E00123A5602B
:10D4C0006370A368E268934204D9E360237843F071
:10D4D000200323700020F8BD237863F07F032370BE
:10D4E00000E0F8BD0820F8BD38B5144660600B4672
:10D4F00059B990F829200169032A02D1A160E1609D
:10D5000005E0A360E360216104E0A160E160FEF753
:10D51000CDFD206100232380002038BD2DE9F84F88
:10D520000B6A06460D46D0F804800BB100221A7033
:10D530004046FEF744FE002864D1DFF8CC90DFF8C7
:10D54000CCA0287404460746316961B14046FEF715
:10D5500091FE002855D0318801F00F01490109EBF7
:10D5600001031B7B13B90020BDE8F88FE52B3FD0EA
:10D570002A6A49440C31AAB3C87A00F00F000F2878
:10D580002ED1A4BB03F01F03013B4FF00D0C0CFB8D
:10D5900003FC5FFA8CFCBCF1130F28D8234613F868
:10D5A0000AB0DAB211F80BE002EB0C00C0B2BEF127
:10D5B000000F05D18B449BF801B0BBF1000F0CD0DC
:10D5C000142807D02A6A01330D2B02F800E0E6D1B7
:10D5D0001A4602E0002701243A461744BFB207E08A
:10D5E0000023D3552846FEF76EFD002400E00124F9
:10D5F0003046FEF7D5FE00B930612B7C002BA3D05E
:10D60000B1E70820BDE8F88FA40F0010C92401007D
:10D6100030B597B0059016A840F8481D154605A9E5
:10D620000022FEF780FD0446B8B9059B0CA80D93B7
:10D6300011AB009308AB01930DF11A03029309A9F2
:10D64000049A07ABFFF79CF8044630B9079919B163
:10D650002846FEF738FD00E00424204617B030BD10
:10D660002DE9F347019002A840F8081D904668464E
:10D6700001A900221E46FEF756FD00284DD1019B50
:10D680009F681A6AB91E8A4202D8C8F8002044E08E
:10D6900093F82990B9F1010F0ED1022504460198A3
:10D6A0002946FEF71DFE80B200B90134019B013509
:10D6B0009B689D42F3D31FE0D968054604460EB12E
:10D6C000B44224D23DB9019801F1010AFEF7D2FD1E
:10D6D00010B313485146B9F1020F05D1038803B9BD
:10D6E00001340230013504E0036803B90134043029
:10D6F0000235013FEDB2E2D1B44209D2019BB9F14A
:10D70000030F1C6204D1012283F8282000E0344674
:10D71000C8F80040002000E0082002B0BDE8F08713
:10D72000B00F00102DE9F04196B0059016A840F812
:10D73000481D012205A9FEF7F6FC002840F0848070
:10D74000059B11AE0D9308AB01930DF11A030293E3
:10D7500000960CA809A9049A07ABFFF711F8002856
:10D7600072D1079B002B6CD0DA7AD4076BD49C8AD9
:10D770005B8BD00643EA04440AD4BDF81A300D226C
:10D78000193393FBF2F3ADF81A30314DE5274CE035
:10D79000059883699C4201D1102055E021460F94E1
:10D7A000FEF784FC2A4D02231090ADF83030059826
:10D7B0001099FEF75FFD08B9082045E0BDF830304C
:10D7C00003F00F035B01EA182B441B7B0C32002B88
:10D7D000D3D0E52B02D0D37A1907DDD50CA8FEF7FC
:10D7E000DFFD0028E3D1C8E7BDF81A3005985A1EBE
:10D7F000ADF81A20E3B11599FEF73CFD0028DBD007
:10D80000BDF8443085F8048003F00F035B01EA188B
:10D810002B441F73BDF81A300C320792002BE3D053
:10D820003046FEF7BDFD0028C6D04FF00108DBE70B
:10D830002146FEF796FE0028BED00598FEF760FF51
:10D8400002E0042000E0062016B0BDE8F08100BF31
:10D85000A40F00102DE9F04F97B0059016A840F8DE
:10D86000481D012205A9FEF75EFC002840F0BE809D
:10D87000059B0DF124080D9311AB009308AB0193A8
:10D880000DF11A0302930CA84146049A07ABFEF768
:10D8900077FF002800F0A780022840F0A7800CA89E
:10D8A00007A9BDF81A20FEF781FE0546002840F0C2
:10D8B0009D80504E05982946D6F800A0FEF706FE3A
:10D8C0000128074601D1082090E0DDF81490394680
:10D8D0004846FEF7EBFB0446002800F086804846E9
:10D8E0002146FEF7C7FC0028EDD0294606F10C00C2
:10D8F0004FF40072F6F7E6FEC4F10105059B2A1904
:10D9000093F82A10D2B291420AD9013493F82C002C
:10D9100039492246012304F083F80028EED0D2E7EB
:10D9200020210B223448F6F7CDFE4FF02E0B1023AA
:10D93000F37586F80CB003F037FE304CC6F82200C1
:10D94000A4F1200581460FCD0FC495E80F0084E8AF
:10D950000F00059886F82DB090F82920BCB2032A54
:10D960004FEA1747F48437840E9B03D10269934230
:10D9700008BF00231F4D5146A5F846301B0CA5F8E3
:10D98000403001232B71FEF775FC00289BD0BDF8B9
:10D990001A30EBB9079800212022F6F793FE079A78
:10D9A000434603CB1060516019889B7811819372B4
:10D9B0009DF82F20079B05981A7301222A711022C7
:10D9C000DA72C3F816905C839F82FEF799FE0DE031
:10D9D000CDF800800CA807A9089AFFF733F90028B2
:10D9E0007FF471AFD6E7072000E0062017B0BDE84E
:10D9F000F08F00BFA40F0010B00F0010D00F001068
:10DA00002DE9F0439FB005901EA840F8681D91468F
:10DA100005A90122FEF787FB002840F0B180059B95
:10DA20000BAD13AE0AAF07AC0F93009601970294AB
:10DA30000EA82946049A08ABFEF7A2FE002840F083
:10DA40009F80089A002A00F098800DF1600E02F184
:10DA50000B0302F11B0CF04618685968724603C2AA
:10DA6000083363459646F7D11868294610601B793C
:10DA70000EA813710DF11E0302938DE8C0004A46F3
:10DA800009ABFEF77DFE002879D0022878D10EA8D8
:10DA900009A9BDF81E20FEF789FD002870D1BDF848
:10DAA0001E30002B3ED1DDF824E042460EF10B0380
:10DAB00008F110089446BCE80300C445186059609A
:10DAC000624603F10803F5D11068DFF8BC901860D6
:10DAD00012794FF001081A712B4603CBCEF80000E3
:10DAE000CEF804101A889B78AEF808208EF80A3019
:10DAF0009DF83720099B89F804801A7329460294FF
:10DB0000049A08AB8DE8C0000EA8FEF739FEBDF8F8
:10DB10001C300D22193393FBF2F3ADF81C304C4648
:10DB2000E5251FE000950EA809A90A9AFFF78AF8D3
:10DB30000028B8D0082023E01799FEF79BFB0028A7
:10DB4000F8D0BDF84C30304603F00F035B01E2180B
:10DB500023440C321D73089284F80480FEF720FCE5
:10DB60000028E7D0BDF81C3005985A1EADF81C20DF
:10DB7000002BE1D1FEF7C4FD02E0022000E0072007
:10DB80001FB0BDE8F08300BFA40F00108279C2F17E
:10DB900063038371436A03B9036A9A711A7B002095
:10DBA00060F3410258711A73704710B5046A204639
:10DBB0001CB1F6F7FBFF646AF9E710BD70B50021F0
:10DBC00004468CB000682022F6F77CFD94F84430BF
:10DBD00018064FD4204610F81C3F4D4A702101FB17
:10DBE00003239B6B69461B6B9847411C05D0B8B15A
:10DBF0002046F6F7DBFF012087E094F84430002050
:10DC00005A1CD2B284F844203BB1082A60717BD1FF
:10DC1000237B43F02003237377E00222627173E0D9
:10DC20003C4D2B78002B3AD09DF81B30012B36D180
:10DC300008A8FDF76DFE90B32B78012B06D19DF857
:10DC4000113023F00F0343F0060326E094F844302C
:10DC5000226863F07F0384F844306D46D0320CAE06
:10DC60002B4603CBB342106051601D4602F10802FF
:10DC7000F6D114E0226803F07F0384F844306D4647
:10DC800002F1D00302F58076186859682A4603C26B
:10DC90000833B3421546F7D106238DF811302368B7
:10DCA0000122DA702268BDF81230A0219377226831
:10DCB0001B0AD3779DF81130226883F07F03DB4382
:10DCC0009370206810220530F6F7FCFC6846F6F7E2
:10DCD0001BFE0246206869460530F6F7A1FC94F861
:10DCE0004420531C520614BF00220222DBB2627190
:10DCF0001F22227103F07F02082A84F8443004BFF7
:10DD000023F07F0384F8443000200CB070BD00BFC6
:10DD1000C4190010B8190010F8B5022A04461646B6
:10DD20000B6804D0012A14BF1F25292500E03F25D8
:10DD30000D712A4618462021F6F7C4FC00224255F0
:10DD4000217D451CFF294FF001021ABF02310170ED
:10DD500002702A70638A6B70638A1B0AAB70638AD5
:10DD6000632B01D9043503E0092B8CBF053506353B
:10DD700022236A1C2B701146234604F1100053F82D
:10DD8000047B834241F8047BF9D100232220202721
:10DD9000E15C222902D009B1102B0BD1D054D15C07
:10DDA00009B9D75402E001F07F01D1540133DBB24D
:10DDB000112BF4D10133DBB2102BE9D994F91130D6
:10DDC0000321002BBCBF2A23AB74627C3E4B16F0B0
:10DDD000010F02F00F0201FB023105F113000CBF2D
:10DDE00003220122F6F71CFC637C5B0644BF3C2344
:10DDF000AB75B70736D505F11900A17D03F062FFB9
:10DE00002F250570E17D013003F05CFF00F8015B18
:10DE1000627D6423B2FBF3F103FB1121C9B203F06D
:10DE200051FF217E03300C2984BF0C39C9B203F0A5
:10DE300049FF2E2300F8013B617E03F043FF237E60
:10DE400003300B2B94BF4123502300F8023C4D2399
:10DE500000F8013C012210F8013B13B100F8012C3D
:10DE6000F9E7F8BD012E28D1A17D05F1150003F0D9
:10DE700029FF2F2300F8013BE17D03F023FF217EE2
:10DE800001300C2984BF0C39C9B203F01BFF2E23CB
:10DE900000F8013B617E03F015FF237E02300B2B5F
:10DEA00094BF4123502300F8013C012210F8013BAC
:10DEB00013B100F8012CF9E7F8BD637C9C0644BF60
:10DEC0004823EB75F8BD00BF3C250100F0B50023E9
:10DED000224F234D8DB004464371207F3B7883420F
:10DEE0002FD9702606FB00539B6B69461B69984728
:10DEF00020B12046F6F75AFE01202CE0227F194976
:10DF000006FB0256531CB26B206A8A4209BF96F880
:10DF10006020082202F07F020732ADF812308DF83F
:10DF20001120237730B9684621460022FFF7F4FE1E
:10DF3000002010E06946002203F0F6F80028CCD05B
:10DF4000F1E701232371237B002043F02003237397
:10DF50002368187058700DB0F0BD00BFC1190010D3
:10DF6000C4190010BC1E0100F0B504468FB02B2070
:10DF700002F0B4FC94F844200023637102AD8AB12E
:10DF8000226884F844302E4602F1D00302F58077EF
:10DF900018685968324603C20833BB421646F7D1A7
:10DFA000062323E094F8343004F138018DE828008A
:10DFB00004F11C000EC903F00DF9421C30D00028FA
:10DFC0004ED12A4F3B781BB39DF82360012E1FD101
:10DFD00005F12000FDF79CFCD0B13B78012B08D166
:10DFE0009DF8193023F00F0343F006038DF8193024
:10DFF0000EE0226884F84460D0322E460EAF3346DD
:10E0000003CBBB42106051601E4602F10802F6D1FC
:10E010002846214694F83520FFF77EFE002023E0B5
:10E02000134B226803F1200153F8040B8B4242F892
:10E03000040BF9D1207F0F4B702202FB00339B6B46
:10E04000DB699847236898702368000AD8701F23FB
:10E050002371237B002043F020036071237303E0CE
:10E060002046F6F7A3FD01200FB0F0BDB81900104F
:10E070001C250100C419001030B5124D91B004AC3C
:10E080000FCD0FC40FCD0FC495E80F0084E80F002B
:10E090000D4B01AC93E8070084E80700F6F712FD8A
:10E0A000024660B10023837108499DF80430702056
:10E0B00000FB03139B6B20461B6804A9984711B013
:10E0C00030BD00BF88190010B0110010C419001035
:10E0D0002DE9F04FA1B00646F6F7C8FD08B1F6F7F6
:10E0E00081FD9F4F0020FBF79DF83B78DFF874928D
:10E0F000012B0DD909EB030212F8011C0D2901D1E6
:10E10000013B04E012F8022C0D2A01D1023B3B70C6
:10E110003D78944C0021C5F1FC0209EB0500F6F7AF
:10E12000D1FA204600212A4602F05CFC99F8003022
:10E13000DFF82C82232B42D198F80030032B28D112
:10E140006378232B25D1A078303810F0FF0000F041
:10E150009783F6F7C9FC002800F09283824B834C2A
:10E160001A78834DC6F16301FF27037B817143F069
:10E170004C030373436A44618561077102770BB1F5
:10E180001846F2E7037B43F020030373036A9E7192
:10E1900076E3F6F797FC002800F0728301234371C1
:10E1A0004377714B027B1B78FF2103776F4B86719E
:10E1B000436142F06C0301710062037360E30EB1CE
:10E1C000002409E098F80020012AF9D12A2BF7D180
:10E1D000684B1B7833B9022400256248AB462B46B6
:10E1E000A84604E0FFF748FF4AE30125534603F140
:10E1F000010A012B5FFA8AFA07D999F80030DFF893
:10E200006481242B40F02D825BE00378002BF4D056
:10E210002C21F6F7A1FA03460028EED0184600F8A4
:10E22000018B5B78413B162BE0D801A151F823F01C
:10E230008DE20000EDE10000EDE1000095E200005C
:10E24000EDE10000EDE10000EDE10000EDE1000096
:10E25000EDE10000EDE10000EDE10000A5E20000CD
:10E2600091E20000EDE10000EDE100009DE2000020
:10E27000EDE10000B5E2000099E20000EDE10000F0
:10E28000A1E20000EDE10000EBE100000225ADE7B6
:10E290000325ABE70024A9E70124A7E70224A5E7AB
:10E2A0000324A3E72C21F6F757FA28B190F801B020
:10E2B000013001E0002599E7042401254FF0020A0E
:10E2C00094E7F6F7FFFB0446002800F0D982037BB1
:10E2D000867143F0040303731F2303713B78022B01
:10E2E00054D9002E52D198F801203D2A4ED198F8E9
:10E2F0000220502A2CD1204B026803F1200153F850
:10E30000040B8B4242F8040BF9D122681B4B2032DC
:10E3100003F1200153F8040B8B4242F8040BF9D1AE
:10E32000174A3F232371127823681A71154B6361D2
:10E330003B78032B40F29081134814A908AA0023CC
:10E3400002F0BAFF002840F09B82089B236283E121
:10E35000542A4FF001001AD184F83500032016E04A
:10E36000F1170010FA170010C01900108DDB000023
:10E37000ABDB000088190010DC240100FC24010044
:10E38000C1190010CDDE0000FD170010012019F8A2
:10E390000010904A002900F0AF80022B40F28D80DF
:10E3A000104414A908AA002302F086FF002840F0B8
:10E3B00067829DF85030884A702101FB03239B6BD4
:10E3C00004F11C00DB6A14A998470546002840F0B8
:10E3D000578208983D21A063F6F7BEF908900028FF
:10E3E00000F0A180421C08920570089B1A78423AFE
:10E3F000132A1AD8DFE802F0141214191919161981
:10E400001919191919190C19100A190E01220AE003
:10E41000022208E0032206E0042204E0052202E0D2
:10E42000062200E0202284F8342094F8342022B11F
:10E430009A1C08925B782C2B75D1684D684F4FF071
:10E440000208089B1A78002A6DD05A1C08921B7883
:10E450003E2B0BD002D83C2B14D064E04C2B1DD0AB
:10E460004E2B60D1002384F835301CE05B4808A9AE
:10E4700002F0F4FF002856D16B78A3B1AB7893B1CA
:10E48000E56310E0564808A902F0E8FF00284AD1E9
:10E490007B7843B1BB7833B1276404E094F835301E
:10E4A0000BB184F83580089B1A78002AC9D05A1C11
:10E4B00008921B782C2BC2D035E05378302B0FD02C
:10E4C000484A12681A445278550701D5313B09E091
:10E4D000212B03D1444B1B78FF2B03D1434BA36368
:10E4E000434B1B788DF85030424B9DF850201B78E1
:10E4F000934205D84A2010E13D4B1A788DF8502000
:10E50000354B702101FB023315AA03F1300103C919
:10E5100082E803009B6B04F11C00DB6A14A9984796
:10E52000002840F0AD81002E6AD020AD2A4E15F8AB
:10E53000303D702707FB03639A6B2F4B9A4204D13F
:10E5400028462146F8F7E6F89AE100214FF4807258
:10E550002068F6F7B7F82068A0218E301B22F6F766
:10E56000B1F89DF85030216807FB03639B6B284688
:10E570005B698E319847002840F082819DF85030C9
:10E58000216807FB0366B36B28469B69A031984757
:10E59000002840F075812368A0219E330893089BD2
:10E5A0005A1E089213F8012C202A02D103F8011CEC
:10E5B000F5E7236893F8A220202A04BFA02283F85D
:10E5C000A220236841221A700C4B6361FD23237142
:10E5D00042E000BFFA170010C4190010F61800102E
:10E5E000F417001000000010FC180010FB170010BA
:10E5F000C0190010C1190010BC1E0100BDDB0000D5
:10E60000A14B226803F1200153F8040B8B4242F81E
:10E61000040BF9D120AD15F8303D9C4E7027591CE4
:10E6200007FB03632268284611719B6B21685B69B5
:10E6300008319847002840F023819DF85030216828
:10E6400007FB0366B36B28469B691A31984700287D
:10E6500040F016818E4B6361237B43F040032373AC
:10E660000EE105AF4046394604AA002302F024FE1D
:10E670008046002840F00481844B9DF814207021CE
:10E6800001FB0232916B834A9A4691420FD09DF86A
:10E690001430702202FB03A39B6B7F48DB6A394670
:10E6A0009847002840F0EC800DF120081DE0049808
:10E6B000F6F72AF90138C3B2DAB2002BE7D0049991
:10E6C00052B2885C013B2028DBB2E0D101F8028025
:10E6D000F2E79DF8313013F0070313D1012D13D069
:10E6E000012E11D0BCF1000F11D120228DE80401C0
:10E6F000002269480499134602F06CFDB0F1000C49
:10E70000E7DDBDE0062BE9D0BCF1000F08D0042CFA
:10E710000FD1BBF1000F0CD11F20FAF783FDAFE042
:10E72000042B06D114F0FB0F01D04020F5E71C4666
:10E7300003252EB1012E08D1002C08BF022409E0C8
:10E74000002C08BF0224354649E0002C08BF0124F4
:10E75000012D44D1BCF1000F32D199F80030402B8B
:10E760002CD14E4B1B7803F00F030F2B01D1462009
:10E77000D3E714ADC646BEE80F000FC5BEE80F00D4
:10E780000FC59EE80F0085E80F009DF81430702239
:10E7900002FB03A39B6B3846DB6814A9CDF80CC0C1
:10E7A0009847FF28DDF80CC06AD09DF83B30013B4C
:10E7B000DBB2012B11D88DF840C00EE03F20ACE752
:10E7C000002130224046F5F77DFF40460499102293
:10E7D000F6F7CAF80020FAF725FD012504E0BCF1A0
:10E7E000000F01D03E2098E7F6F76CF98446002828
:10E7F00046D0042C867110D19DF81430702202FB93
:10E8000003A3E81E45429B6B454100959C68384632
:10E81000414662465B46A04732E0214B214EC1464D
:10E8200097E8070083E80700B9E80F000FC6B9E8CA
:10E830000F000FC699E80F0086E80F00032D1FD8C0
:10E84000DFE805F0020E0E029DF81430702202FB84
:10E8500003A39B6B38461B684146624698470FE00E
:10E860009DF81430702202FB03A3A91E4D429B6B3E
:10E870004D4100955D683846414622466346A847AB
:10E8800021B0BDE8F08F00BFDC240100C4190010E6
:10E8900069DF0000F02701000C130010C5170010FD
:10E8A000B01100108819001038B5084D6B69084C7C
:10E8B000DB4302201C4000F0FFFD6A69044BD24399
:10E8C00013409C42F2D1204638BD00BF20C0092031
:10E8D00000000C0C084B094A5878012806D1126830
:10E8E00012B906225A70704700207047106810B1A4
:10E8F00002225A7001207047B9190010C806382347
:10E900002DE9F74F72B6FFF7E5FF10B14FF6FF7034
:10E9100097E0FFF7C9FF4001F5D54C4B01221A6083
:10E920004B4A1368002BFCD14FF4807000F0EEFDD1
:10E93000FFF7D0FF0028E9D100F0F6FD0446FFF70D
:10E94000B3FF410102D5002CF2D000E0BCB13F4C36
:10E9500000232360492000F0AFFD01232360452000
:10E9600001F0BCFFFFF7B6FF0028CFD1FFF79CFFF7
:10E970004201F7D4374B1A7842F001021A70354E33
:10E980000024354F2546B3467378012B32D1072D2D
:10E9900030D1DA2000F0BAFD4FEA540909F01F0A1D
:10E9A0007B696FEA03089BF8003003F0040303F06F
:10E9B000FF02C3B9019200F0B7FD019A98B1B9F115
:10E9C0005F0F10D825490B7853450CD11F4B65209C
:10E9D0001A60019300F070FD019B01221A603378E8
:10E9E00043F00403337018F0806FD9D01C4B08EA51
:10E9F000030305E07A69D2435301FBD5184B13405A
:10EA000013F0006F0CBF4FF000084FF08008FFF7C5
:10EA100061FF00287FF47AAFFFF746FF10F08069AE
:10EA2000F5D10135EDB2082D48EA5404ACD10520EA
:10EA300000F042FD054B3220C3F8009000F03CFD91
:10EA4000204662B600B203B0BDE8F08F84070842EA
:10EA5000EC063823B919001020C00920BD19001098
:10EA600000000C0C2DE9F84306460C46FFF732FF78
:10EA70000246002840F09180494B1978984611F0E1
:10EA8000040F09D03046214600F0AEFF002800F008
:10EA90008580FFF71FFF80E0FFF706FF3C2000F0B6
:10EAA0000BFD404B01221A60FFF714FF002874D1C0
:10EAB000FFF7FAFE0501F7D554B93A4B00221A6068
:10EAC000282000F0F9FC11E0FFF7EEFE040108D465
:10EAD000FFF700FF0028F7D05FE0FFF7E5FE000139
:10EAE000EBD5FFF7F7FE0028F7D056E0FFF7F2FE70
:10EAF0000446002851D1FFF7D7FE0101F6D51520B5
:10EB000000F0DAFC274F284DB946FFF7CDFE020191
:10EB100003D4072388F801303FE02D2000F0CCFC1F
:10EB2000012303FA04F2324008BF2A604FF01600B6
:10EB300018BF2B6000F0C0FC01233B601B4B01346D
:10EB40001B78DB074CBF22204B2000F0B5FC0023D4
:10EB5000C9F80030162000F0AFFC01232B600E2016
:10EB600000F0AAFC082CD0D1FFF7B4FEA8B9FFF73B
:10EB70009BFE0401F8D4FA2000F0C8FC0C4C0D4DAB
:10EB8000236813B90020BDE8F8832B68002BF9D166
:10EB900000F0CAFC0028F3D0F4E7FF20BDE8F883BA
:10EBA000B91900108007084284070842F3170010C3
:10EBB000EC063823C806382308B5134B1B6813B17D
:10EBC000124B00221A60012000F08AFC104B114AFF
:10EBD0001B681268002B14BF08230923002A0CBFEE
:10EBE000022200221A440C4B1B68002B0CBF04238A
:10EBF00000231A44094B1B68002B0CBF0823002379
:10EC00001A44074B1A7008BDC80638238407084207
:10EC1000F4123823F0123823E80E3823E40E382398
:10EC2000BD1900102DE99F48A34C49200026A34F91
:10EC3000FAF7F8FA66706378082BFDD8DFE813F06E
:10EC4000290080005200DF00E500F0001701BA0241
:10EC500009009B4B01259A6A002022F007029A6264
:10EC6000984B3D601D60FAF7DDFA974B1D60A3F5E8
:10EC7000E9631D60954D2A78944B110702D401F089
:10EC800083FDF8E71A7802F0F7021A7000F0DCFA58
:10EC9000CBE2002001F0E6F9894BDFF838829A6A6E
:10ECA0008A4D42F007029A62D8F800309BB92A7860
:10ECB000864B520702D0F7F7EBFE09E02A781007DF
:10ECC00006D51A7802F0F7021A700823637002E082
:10ECD00001F05AFDE8E76378082BACD0764B0222AE
:10ECE0005A70A8E7774A01231360754900223A60F9
:10ECF000886A774D20F00700886263702378FA20D5
:10ED000023F00D03A270237000F000FCDFF8C48133
:10ED10002B681BB16E4A6F4906200DE000F004FC21
:10ED20000028F7D1D8F80030002BF1D1062363700A
:10ED3000EEE70B6803B960701368002BF9D17AE72E
:10ED4000FFF7DEFD061E01DA4320D1E1412001F08C
:10ED5000C5FDF0B201F012FE01F03BFE3F2E02D1E4
:10ED6000A378012B03E05F2E06D1A378022B55D1A7
:10ED7000514B00229A7051E0574B1B7803F140022F
:10ED8000964201D1022303E020339E4202D10123A7
:10ED9000A3702EE006F06003602B2ED1612E08D107
:10EDA000A178454A022904D111781E4641F0080194
:10EDB000117006F0F00306F00F00E02B3E4DE070FE
:10EDC00019D133B2EF2B04D10520F5F715FF80B12F
:10EDD00009E0F5F74BFF804658B18369984728B1A1
:10EDE0004046F5F7E3FE07236B7024E74046F5F74E
:10EDF000DDFE03231AE20523F6E7042316E2354B72
:10EE00001B68002B31D0012310E22D4B9A6A22F0AF
:10EE100007029A622B4A012313603B60052305E237
:10EE200023782E4D23F010032370DFF8A8900023E1
:10EE30002B70AA46A278D9F80030B3B1002AFAD0D4
:10EE40002B78002BF7D023784FF0000843F0100305
:10EE500023708AF8008001F00FF9A378022B0CBF11
:10EE60000120404601F0FEF8E4E70623DEE1144B02
:10EE70009A6A42F007029A62A378012B40F09A80C6
:10EE80005FFA86F84C2008F00F0A01F027FD504683
:10EE9000F5F7ECFE054638B1037B190704D5DFF81A
:10EEA000189008F0F00B49E008F0F003F02BF6D0D2
:10EEB000632001F013FD6DE1B919001084070842C9
:10EEC0000080004080070842340B38238C1B001060
:10EED000E8063823C8063823BD190010741900103D
:10EEE000AD4B03A89A6A42F007029A6200F040FD17
:10EEF000039B8046580329D513F0806F99F80030A2
:10EF000014BF43F0010323F0010389F8003018F423
:10EF1000004F7FF490AEBAF10F0F1BD19F4A1378C8
:10EF2000F92B04D8591C11709D4A02F803802378EC
:10EF3000DA0703D543F0020389F8003023785A0733
:10EF4000CED4D90602D5FBF76FFD01E0FFF7D8FC60
:10EF50008046DCE7BBF1F00FE0D02B7B980709D5AA
:10EF60006B692846984700287FF465AE5046F5F750
:10EF70007DFE05466A792B68284603F80280F5F77E
:10EF80008BFE6B792A799A4238BF2B710133DBB241
:10EF90006B711BB92B7B43F002032B73EB79002BB6
:10EFA000CCD02378D907C9D56B6928469847002863
:10EFB000C4D040E6022B40F0ED8001233B603220BC
:10EFC00000F07AFA774B00221A60462000F074FABB
:10EFD00006F00F09542001F081FC4846F5F746FE83
:10EFE0000546002800F0D6806F4B1B785A0703D5E2
:10EFF0004FF4B47000F060FA23781B0713D5DFF8E4
:10F00000B081FFF767FC00287FF415AED8F8003018
:10F01000002BF6D104226A713B60624B01221A6018
:10F02000322000F049FADFF87C8130E0BBF1000FBC
:10F030006FD16B795A1C6A712A799A422CD8297B34
:10F040006B6911F0200F40F08E8028469847002809
:10F0500040F0A0804846F5F709FE237805461907D9
:10F0600015D5782000F052FADFF844A1DAF8003024
:10F07000002B40F08980FFF72DFC00287FF4DBADEA
:10F0800001233860C8F80030322000F015FA2B7BDD
:10F090005A077FD54FF0010A95F804B06B792078B4
:10F0A000BBEB030EDEF1000B5BEB0E0B10F0080F59
:10F0B0002A6820D100F01000BBF1000F43D0297B5B
:10F0C000890640D5002839D0D05C0121FBF7F6FC39
:10F0D00023788346580707D5322000F0EDF9002346
:10F0E000C7F800A0C8F80030BBF1000FA1D0512034
:10F0F00001F0F4FB9FE50021D05C8B4514BF80221A
:10F10000812200F071FC034600288FD0FFF7E2FB5C
:10F1100091E52A7B90068CD56420019300F0CCF910
:10F120006420C8F800A000F0C7F9019B6420C8F86B
:10F13000003000F0C1F9C8F800A07AE7D05C0121E6
:10F14000FFF790FCC4E700F0FF0120B1D05C002184
:10F15000FBF7B4FC02E0D05CFFF784FC00283FF42E
:10F1600068AF5620C4E7B9F10F0F3FF46EAFEA79EC
:10F17000002A7FF46AAF0D4883423FF466AF0B4626
:10F1800062F382032B7305E000F0CEF900283FF410
:10F190006DAF70E7072349E000800040F1170010D1
:10F1A000FA17001080070842B91900108DDB000023
:10F1B000EC0638231E4B01209A6A42F007029A623D
:10F1C0001C4B1860386023789B0729D51A4B1A7896
:10F1D000022A12D0194A10601A7812B11B788342A1
:10F1E00005D10620F5F708FDF7F74EFD0020FCF7E6
:10F1F00077FEF9F7F1FA00F027F8E0780F2802D14E
:10F20000F7F7C8FE05E00E4B4FF6FF721A80FEF7C7
:10F210005FFF0C4B00221A70237823F00203237047
:10F220000220F5F7E9FCF7F7DFF80023637002E549
:10F230000080004080070842F0170010B40B38230C
:10F2400004000010F1170010084B19781A4601232A
:10F2500009B1074900E007490B6013781B0914BF87
:10F26000054A064A01231360704700BFC517001006
:10F27000B40B3823340B3823EC0338236C033823C6
:10F2800007B5084B01221A600DF107025A60A02051
:10F290000549012201F03EF80028F8D103B05DF8DD
:10F2A00004FB00BFC01100100800001007B50A4B96
:10F2B00080B2020A1A705870084B0DF107025A60AA
:10F2C00007490122A0201A6001F024F89DF80700E8
:10F2D00003B05DF804FB00BFBC110010C0110010AA
:10F2E0000800001007B50A4B80B2020A1A70587065
:10F2F000084B0DF106025A6002221A6006490122EB
:10F30000A02001F007F8BDF8060003B05DF804FB8B
:10F31000BC110010C01100100800001010B589B217
:10F32000064B0C0A59701C70054B06491A60586050
:10F330000122A020BDE8104000F0ECBFBC1100107D
:10F34000C01100100800001007B580B202AB094AD6
:10F3500003F8011D010A11705070074A07495360F4
:10F36000A0200123136000F089FFFFF789FF03B09D
:10F370005DF804FBBC110010C01100100800001063
:10F380002DE9F843DFF84880DFF848900746144637
:10F390008DB2CCB105F01F0633191F2B8CBFC6F1FF
:10F3A000200626462B0A88F801500849A02035443B
:10F3B00088F8003089E8C000ADB200F05FFF374444
:10F3C000FFF75EFFA41BE4E7BDE8F8830800001028
:10F3D000BC110010C011001007B5024602A820F8A9
:10F3E000021D11460222FFF7CBFF03B05DF804FBBC
:10F3F000224A01232249F0B5136000224A602149C4
:10F40000F8240B602049214DC868214F20F07F402F
:10F41000013848601F48DFF89CC080F8234007206F
:10F420008A6008601C491D4C0B6041F8043C0B6568
:10F430001B491C480B604FF040268B60C1F8A83078
:10F4400009212B6023600360F960F160CCF80C1097
:10F450002421B962B1622A6022600260124A1360FC
:10F46000124A1360A2F50022136002F18C7213603D
:10F470000F4B04221A6002221A60F0BDC018F84334
:10F4800000000B40E835F84310E000E08400104233
:10F490000080004000ED00E08818F8438400084236
:10F4A0000835F8438400204388022043800010423E
:10F4B00000E100E000000940074B0022DA6064220E
:10F4C00050430649092218601A720A68002AFCD0C3
:10F4D00000221A72704700BF00000B400001604319
:10F4E000074B0022DA6009221A72064A0649504385
:10F4F00018600A68002AFCD000221A72704700BF08
:10F5000000000B40A086010000016043044B002274
:10F510009A600A2250439861024B01221A60704798
:10F520000000094080002043034B1868D0F101001F
:10F5300038BF0020704700BF80002043134B144A9F
:10F5400000280CBF10461846012202604FF04023ED
:10F5500010221A600F48104A13682BB90029FBD0FB
:10F560000368002BF8D000E031B10A4B1B681BB1D7
:10F570004FF040239A6802E04FF04023DA6A074BCD
:10F580001A6024224FF040239A6270470405084213
:10F5900000050842C806382310000842CC110010AC
:10F5A000134B144A00280CBF104618460122026073
:10F5B0004FF0402320221A600F48104A13682BB9DD
:10F5C0000029FBD00368002BF8D000E031B10A4BD2
:10F5D0001B681BB14FF040239A6802E04FF04023B4
:10F5E0001A6B074B1A6024224FF040239A6270472F
:10F5F000100508420C050842C806382314000842CA
:10F60000CC11001030B54FF040239D68104B1C68A2
:10F610000444A54202D90F4C012525601B681844FB
:10F620004FF0402398610120186029B1D96B21F077
:10F63000300141F0200104E0D96B21F0300141F0AC
:10F640001001D9631AB1044A1368002BFCD030BDF5
:10F65000CC110010580338230000084210B54FF0B9
:10F6600040239C680E4B1A680244944202D90D4A0A
:10F67000012414601B68022218444FF04023D86113
:10F680001A60DA6B22F0C00211B142F0800201E090
:10F6900042F04002DA63044A1368002BFCD010BD2C
:10F6A000CC11001058033823040008422DE9F04122
:10F6B000077E06464F40054600244FF00108297C8E
:10F6C000305908FA01F100223940FFF79BFF297DEC
:10F6D000305908FA01F104343940FFF7BFFF102C0C
:10F6E00005F10105EBD1BDE8F08100001248134A95
:10F6F0000123002110B50360136001601160104AFE
:10F700000421C2F880100221C2F880100D490E4A6F
:10F71000886A10604FF04022946A0C4804602420EC
:10F720008862906240F2492048615061084A136043
:10F73000A2F50022136010BD84001042840008422C
:10F7400000E100E000800040D0110010D411001052
:10F75000800010420F4B01221A600F4AD36B03F056
:10F760000F03D3634FF04023D96B01F00F01D9632E
:10F770000021516159610949096891620849096884
:10F7800099623F2111601960064B04221A6002221F
:10F790001A6070478802104200800040D0110010AB
:10F7A000D411001000E100E070B504460D46164685
:10F7B000FFF79CFF094A01230020136001465360B4
:10F7C000FFF7BCFE28462146FFF770FF3046FFF7E3
:10F7D00073FEBDE87040FFF7BDBF00BF8007084261
:10F7E0002DE9F041074688461646FFF77FFF00F0F7
:10F7F000DDFF154B0124154D1C600F205C60FFF7E9
:10F800005BFE2B68ABB920462146FFF797FE2D68BB
:10F810007DB940463946FFF749FF304621462A4622
:10F82000FFF7F0FE30462946FFF718FF2046FFF7A6
:10F8300043FE00F0BDFFFFF78DFF044B186800305A
:10F8400018BF0120BDE8F08180070842C8063823B0
:10F8500010B50A4B0A4A1968946801448C4202D3D5
:10F86000084901240C601B68184493688342FCD348
:10F87000054B06485B69DB43184010BDCC110010F6
:10F88000008000405803382320C0092000000C0CE1
:10F89000F8B500240746054626463859FFF7D8FF35
:10F8A0002B7CC0F3806202FA03F32A7DC0F3C060B0
:10F8B0009040043418430643102CF6B205F10105BC
:10F8C000EBD1387E7040F8BD38B505460C46FFF7E1
:10F8D0000DFF00200146FFF731FE2846FFF7D8FF55
:10F8E00005462046FFF7E8FDFFF734FF284638BD00
:10F8F0002DE9F8431C4E1D4D022400204FEA00194B
:10F900005FFA89F93368002BFCD00320FFF7D4FDA0
:10F910006A695FFA89F9D24312F0806F14BF4FF021
:10F9200000084FF0080812F0006F0CBF02270027F4
:10F930003368002BFCD10320FFF7BEFD6B69DB436E
:10F9400083F00060C0F3C06049EA000013F0806FEC
:10F9500040EA080014BF002204223843013C40EA78
:10F960000200CBD1BDE8F883C806382320C00920A7
:10F970002DE9F0410546FFF7B9FE00F017FF164BE1
:10F9800001221A60154F5A60154E04339846012023
:10F990000146FFF7D3FD3B6813B10023C8F80030E0
:10F9A0003468002CF3D10F48FFF772FF064640F28F
:10F9B0009E20FFF74DFF2146286040F2DA20FFF736
:10F9C0004DFE0A20FFF778FD00F0F2FEFFF7C2FEC1
:10F9D0003046BDE8F08100BF80070842C8063823E2
:10F9E000E8063823CC2601002DE9F0411746804671
:10F9F0000E4602F07F04FFF779FE00F0D7FE234B9E
:10FA000001251D60032043F8045CFFF755FD3B060C
:10FA100005D51F4A10680028FCD1012101E02846C5
:10FA20002946FFF7BDFD1B484146FFF73FFE6CB17D
:10FA30000A20FFF741FD00F0BBFEFFF78BFE164BDF
:10FA40001868003018BF0120BDE8F0814FF4027043
:10FA50003EB101212246FFF7D5FD4FF40270214649
:10FA600006E031463246FFF7CDFD4FF4027001212A
:10FA7000FFF7F4FD0320FFF71FFD0549064A0B6859
:10FA8000002BD5D11368002BF9D0D1E784070842A9
:10FA9000EC06382360250100C806382338B5054632
:10FAA000FFF724FE104A1368002BFCD00F4B0124F3
:10FAB0001C6020460021FFF773FD29460C48FFF724
:10FAC000F5FD00210A4640F2BE50FFF79BFD21469E
:10FAD00040F2BE50FFF7C2FD0520FFF7EDFCBDE888
:10FAE0003840FFF737BE00BFEC06382380070842D6
:10FAF0003C2701002DE9F04705468846FFF7F6FD53
:10FB0000204A1368002BFCD01F4A012010600021FE
:10FB1000FFF746FD05EB08094FF4D7765FFA89F940
:10FB2000EBB2994518D015F8017B06F5916A344679
:10FB3000204607F080010022FFF764FD204607F011
:10FB4000400104F59174FFF789FDBF005445FFB2F1
:10FB5000EED106F26456E3E740F2645303FB08F883
:10FB6000002108F1B4080A464046FFF74BFD404625
:10FB70000121FFF773FD0520FFF79EFCBDE8F0476C
:10FB8000FFF7E8BDEC063823800708420B4B002244
:10FB90001A600B490B4A0B6813B91368002BFAD093
:10FBA000084B1B684BB9054B01221A600449054AF2
:10FBB0000B6813B11368002BFAD070478007084216
:10FBC000EC063823C80638232DE9F8430746FFF72B
:10FBD0008DFD00F0EBFD1A4B00209A68194B0A329C
:10FBE0001A6001460122FFF70DFD782440F648080F
:10FBF00017F8016B04F5F0792546284606F0010157
:10FC00000022FFF7FFFC284606F002017835FFF7D7
:10FC100025FD4D454FEA9606EFD104F5FA744445AB
:10FC2000E6D1204600220121FFF7ECFC204601210D
:10FC3000FFF714FD00F0BCFDBDE8F843FFF78ABDF7
:10FC400000800040CC11001038B5FFF74FFD0B4C81
:10FC500000F0ACFD0A20FFF72FFC012000212060FE
:10FC6000FFF76CFC0648FFF713FE002305462360F0
:10FC700000F09EFDFFF76EFD284638BD8407084260
:10FC80009426010002494FF4E672FFF7A9BD00BFB8
:10FC90002426010002494FF40272FFF7A1BD00BF04
:10FCA0000826010038B50546FFF720FD00F07EFD6F
:10FCB0000F4B01241C6020460021FFF771FC2946F0
:10FCC0000C48FFF7F3FC40F2771500210A4628465E
:10FCD000FFF798FC21462846FFF7C0FC0A20FFF7F3
:10FCE000EBFB00F065FDBDE83840FFF733BD00BF1A
:10FCF000800708422027010010B5FFF7F7FC00F04D
:10FD000055FD0D4B01221A600C4A1368002BFCD0E4
:10FD100000210120FFF744FC0948FFF7B9FD00214D
:10FD20000122044640F21220FFF76CFC00F040FD77
:10FD3000FFF710FD204610BD80070842EC0638236F
:10FD40007C250100F0B5174B1749184D02240122FC
:10FD500010F0010608BF1E6000F0020618BF1A600E
:10FD600006F0FF070EB10A6000E00F602E68002E5B
:10FD7000FCD000F0040606F0FF070EB11A6000E0A8
:10FD80001F6000F0080606F0FF070EB10A6000E0F1
:10FD90000F602E68002EFCD1013C4FEA1010D7D125
:10FDA000F0BD00BF8007084284070842C806382318
:10FDB000F8B5114E114F042400253368002BFCD0F8
:10FDC0000320FFF779FB3B68003318BF012343EAA8
:10FDD0004505EDB23368002BFCD10320FFF76CFB27
:10FDE000064B1B68003318BF012343EA4505013C5D
:10FDF000EDB2E2D12846F8BDE8063823EC063823F8
:10FE000008B50A4B1B687BB1094B1B78022B08D144
:10FE1000FFF76EFD074B1870FFF76AFD064B187071
:10FE200008BD064B00221A6008BD00BFC806382373
:10FE300075190010841900107C19001084070842FD
:10FE400008B5084B1B78012B0AD1074B1B683BB147
:10FE5000FFF7AEFF054B1870FFF7AAFF044B1870B1
:10FE600008BD00BF75190010E8063823841900107A
:10FE70007C190010144B002210B514491A60144A62
:10FE80000B6813B91368002BFAD0114B1C68B4B976
:10FE9000FFF72CFC00F08AFC0B4B01201860214678
:10FEA000FFF77EFB0B48FFF7F3FC04461420FFF737
:10FEB00003FB00F07DFCFFF74DFC204601E04FF610
:10FEC000FF7000B210BD00BF80070842EC06382367
:10FED000C80638234026010070B50646FFF706FC29
:10FEE00000F064FC154B00221A601549154A0B6896
:10FEF00013B91368002BFAD0124B1B68C3B90F4B10
:10FF000001241C6020462146FFF718FB0D4B1D689D
:10FF100075B90D483146FFF7C9FB4FF4F070214623
:10FF20002A46FFF76FFB4FF4F0702146FFF796FB70
:10FF300000F03EFCBDE87040FFF70CBC84070842AF
:10FF4000E8063823C8063823B425010070B50646F4
:10FF5000FFF7CCFB00F02AFC0E4B01241C600320B1
:10FF600043F8044CFFF7A8FA20462146FFF718FB98
:10FF7000094B1D683DB909483146FFF797FB14202E
:10FF8000FFF79AFA2C4600F011FCFFF7E3FB20463E
:10FF900070BD00BF84070842C806382374270100DB
:10FFA00001480C21FFF790BCB026010001480C214C
:10FFB000FFF78ABCE826010008B503491322FFF7C2
:10FFC000F3FB002008BD00BF9825010008B50349D8
:10FFD0001622FFF7E9FB002008BD00BF5C260100E8
:10FFE00008B503490C22FFF7DFFB002008BD00BF66
:10FFF0000427010001481421FFF766BC78260100A0
:020000021000EC
:1000000001481421FFF760BCD025010001480C21F4
:10001000FFF75ABC5827010008B503491622FFF71D
:10002000C3FB002008BD00BF9027010008B50349AD
:100030000F22FFF7B9FB002008BD00BFEC2501002F
:10004000014B5869C0B2704740C00920044B5A693F
:1000500022F0FF02104358610120FFF72DBA00BFC4
:1000600040C0092020B9034B9A6942F0FF029A610F
:10007000704700BF40C0092038B5044C4FF40065FC
:10008000E5610220FFF718FAA56138BD40C00920DC
:1000900010B50C4A1368591C11600B4918780B688D
:1000A000C0B2013B0B6063B9084C23689B6843B145
:1000B00023601C685B680C601360054B1A78013A7A
:1000C0001A7010BDF0110010EC110010DC110010BE
:1000D000D8110010094A1368591C1160084918709A
:1000E0000B68013B0B6043B9064803689B6823B16A
:1000F000036018685B68086013607047F0110010B7
:10010000EC110010DC11001010B5424C636822465F
:10011000282B2AD00CD8102B19D004D8002B69D04A
:10012000082B14D010BD182B33D0202B15D010BDA8
:10013000402B36D004D8302B0FD0382B2DD010BD0B
:10014000502B3CD0582B4BD0482B61D105E0324B83
:100150001B7893602823936110BD304B01221A70E5
:100160002C4B10221A60282227E02D4B1B785BB104
:100170002C4B1B7843B9284B1A7842F001021A70B5
:1001800020232360082329E0274B224C1B68002BE7
:100190002AD0FFF77DFFA0601FE0202323601823F3
:1001A0001CE0214B1B68012B2CD1204B1B689B684A
:1001B00043BB0423A361174B28229A6110BD1A4B3D
:1001C0001B68012B21D1194B1B689B68EBB90423D9
:1001D000A361A068C0B2FFF77DFF2823A36110BD13
:1001E000A068C0B2FFF776FF102323602823A36125
:1001F000042204E0102323602823A3610322074B79
:100200001A7010BD04231360D5E704232360E0E7D0
:1002100010BD00BF00C00540F5110010F611001020
:10022000D9110010D8110010EC110010DC110010D1
:100230000E4B012200211A6059600D4B4FF4FA71E8
:10024000196159610B494FF4006008600A490A605E
:100250002C229A61A3F540339A6E42F4C0129A663A
:100260005A6842F470725A60704700BF9835F8437C
:1002700000C0054000E100E01800B84210B50F4C86
:100280000023207048680E4C0E4A206008680E4C0F
:10029000137020600D4803700D4803700D4B1960FA
:1002A0000D4B0121196013780BB930BFFBE7054BEB
:1002B0001878043818BF012010BD00BFF5110010D8
:1002C000F0110010F6110010EC110010D9110010FF
:1002D000D8110010DC1100101400B84210B5054C04
:1002E0002170054981E80C000449BDE81040FFF782
:1002F000C5BF00BFF4110010E01100101400001081
:1003000007B502AB03F8012D0122FFF7E7FF03B0A9
:100310005DF804FB104B10B500241C700F4C00F06E
:10032000FE00207048680E4C206008680D4C20606C
:100330000D4C012020700D4C22700D4A11600D4AA9
:1003400010601A780AB930BFFBE7034B18780438FD
:1003500018BF012010BD00BFF6110010F5110010EC
:10036000F0110010EC110010D9110010D81100107C
:10037000DC1100101400B84210B51C46044B197073
:10038000044B054983E814000122FFF7C3FF10BDA9
:10039000F4110010E01100101400001007B5002245
:1003A00002AB03F8012D0122FFF7E6FF10B99DF81B
:1003B000070001E04FF6FF7000B203B05DF804FBE8
:1003C000124A01231360124A136042F8043C114A96
:1003D0001360114B114AD9680A43DA60104A516917
:1003E00041F400615161116841F4006111601A6FBC
:1003F00042F400621A671A6F42F0FF021A67A3F50F
:100400007E535A6B42F480725A63704780071042E1
:10041000840708428407104200C00240F030FC0FFD
:1004200040C0092010B50F4B0F4C1A7A12F0010F83
:100430000ED0596C0D4A914208D19A6C0C4B9A42DD
:1004400004D10C4800F0C3FA022305E00A4800E09A
:100450000A4800F0BCFA01232370BDE8104000F008
:10046000B8BA00BF00400240851B0010EFBEADDEF1
:1004700031EAE2FCAC270100B7270100D3270100D5
:10048000144B1B78022B07D0134B1A6802609A8812
:100490009B79828083717047104B93F82020027003
:1004A00093F824200178427093F82820827093F802
:1004B0002C20C27093F8382002719A8F92B26C3A55
:1004C000427193F83020827193F820209142E4D158
:1004D000704700BF851B00105328010000400240F8
:1004E000104B02221A72017883F82010417883F8A9
:1004F0002410817883F82810C17883F82C100179B2
:1005000083F83810417901F26C719987817983F809
:100510003010012119720449596404499964044B4B
:100520001A70704700400240EFBEADDE31EAE2FCD7
:10053000851B0010094B01221A60094B07221A6023
:1005400008B9062200E0FA221A6102225A60054A1E
:1005500001231360044A1363704700BF5035F8430A
:1005600000000340F418F84300400050034A1368A9
:10057000002BFCD0024B9860704700BF84016042A2
:100580000000034010B50A4A1368002BFCD109484B
:10059000094C0268084B07490AB1A368F9E7FF2232
:1005A0009A600A68002AFCD09868C0B210BD00BFEB
:1005B00090016042880160420000034010B5064B84
:1005C000064A0144884206D01C68002CFCD010F872
:1005D000014B9460F6E710BD8401604200000340C7
:1005E000F0B52D4A1368002BFCD12C4A2C4C136813
:1005F0000BB1A368FBE78B0705D00B46294C274AB4
:10060000274DFF2623E010F00304F6D1264B274D9B
:1006100001229A601A61C3F80051C3F8040141F045
:100620000460C3F80841C3F80C0141F20700C3F8A5
:1006300010011B4BFF205A621A4A22E06BB917685F
:1006400027B1AF68013900F8017BF8D14BB9002917
:10065000F4D10FE01768002FF1D12768002FF9D0EF
:10066000EDE72768002FF2D01768002FEFD1013B8C
:10067000AE60EBE7F0BD0139986004D01468002C3F
:10068000F9D10029FAD10A4A136913F00103FBD109
:10069000034A5362F0BD00BF90016042880160428E
:1006A0000000034084016042004000500800034005
:1006B00000410050074A1368002BFCD0064B002273
:1006C0005A6008B9062200E0FA221A6102225A6032
:1006D000704700BF8001604200000340064A136873
:1006E000002BFCD0054B00F0FD0001284FF040022C
:1006F0000CBFDA619A6170478001604200C0092036
:1007000072B670471B4B01211A6822F4704242F402
:1007100080421A60184A116018490A68002AFCD001
:10072000174A0120C3F80C01AA21C3F884205522DE
:10073000C3F88C10C3F88C20C3F88000C3F88C1069
:10074000C3F88C200B490222C3F80421D1F8882079
:10075000084B5201FAD50322C3F88020AA22C3F81D
:100760008C205522C3F88C20064B4FF400121A60DF
:10077000704700BF00C00F401434F8431834F843EA
:100780001800010000E100E030BF704772B64FF082
:1007900080434FF480725A604FF000421A61032286
:1007A0001A70AA221A7255221A72FEE772B67047A0
:1007B00062B67047044B1B6823B1044B10221A60C9
:1007C000FFF71EBB704700BF1000104200800040C2
:1007D000044B1B682BB110224FF040231A60FFF727
:1007E0002FBB70471000084208B50B4B1B6813B9AC
:1007F0000A4B1B6823B10A4B01221A6000F0A2FFCA
:10080000084B1B6833B1084B01221A60BDE8084051
:10081000FAF704B908BD00BF0011504280105042E1
:100820008011504220155042A0155042014B012228
:100830001A60FEE758033823014B01221A60FEE7D5
:1008400058033823014B01221A60FEE7580338236E
:10085000014B01221A60FEE758033823F0B51A4B0A
:100860009A68D1072FD402F00E02023A0A2A2AD837
:10087000DFE802F006292629282929292929260026
:10088000124B13481968026891421CD0114C0E4D4E
:10089000102219461F680668B74209D0013A07D0EE
:1008A0000E68A65D2E700E680136F6B20E60F1E796
:1008B0001A6803689A4206D1074B00221A60F0BDFD
:1008C0001B78F0BD1B7DF0BD00C00040F81100108A
:1008D000FC120010FC1100108400184230B50C4BC3
:1008E0000C4A196814681A6801319442C9B205D1DA
:1008F000094A126812B1094B187030BD084A002429
:1009000014601C68074D196001232855136030BD21
:10091000FC120010F81100109402184200C00040B0
:1009200084001842FC1100100D4A012313600D4A87
:100930000021136051600C4A832010733620107020
:100940000A48117101601372094A1360094B202291
:100950001A60094B1A6842F050021A60704700BFD3
:100960008C18F8431835F84300C000409C01184229
:100970008400184200E100E000C0024010B50446C7
:100980000009092894BF30305730FFF7A7FF04F063
:100990000F00092894BF30305730BDE81040FFF7F2
:1009A0009DBF00000348044902680B689A42FBD1CE
:1009B000704700BFF8110010FC12001010B5441E63
:1009C00014F8010F10B1FFF789FFF9E710BDFFF729
:1009D000F5BF08B50D20FFF781FFBDE808400A20EC
:1009E000FFF77CBF2DE9F8438846174646180024D8
:1009F00004EB0805BC42A8B242D2000AFFF7BEFFD2
:100A0000E8B2FFF7BBFF7C20FFF768FF2020FFF76D
:100A100065FF00252B19BB4203DA705DFFF7AEFFBF
:100A200005E02020FFF75AFF2020FFF757FF202086
:100A30000135FFF753FF102DECD17C20FFF74EFF5F
:100A400000252B19BB420DDA337806F10109A3F119
:100A50002000C0B25E2894BF18462E20FFF73EFF4C
:100A60004E4602E02020FFF739FF0135102DE8D176
:100A70007C201034FFF732FFA4B2FFF7AAFFB7E7DC
:100A8000BDE8F8830C4B1A7842F02002702A0DD092
:100A900004D8642A0ED1002018707047732A03D03E
:100AA000752A07D1032202E0012200E002221A7017
:100AB0000020704701207047A41700100B780370C6
:100AC00012238380002070470A46007800211023FB
:100AD000FBF78CBA0A46002111741023FBF786BA83
:100AE0001F20F8F79FBB000008B50B4A2123FBF736
:100AF0007DFA01280ED80ED007490223585C1A4609
:100B0000202803D1044B0020985408BD01330F2B3B
:100B1000F4D1F7E7FF2008BDA4170010F7B5174B75
:100B2000174601221A608D8B044629460078FFF78C
:100B3000DBFF0646E0B921232946114A2078FBF75E
:100B400055FA104820211022F3F7BCFD0C4833461B
:100B50000133FA1812F8011C11B11A189173F7E752
:100B60000123009320782946054A2123FBF766FAE2
:100B700003B0BDE8F040FEF767BB00BFB40B3823FD
:100B8000A4170010B317001073B58E8B04460D46E2
:100B900000783146FFF7A8FFA8B90C492846F3F7BB
:100BA00055FE29462046FAF76DFD094A2D2313709C
:100BB0000123207800933146FBF740FAD0F1010081
:100BC00038BF002000E0FF2002B070BDA617001063
:100BD000A41700102DE9F04F044698460078604BAA
:100BE0001746702202FB003292F83C208DB012F0C2
:100BF000020F0D46994601D11A2007E09DF85830A2
:100C0000CBB1898BFFF770FF18B13E20F8F70AFBD4
:100C1000A3E0FFF737FF0028F7D105F12000514985
:100C2000F3F714FE01230093204629463A46434633
:100C3000FBF79CF891E0084600F02EFA08B121205D
:100C4000E4E794F800B0DFF820A1122658463146B8
:100C5000FFF74AFF10B1FF2807D17EE09AF8003075
:100C60002D2B02D02136B6B2F0E7112E75D93E48B1
:100C70002021212207F00707F3F724FD032F6CD86A
:100C8000DFE807F002040608442204E0532202E0F1
:100C9000502200E05522344B334F1A703A233A4623
:100CA00002F8013F302107F1090302F8011F9A42BF
:100CB000FBD14FF0000A87F80AA02378702000FBD0
:100CC0000390284903AACDF82CA0FCF7A1FC60B939
:100CD000264A302112F8013C0133DBB2392B02F8ED
:100CE000013CEAD902F8011DF4E7022835D10022BF
:100CF0000132AB1813F8013C13B1B9188B73F7E745
:100D0000184905F12000F3F7A1FD2023BB723A2317
:100D1000BB730D23FB77DFF850900A2387F8203050
:100D200001272078009731464A462123FBF786F9B0
:100D300098B900904346204629460F22FBF716F843
:100D40000B4B1B784BB12D2389F80030207800978E
:100D500031464A463B46FBF771F90DB0BDE8F08FCE
:100D6000C4190010A6170010A4170010AE17001029
:100D700072190010F0B5324E8BB005460C4606F1E4
:100D80000F07A9882878FFF7AFFE014620B1FF289A
:100D900014BFFF20012050E020463022F3F792FCE0
:100DA000AB88A383AB882133AB80FFF76BFE0028B1
:100DB000E7D10323E37633786374224B13F80129D8
:100DC000202A02D1BB425870F8D11F4B224603F1B2
:100DD000100153F8040B8B4242F8040BF9D1637CE9
:100DE0001BB32A78194B702000FB0230184901AA66
:100DF000FCF70EFC30B10228C3D00121FAF7EEF85F
:100E000001201AE0134A019B93429DBF03F1FD01AB
:100E1000FE22B1FBF2F24FF6FF126282FE22B3FB1A
:100E2000F2F102FB1133237500E0638252236375F4
:100E30000823A3751F23E375002040B20BB0F0BD5B
:100E4000A4170010C2170010B3170010C419001027
:100E5000A6170010020BF80070B505460C46007886
:100E6000898B1646FFF740FE20B13E20BDE870405A
:100E7000F8F7D8B9FFF706FE0028F6D104F12000F4
:100E80000449F3F7E3FC284621463246BDE87040AA
:100E9000FAF744BAA61700102DE9F041344CFFF7D9
:100EA0002FFC2368334E43F0C25323604FF0C053EE
:100EB000A3614FF48003E3612F4B304F1A68012583
:100EC00042F400521A604FF400529A6135603D605E
:100ED000FFF72AFD2846FFF72DFBFEF789FAFFF7FB
:100EE0006FFAFFF7A5F9FFF70DFCFFF761FCF3F7C9
:100EF000A1FDFDF761FE00F035FB00F02FFCF7F7D8
:100F0000ABFC0020FAF7ECFFF7F766FCF5F7BCFE48
:100F10001B48FFF75CFD1B4B1878FFF72FFDFFF711
:100F200058FD194B194A1D605169616989021CD429
:100F30001748DFF864E0DFF864C0984653696169D8
:100F400013F080710ED0036813B9CEF8005000E0A2
:100F50003D60DCF8003013F0FF0F14BF3560C8F8B7
:100F60000050EBE70B4B1A781970FDF75BFE00BFE2
:100F700000C00920B40B382340C009206C0338237B
:100F800030280100BD190010340B382320C009207F
:100F9000800238238C1B0010EC0338238402382392
:100FA000034BFF221A70034B00221A60704700BFE8
:100FB000001300100413001070B50C4B1B78834213
:100FC00011D10B4B0B4D1C6814260023A3420AD0F1
:100FD00006FB03F25059884203D1064810440430FE
:100FE00070BD0133F2E7002070BD00BF0013001098
:100FF0000413001000C007202DE9F041124D904667
:101000002B6840F26662934204460F461AD00F4E98
:101010003378834202D0FFF7C3FF34702E68142365
:1010200073430B484246C418C750043408F11007F4
:1010300010685168234603C30832BA421C46F7D1F0
:1010400001362E60BDE8F08104130010001300107B
:1010500000C00720A0F16103DBB2192B01D82038B2
:1010600005E000F13F03DBB2192B01D88038C0B294
:101070007047000010F8043B054A702101FB032370
:1010800003C8303383E80300024B01221A70704713
:10109000C4190010841B0010013810F8013F53B12F
:1010A00003F0FD023D2A08D003F0F702222A04D003
:1010B0002C2BF2D101E01846704701207047000048
:1010C00070B5164A1378FF2B06D0036819782129CA
:1010D00002D159783A2903D00023114D0A2607E09E
:1010E00002330360107870BD202A0ED101310160F7
:1010F00001682C680A78144464786407F4D5734353
:10110000303ADBB21344DBB2F0E7402AEED013B939
:10111000044B187870BD013BD8B270BDFC180010AC
:1011200000000010C01900102DE9F04791468846D4
:10113000451CC24618F8014B6E1E002C3DD0B9F17B
:10114000000F09D015F8010CFFF784FF0746204671
:10115000FFF780FF044601E015F8017C2A2F02D03A
:101160003F2F28D025E01A4B1B78DD0629D53046C5
:10117000F3F7CAFB04465046F3F7C6FB3444504429
:10118000851E023C013EB4421BD0B9F1000F07D0CE
:101190006078FFF75FFF07466878FFF75BFF01E0C5
:1011A00067786878874201D03F2F0DD1013D013C1F
:1011B000E9E7A74208D10135BBE733780BB12A2B09
:1011C00002D10120BDE8F0870020BDE8F08700BF14
:1011D000F31700102DE9F84F9DF828600B9C81460D
:1011E0000D469246984606F0070B99F800301D49C7
:1011F000702202FB03139B6B48461B6B21469847EA
:10120000074660BB637CBBF1000F03D086EA030294
:101210005107EAD19A0601D5B306E6D54DB1E27E73
:101220002846012A18BF00222146FFF77DFF00282B
:10123000DBD0BAF1000F07D004F1150051460622A9
:10124000F3F7BAF90028D0DBB8F1000F07D004F1AA
:10125000150041460622F3F7AFF90028C5DC78B245
:10126000BDE8F88FC4190010F7B516461F46104A9E
:1012700003780D46702101FB03239B6B0446DB6A58
:101280000C4821469847024660B98DE8C0000948DD
:1012900029461346FFF79EFF041E05DA3E20F7F7A6
:1012A000C1FF01E0012000E0204640B203B0F0BDE4
:1012B000C41900100C1300102DE9F04F8FB00190ED
:1012C0000D4614461F462BB93A21F3F745FA00287C
:1012D00000F0868001A8FFF7F3FE4C4B1B78834299
:1012E00001D84A2036E04A4B2A464FF0700A02F8ED
:1012F000040B0AFB0030303003C882E80300019E73
:10130000984632782F2A02D14FF0000937E0304654
:101310003A21F3F721FA206008B9266073E0013022
:1013200020606DE02F2E06D03A2E04D09B4613F895
:10133000016B002EF6D18BF80090284601992022EF
:1013400002ABFFF791FF00282DD0324B1B783E2BCC
:1013500058D12720F7F766FF54E0531C019310780B
:101360002F2811D150782F2814D12B788DF8089080
:101370000AFB03839B6B28469B6B02A99847019A43
:101380001378002BE9D139E03A2838D00028F6D17B
:10139000226038E03A2803D00028C7D1236032E029
:1013A000023222602CE09DF8193003F00703062B6F
:1013B00009D0002FCDD0002ECBD10198FAF7A8FA92
:1013C0000028C6D01AE02B7828460AFB03839B6BC3
:1013D00002A99B6B98478BF80060CDF804B0CEE76C
:1013E0000D4B70211A7805F8042B1B78084A01FB75
:1013F0000323303393E8030085E80300019B236057
:10140000002000E001200FB0BDE8F08FC1190010EE
:10141000C419001072190010C019001070B50346ED
:101420001A681178202902D101321A60F8E70A4DB2
:1014300000200A261A6829681478214449784C0744
:1014400008D5511C70431960127880B2303A1044AC
:1014500080B2EFE770BD00BF0000001038B5054650
:1014600008460C46FFF7DAFFC0B20C28687077D840
:1014700023685A1C22601B782F2B71D12046FFF75E
:10148000CDFFC0B21F28A8706AD823685A1C2260FA
:101490001B782F2B64D12046FFF7C0FFC0B24F2826
:1014A00098BF6430287023681A780AB12C2A03D1B7
:1014B0000020E87028713BE05A1C22601B78202B2A
:1014C0004ED12046FFF7AAFFE87023685A1C22601D
:1014D000EA781B78172A43D83A2B01D02E2B3FD11C
:1014E0002046FFF79BFF28712268531C236029794F
:1014F00013783B2934D82C2B18D005D8B3B1202B26
:101500002ED100236B7115E02E2B01D03A2B27D161
:101510002046FFF783FFC0B23B28687120D82368BC
:101520005A1C22601B78202B1AD103E02260002075
:10153000687138BD23685A1C22601B78412B04D087
:10154000502B0DD1EB780C33EB70EB78172B07D8C1
:1015500023685A1C226018784D3818BF012038BD06
:10156000012038BD10B5074CF6F786FF23780BB184
:10157000042204E0FEF756FF237813B10322024B46
:101580001A7010BD851B001008130010054B1B7846
:10159000032B03D0042B03D1F6F7D8BEFEF770BFA0
:1015A000704700BF0813001007B56846FFF7EEFF4D
:1015B0009DF803209DF80230120442EAC3229DF8F0
:1015C00001309DF8040042EA43129DF800300130DA
:1015D00042EA53029DF80530503B42EA436343EA36
:1015E000405003B05DF804FB054B1B78032B03D080
:1015F000042B03D1F6F7F6BEFEF772BF704700BFAB
:1016000008130010EFF3108372B6024A106883F3D8
:1016100010887047941B001070B501F00704034652
:10162000A0B260B1FF2646FA00F0CD085D5D083A31
:1016300021F0070122440831284052B289B2072A1A
:1016400008DDCC081C5D0831083A04EB002089B2A3
:1016500052B2F4E7002A08DDC9085B5C9040C2F191
:10166000080243FA02F2104470BD1CBF5242D0403F
:1016700070BD000008B50020FFF730F8054B0122CF
:101680001A60FEF77FFFFEF77DFFBDE80840FEF71A
:1016900079BF00BF700338232DE9F74F1446814608
:1016A00000208846F2F752FD210EF2F74FFDC4F3F9
:1016B0000741F2F74BFDC4F30721F2F747FDE1B212
:1016C000F2F744FD24BA400040F0010709F1010996
:1016D000DFF86CA0FFB20A265FFA89F94846FEF7E8
:1016E000FDFF0123CAF800304046FEF73FFF02A885
:1016F000042140F8044DFEF761FF3846FEF736FF3F
:10170000FFF780FF00F1320BFEF73CFF02060546B3
:1017100002D42B0710D506E0FFF774FFCBEB0000D7
:101720000028F1DBF5E77820013EFFF7D7F8FFF757
:10173000A1FF16F0FF06D1D1284603B0BDE8F08F17
:10174000F0033823034B1A68034B02B101221A70CD
:10175000704700BF80023823F01700100B4B402267
:101760009A611A6842F040021A60094B1A6842F402
:1017700028221A60A3F57E531A6942F001021A6109
:101780005A6942F001025A61704700BF00C0092047
:1017900000C00240064B1B683BB9064B1B6813F0A8
:1017A000FF0F0CBF0020042070470320704700BFCC
:1017B00080023823840238232DE9F743044608B118
:1017C0000320B7E0FFF7E6FF800700F1B0800120BB
:1017D000FEF770FF0325594FDFF86891A8460020F7
:1017E00087F8008089F80000FEF778FF544B01224B
:1017F0001A600A24FF20013CFEF7B8FE14F0FF0433
:10180000F8D1402122462046FFF746FF0646FFF763
:1018100031FF310601D501208CE0012E04D0013DBD
:10182000ADB2002DDBD1F6E7204648214FF4D5724A
:10183000FFF732FF01280ED101A80421FEF7D0FEE8
:10184000019B1BBA0193FFF715FF019BC3F3032311
:10185000012BB5D101E0FFF70DFFFFF70BFFFFF7FD
:10186000D1FE00F13206002077210246FFF714FF77
:101870000546FFF7FFFE012D28D169214FF0804278
:101880000020FFF709FF0446FFF7F4FE012C05D105
:10189000FFF7B8FE801B0028E5DB17E0B4B920464F
:1018A0007A212246FFF7F8FE01280DD802A840F859
:1018B000044D0421FEF794FE019B4FF0804212BAC2
:1018C0001A421CBF1F4B1D70FFF7D4FEFFF79AFE94
:1018D00000F13205002041214FF08042FFF7DCFE8D
:1018E0000446FFF7C7FE2CB1FFF78CFE401B002813
:1018F000F0DB90E77B2101222046FFF7CDFE054675
:10190000FFF7B8FE012D3FF65BAF204650214FF4A4
:101910000072FFF7C1FE0446FFF7ACFE002C7FF417
:101920007AAF2046FEF7C6FE044B02221A7020460C
:10193000FFF730FF03B0BDE8F08300BFF0170010E1
:1019400070033823091300102DE9F74F0E46174690
:10195000984648BB304B1A7802B97F020024E3B2A4
:10196000434523D207EB4429002504EB070A2A4B01
:10197000187810F0010003D000205121524601E0F8
:1019800051214A46FFF788FE90B9FFF73BFE00F170
:10199000320BFEF7F7FDFE2811D0FFF733FECBEB3D
:1019A00000000028F5DB03E0042031E000202FE0F8
:1019B000FFF760FE194B03221A70012028E04FF454
:1019C00000713046FEF70CFEFEF7DCFD0190FEF7DD
:1019D000D9FD314683464FF400720020F2F7CAFB6E
:1019E000019B4BEA03239BB2834208D00135582068
:1019F000EDB2FEF773FFFFF73DFE0A2DB7D1FFF7FB
:101A000039FE092D04F10104D7D806F50076A6E7C2
:101A100003B0BDE8F08F00BF09130010F0170010ED
:101A20002DE9F84F0F4615469A4600285AD1334BF8
:101A30001B6813F0FF0F58D1314B1A7802B96D02B1
:101A40000024E3B2534556D205EB4429002604EBAB
:101A500005082B4B187810F0010003D00020582106
:101A6000424601E058214A46FFF716FE834628B158
:101A7000FFF700FE234B03221A7039E0FE20FEF729
:101A800075FD38464FF40071FEF798FD39464FF466
:101A900000725846F2F76EFB8346C0F30720FEF74C
:101AA00065FD5FFA8BF0FEF761FDFEF76BFD00F060
:101AB0000F00052809D001365820F6B2FEF70EFFB8
:101AC000FFF7D8FD0A2EC4D103E0FEF75BFD002826
:101AD000FBD0FFF7CFFD0A2E04F1010408D007F573
:101AE0000077AEE70420BDE8F88F0220BDE8F88F4C
:101AF0000120BDE8F88F0020BDE8F88F840238236C
:101B000009130010F017001070B50D4686B014468A
:101B100008B1032046E0FFF73DFE8607F9D4002D0B
:101B20003FD1284649212A46FFF7B6FD10B1FFF7FD
:101B3000A1FD36E0FEF726FD0028FBD001A812210A
:101B4000FEF74EFDFFF796FD174B01A81B78DD074A
:101B500006D53A211622FFF75FFD0130850218E015
:101B60004E210322FFF758FD362106460C2201A81C
:101B7000FFF752FD2C21451C042201A8FFF74CFD64
:101B80003044C31FDBB2013BDBB2FF2B01D06D0041
:101B9000F9E7082323700223A370E3706560002037
:101BA00000E0012006B070BD09130010054A064B85
:101BB0005B69506903F0D073400000F48000184363
:101BC000704700BF00C0092020C009202DE9F04166
:101BD000FFF7ECFF354E364D3368364F984233D021
:101BE00029683A68521A12F1040F28D5324C22782B
:101BF000A04612F0800F03D0237803F07F0305E0A6
:101C000013F0A07F04D1237843F00403237016E07F
:101C1000D80107D4FFF7CAFFC10103D5237843F0E9
:101C20000103F3E733685A0209D4FFF7BFFFC3018A
:101C300005D598F8003043F0020388F800302B688F
:101C40003B60FFF7B3FF30602B6801332B601B4B09
:101C50001B78DC070AD5164B1B68180706D1184BF2
:101C60001A68D2F1010238BF00221A603B68296865
:101C70000F4A591A11F1040F15D5316801F0A071FE
:101C8000B1F5800F0FD111685B1A13F1C80F0AD597
:101C9000094B1978090706D4197841F088011970A1
:101CA0001268044B1A60BDE8F08100BF901B001061
:101CB000941B0010881B00108C1B0010BE19001014
:101CC000EC023823632910B509D96422B1FBF2F381
:101CD00002FB131103F130040470C9B201300A226F
:101CE000B1FBF2F303F1300402FB13133033047041
:101CF0004370023010BD020900F00F030A2000FB00
:101D00000230C0B270470A22B0FBF2F302FB1300AC
:101D100000EB0310C0B2704730B500B9106803463D
:101D200018781C46884203F10103F9D060B12046BF
:101D300005780346013025B18D42F9D10021197093
:101D400003461360204630BD30BD10F8013BCBB1D7
:101D5000A3F14102D2B2192A0CD9A3F16102D2B285
:101D6000192A02D8203BDBB209E003F13F02D2B2CC
:101D7000192A01D8803BF6E77E2B08BFFF2300F825
:061D8000013CE2E77047A0
:101D88000020202020202020202028282828282043
:101D9800202020202020202020202020202020203B
:101DA80020881010101010101010101010101010A3
:101DB8001004040404040404040404101010101093
:101DC800101041414141414101010101010101015D
:101DD80001010101010101010101010110101010AF
:101DE800101042424242424202020202020202022F
:101DF8000202020202020202020202021010101083
:101E080020000000000000000000000000000000AA
:101E180000000000000000000000000000000000BA
:101E280000000000000000000000000000000000AA
:101E3800000000000000000000000000000000009A
:101E4800000000000000000000000000000000008A
:101E5800000000000000000000000000000000007A
:101E6800000000000000000000000000000000006A
:101E7800000000000000000000000000000000005A
:101E88000000000012014690A2060300015900005C
:101E980012012390A20A030091580000280350045D
:101EA80016010100B95900000101000416010100E2
:101EB800E157000085520000755E0000A14D00004A
:101EC8004961000059540000515400004954000071
:101ED800155E000055500000BD5000000D64000064
:101EE800E54D0000BD540000C161000081510000B3
:101EF800895300004155544F535741502E4C535469
:101F08000023504554534349494155544F53574171
:101F1800502E47454E00FFE20053595354454DA0FB
:101F2800A0A0A0A0A0A0A0A0A00000000000000009
:101F3800000000000D009F9C0300B0DA04003B97EE
:101F48000400387E0400301B05000E8B0500309914
:101F580006008102180896C11809692E010081DD62
:101F680007003E391700015A090079B90A016924A6
:101F78000B01794D0C01BCB20C0172B20C01EDDA07
:101F88000D028D3F0E0247C90E0340F10F047E7308
:101F980010045A75110420291104E9181105049830
:101FA8001105F54811055613110585E81105CA4EA6
:101FB8001105F6DB1105ABE41105E56D1105FF30E0
:101FC8001105E7461105532211056AC212060C5580
:101FD80012065B8213075B2413072170130737D59A
:101FE800130735F61307C143140070481500252957
:101FF8001600A6121900920C08000000000000004C
:102008000303030085990000000000009A050400FE
:10201800699A00000000000000040400699A0000AA
:10202800000000009C0505002D9B0000000000003A
:102038009A0505002D9B000000000000030406001F
:10204800699A0000010000007F051800C19B00008C
:102058000000000000070100419C00000000000093
:1020680036030700DD9D0000000000000003170094
:10207800659E00000000000000050800DD9E0000CD
:1020880000000000A901090021A0000000000000D4
:1020980057040A00C9A300000000000070040B00E8
:1020A800C9A3000001000000E2030C004DA10000DC
:1020B80000000000DC030C004DA10000000000003F
:1020C800FF030D004DA10000000000000F040E00EA
:1020D8004DA100000000000000040F00BDA4000096
:1020E8000000000000041000BDA400000100000072
:1020F8000003110059A500000000000000041200B0
:1021080059A50000000000000003130059A50000B5
:10211800000000000005130059A5000000000000A1
:102128000003140089A70000000000000005150046
:1021380051A9000000000000F4051600B9A900002C
:10214800000000000005190085AC00000000000038
:10215800000000000000000000000000A0FE0DEDDF
:10216800C6E534B1FEFF000000000000436F64655F
:10217800206578656320617420002C204352432039
:10218800004D2D572043524320726573756C743A85
:1021980020002078782F78782F78782078783A7807
:1021A800783A787820784D0D00000A002A04FF66F6
:1021B8000B004F04FF660000000000000000000054
:1021C80000000000A1FF0000B9FF0000ADFF000003
:1021D800CDFF0000ADFF0000E1FF0000F5FF0000AB
:1021E80019000100ADFF0000E1FF0000010001003F
:1021F800190001000D0001002D0001000000000081
:1022080085FC00000000000095FC000053554E2E90
:102218004D4F4E2E545545535745442E544855520C
:102228004652492E5341542E004453333233312001
:10223800006E6F7420666F756E6400696E76616CEF
:10224800696400454550524F4D46532020202020B8
:1022580020202000454550524F4D46532020202035
:10226800202020200000000011870000C186000007
:102278000785000039860000C9840000A585000094
:1022880091850000D5850000178500000D850000A8
:10229800D1850000C185000021850000E5BF000050
:1022A800E98400001786000045452032410080205F
:1022B8004F4B810053205343524154434845448275
:1022C800080994959697989B0103999C02039A0292
:1022D8002050524F54454354204F4E9D05494420A9
:1022E8004D49534D415443489E9FA0A1A253594E76
:1022F80054415803A7BE0004464F554E44B2070444
:1023080050524553454E54B34F564552464C4F577D
:1023180020494E2007B4000B4C41524745BC0220CF
:10232800002006BD000406BF0020455849535453F9
:10233800C0002054595045204D49534D41544348FD
:10234800C10C424C4F434BC2C30A20545241434B29
:10235800204F5220534543544F52C60C4348414ED8
:102368004E454CC744495203C80546554C4CCA44CF
:1023780052495645040159CD0920080ACE4255460E
:102388004645520B534D414C4CCF494D4147452092
:102398000020494E56414C4944E3434C4F434B209F
:1023A800554E535441424C45FF8046494C45815255
:1023B80045414482575249544583204552524F5211
:1023C80084204E4F5420854449534B20864F504516
:1023D8004E875245434F52448850415254495449BC
:1023E8004F4E208953454C45435445448A494C4CEB
:1023F8004547414C8B20544F4F208C4E4F20FF5364
:1024080044324945432056312E302E30414C5048F5
:1024180041302D39382D4741413833393543002D66
:102428006C7063313736382D61726D32696563318E
:1024380000130D140F141100756E6B6E6F776E3AE2
:102448000D0A0031323853595354454D31004E4925
:1024580050504F4E0042554620455252004E455866
:102468005400130C140F1706180400001DB30000C5
:102478006DBD000009BE000085B600001DB7000054
:102488009DB7000099AE000075AF0000EFB80000DE
:10249800D9B80000E9AE0000E9B3000019B40000A3
:1024A800E9B6000099B9000071BB0000626F6F7453
:1024B800736563742E3132380043363446696C656F
:1024C8000001030507090E10121416181C1E4641B8
:1024D80054333200010401010000122253443249EE
:1024E8004543202020202020202020202220494B46
:1024F800203241000101000020202022535953546A
:10250800454D222020202020202020202020535903
:102518005320200001010000424C4F434B532046FA
:102528005245452E20202020202020202020202019
:102538002000000044454C534551505247555352D2
:1025480052454C43424D4449523F3F3F4E4154341B
:10255800312037312038312064000000C8000000E5
:10256800360100009A010000000204060103050775
:102578000000000078000000DC0000007C01000082
:10258800E00100000706030205040100FF00000047
:10259800B40000001801000086010000FE010000E0
:1025A80003020406010005070F0000008C0000006C
:1025B800DC0000002C0100007C0100000002040681
:1025C8000103050700000000AA0000001801000030
:1025D800C2010000620200000706030205040100B0
:1025E800FF00000046000000960000000401000003
:1025F8007201000000020406010305070000000044
:102608008C000000F000000054010000B801000038
:102618000002040601030507FF0000008C0000000B
:10262800DC0000002C0100007C0100000002040610
:1026380001030507FF0000008C000000F000000007
:102648007C010000E0010000070603020504010008
:10265800FF0000005A000000C80000004001000010
:10266800B801000003020406010005070F0000007E
:10267800A0000000040100009A0100001C020000F4
:102688000706030205040100FF000000AA0000007D
:102698002C010000A4010000080200000706030244
:1026A80005040100FF000000960000002201000060
:1026B800AE0100004E0200000406030205070100F7
:1026C800FF000000B90000003B010000A901000064
:1026D8002B0200000406030205070100FF000000AA
:1026E80096000000220100008B010000F9010000A3
:1026F8000406030205070100FF0000004600000071
:102708008C000000F00000004A01000000020406EE
:1027180001030507000000003200000082000000ED
:10272800D200000022010000000204060103050790
:102738000000000036010000580200007A03000083
:102748009C040000070503010604020000000000C5
:10275800960000000401000072010000E001000082
:102768000002040601030507FF00000064000000E2
:10277800C80000002C0100009001000007060302B9
:1027880005040100FF0000005A000000E6000000F8
:1027980072010000FE0100000302070601000504A3
:1027A800FF0000004C504320525443206F6B004CF4
:1027B80050432052544320696E76616C6964202826
:1027C8007369676E617475726529004C50432052B5
:1027D800544320696E76616C69642028646973616A
:1027E800626C656429000000590E0100D50B0100D8
:1027F800E10A0100890B0100D50A0100C90A01009C
:1028080099AE000075AF0000EFB80000D9B800001D
:10281800E9AE0000BD0A0100750D0100E5BF00002A
:10282800D5BF00001D0B01000D0A73643269656392
:1028380020312E302E30414C504841302D39382D22
:1028480047414138333935432023000000001F0732
:0228580052022A
:10285C00881D0100FFFF000002000000BC110010E9
:10286C00C011001001000000F4110010E011001064
:0400000300004109AF
:00000001FF
